:020000040000FA
:1000000000F80202ED6F0000113500008D42000083
:1000100000000000000000000000000000000000E0
:1000200000000000C04E0100084F01001135000023
:10003000000000000000000011350000897600007B
:10004000ED32000011350000113500000D70000088
:10005000954A0000996B0000A1340000953500001E
:1000600059180000951700001135000015350000E3
:10007000694A0000C98C00008D6F0000B96F000054
:10008000113500001135000011350000E579000040
:10009000057A00001135000011350000113500000F
:1000A000997E0000A37E0000EF320000A16E0000E8
:1000B00011350000016C000000000000000000008D
:1000C0000348854600F016FF0048004749CA000073
:1000D00000F8020230B50B46014600202022012420
:1000E00009E00D46D5409D4205D31D469540491B6C
:1000F0002546954040191546521E002DF1DC30BDB5
:1001000070B500242546002801DA01244042002968
:1001100001DA01254942FFF7DDFFAC4200D0404241
:10012000002C00D0494270BDF8B5002425460029B6
:1001300004DA0E46012400214042B141002B04DACA
:100140001E46002352420125B34100F0D1FC8C46EB
:1001500017461E46AC4203D0002540428D41AC46B6
:10016000002C02D0002657429E4161463A46334653
:1001700001B0F0BD03460B439B0703D009E008C95B
:10018000121F08C0042AFAD203E00B780370401C47
:10019000491C521EF9D27047D2B201E00270401CD5
:1001A000491EFBD270470022F6E710B513460A46F7
:1001B00004461946FFF7F0FF204610BDCAB2401EA4
:1001C0004178401C8A4202D00029F9D100207047B2
:1001D000421C0178401C0029FBD1801A704730B5C1
:1001E00004460020034600E05B1C934203D2E05C1F
:1001F000CD5C401BF8D030BD30B50546002003462D
:1002000000E05B1C934205D2EC5CC85C201A01D173
:10021000002CF6D130BD00000FB400B58DB00990B0
:100220000B9010A900200091C0430A9000200C9070
:1002300006480690064807906A4609A80F9900F0FC
:10024000C1FC0DB008BC04B018470000E50B00006D
:10025000050C0000FFB5002083B0009050680190AD
:1002600091691446002697680498884705460C99BA
:100270000698084305D009E0A169761C04988847D0
:100280000546216A284688470028F5D1681C03D016
:100290000198C00704D017E00020C04307B0F0BDAC
:1002A0002068011D2160006800900DE00198C007E2
:1002B00004D1009805700098401C0090A169761C3C
:1002C0007F1E049888470546002F1CDD681C1AD045
:1002D000069800280FD0E817C00E401941118A0077
:1002E00006994009511840012A1A096801209040D6
:1002F0000142DBD107E00C980028D7D1216A2846BB
:1003000088470028D2D0E169049888470C980028D3
:1003100007D1002E05DD0198C00702D10098002109
:100320000170A068B84204DD0C98002804D0002FAA
:1003300002D00120C043B1E73046AFE770B50646B2
:1003400011F020F9046805460A220021304600F029
:10035000C5FC2C6070BDF8B502464A40D40F42007F
:100360004B0052085B089A4202D2024608461146E8
:100370004A0023D0C30D4A00DDB2120EAD1A202D63
:1003800035DA49020126490AF6058A19002C00D0FF
:10039000524220214F1B1146B9402A411018C20D6C
:1003A0009A4221D0002C17D0012D08DCDA05801AE2
:1003B000D20F8019D207DBB200F0D0FCF8BDDA050D
:1003C000801A012340001B06C01880185A4280186A
:1003D000CA0F1043490007E04908C2071143DA0574
:1003E000801A80194008801800F0B0FCF8BD610048
:1003F0000122511A001BF7E70122D2075140AAE758
:100400000122D2075040A6E7024670B54A40D30FFA
:10041000DB0740002DD04A002AD0010E140E000246
:1004200012020919400A520A8418E501044654438D
:10043000000A120A2E045043A4194219200CC54385
:10044000AA18120C0125AD03521C521912047F394F
:10045000240400D0521C104301D44000491EC2B2F3
:100460000C06C0092018401C4008802A02D003E076
:10047000002070BD40084000002900DA0020184329
:1004800070BD70B502464A40D50F40004A00ED07E6
:1004900040085208002814D0002A12D0C40DD30DF1
:1004A00041020120C0055202490A520AE41A091801
:1004B00012187D34914201D3641C00E04900002CE5
:1004C00001DA002070BD0023914201D3891A034351
:1004D000400849000028F7D100290AD0914202D1F2
:1004E0000121C90705E0914201D2012101E001216A
:1004F000C943E005C018401900F028FC70BD000099
:10050000F0B507460846584087B0C00F0490480031
:100510000E46590040084908BC1A884105D23846A1
:1005200031461E4617460B46024658004008104307
:100530004CD0300D039040055900400D490D0590F9
:10054000401A0290402872DA18030121000B0905B5
:100550000843019004980092002805D00199524266
:100560000020884100920190029840210A1A0199C6
:10057000009800F0EDFA05460C466B4607CB00F0FC
:1005800008FBC0197141039A0E0D0023D71756407E
:100590001A467A40164344D0049A002A2DD0029A73
:1005A000012A039A15DC1205C01A9141012636056D
:1005B000001C7141D20F059ED20700930192029652
:1005C0002A46234600F010FC07B0F0BD38463146FD
:1005D000FAE71605224A0F46B218C01AB7410121A0
:1005E0000905001C4F4100187F4111461818794138
:1005F000E20F10436D19644113E0E2076D081543E3
:100600006408C2071443039A01261205C01A9141D7
:100610003605001C7141CE07400830434908C01818
:1006200051412A46234600F0D2FBCDE7FFE704986C
:1006300001224000C117121A00238B410498314651
:10064000C417381AA141EEE730B40124E40763402F
:1006500030BC55E730B40124E407614030BC4FE7BB
:100660000000E0FFF0B51FB488B00B990998002492
:1006700048400999C00F490049080991C0070B99E2
:100680000090490049080B9109990898A64608432B
:100690001CD00B990A98084318D0099801244000EF
:1006A000420D4800410D099824050003000B20432A
:1006B00009900B980003000B20430B9050181C4925
:1006C0004018002201901446104605E00020014623
:1006D0000DB0F0BD032801DA034600E003239C4679
:1006E000C11A0AAE0AE05F0008ADED5B4F00F75B90
:1006F0007D430027AA187C41491C5B1E6145F2DD41
:10070000410004AB5A522104120C0A43240C401C31
:100710000828DFDB01980290009970460191009053
:10072000059B049A0799069800F05EFBD0E700004D
:100730000DFCFFFFF0B50C465C4085B0E40FE4070C
:1007400003944C0000266408590094464908024668
:100750000296224321D062460A431ED06200570D02
:100760004A000E032303550D012402462C4924059B
:10077000781B1B0B360B4018234326436146009021
:100780001C46501AB44103D30098401C009002E06C
:10079000921800985B41002803DA0020014605B05A
:1007A000F0BD0020012109050746864611E0644698
:1007B0001D46141BB54106D36546521BB341744612
:1007C00007430C43A646CD07400849082843921822
:1007D0005B4105460D43EAD11046184313D06046ED
:1007E000194650407140084306D06046101AB34184
:1007F00006D20122002306E000220123DB0702E0EB
:100800000122D2435310009874460105381C6141FF
:10081000029C039D0019694100F0D9FABFE700006E
:10082000FD0300000122D207002800DB101A002976
:1008300000DB511A814201D8012070470020704727
:100840000122D207002800DB101A002900DB511A10
:10085000814201D201207047002070470122D20757
:10086000002800DB101A002900DB511A814201D355
:1008700001207047002070470122D207002800DBCA
:10088000101A002900DB511A814201D9012070475A
:10089000002070470122D207002800DB101A00292F
:1008A00000DB511A814201D10120704700207047BE
:1008B00010B5002904DB0C460121C9074042A141C3
:1008C000002B04DB1C460123DB075242A341801AA4
:1008D000994101D3012010BD002010BD10B50029A1
:1008E00004DB0C460121C9074042A141002B04DB77
:1008F0001C460123DB075242A341101A8B4101D34E
:10090000012010BD002010BDC217C10F504010B50E
:100910004018CA079623002100F020FA10BD10B538
:1009200000229623114600F019FA10BD0EB5C21729
:10093000C10F5040CA0740180021054B0293019295
:1009400000910A460B4600F04FFA03B000BD0000CC
:10095000330400000EB505490291002100910A46BA
:100960000B46019100F040FA03B000BD33040000D3
:100970003EB5CA17CB0F002450405140C01861410A
:10098000DA07054B0293019200942246234600F0B9
:100990002BFA03B030BD000033040000C20F410049
:1009A00040020123400ADB05D207090EC0187F2947
:1009B00001DA00207047962903DC9623591AC840B3
:1009C00001E096398840002AF4D040427047410047
:1009D00040020122400AD205090E80187F2901DA5F
:1009E00000207047962903DC9622511AC8407047B0
:1009F000963988407047000070B5CD0F4A00090352
:100A00000123090B1B0519430B4BED070024520D65
:100A10009A4201DA002070BD074B34339A4203DC5E
:100A20009A1A00F0A5F802E00449511888402C43B6
:100A3000F1D0404270BD0000FF030000CDFBFFFF7E
:100A400070B5CD0F4A0009030123090B1B0519439B
:100A50000D4BED070024520D9A4202DA00200146A8
:100A600070BD094B34339A4203DC9A1A00F080F8C7
:100A700003E0064BD21800F06BF82C43F0D00022B4
:100A800040428A41114670BDFF030000CDFBFFFFCD
:100A9000C20FD207400040080BD0C10D0723DB0175
:100AA000C91840020905400A1143C2084007114312
:100AB0007047002001467047CB0FDB07490010B597
:100AC000490802460A4307D00A0D07240903E40136
:100AD000090B121B002A01DC002010BDC900440FC5
:100AE0000C43C100E018D205801800F02FF910BDAA
:100AF000F0B51FB40646002082B00546402401919F
:100B000000901BE0019922460F46304600F030F875
:100B1000049A059B801A994110D310461946224623
:100B200000F016F8361A8F41019722460120002165
:100B3000009F00F00DF838184D4100902046641ECB
:100B40000028DFDC019B00982946324607B0F0BD43
:100B500010B5202A04DB0146203A9140002010BD48
:100B6000914020239C1A0346E3401943904010BD56
:100B700010B5202A04DB0846203AD040002110BDE1
:100B80000B46D340D0402024A21A91400843194676
:100B900010BD10B5202A06DBCB170846203A1041BD
:100BA000C1170B4306E00B461341D0402024A21A84
:100BB00091400843194610BD02681378511801602E
:100BC0001846704710B5D16004495161044911625B
:100BD00000211161114600F0ADF910BDB90B000004
:100BE000210F00004268002A08D001680B78491CD8
:100BF000002B03D0521E06C0184670470121C16069
:100C0000881E70474268002A0BD0C3680168002B19
:100C100007D183688B4204D0491E521C06C00020B5
:100C200070470020C04370470FB400B589B00A4632
:100C30000DA9009100230C99002ACB60234B069349
:100C4000234B079301D0042300E00023214A0292A2
:100C5000214A0892019302466B46002000F095FB62
:100C600009B008BC04B01847F0B585B007460020AD
:100C7000C04301901E46002015460C46009102918B
:100C800004903B466A46314604A8FFF7CDFF04991D
:100C900002466018002D05D0002901D0034600E06F
:100CA00023462B6000290ED0002A02DD00998142E4
:100CB00009D0001B019000943B466A4631460294DD
:100CC00004A8FFF7B1FF05B0F0BD0000E50B000080
:100CD000050C0000FFFFFF7F210F0000F7B5009C0F
:100CE0000F4600262578641C002D05D000F014F96D
:100CF0000068405DC007F5D12B2D02D02D2D18D0F6
:100D0000641E39462046029A00F06AFC002F04D087
:100D10003968A14201D10099396071050224002986
:100D20000BDA4042002803DD10F02CFC0460A00721
:100D3000FEBD012080020643E3E70028F8DA10F048
:100D400021FC04600048FEBDFFFFFF7F002904DA9C
:100D5000401C490001D140084000704770B4002495
:100D6000050C05D11024000402D1002921D0112442
:100D7000050E01D100020834050F01D10001241D28
:100D8000850F01D18000A41C002801DB4000641CF9
:100D9000002908D020252E1B0D46F540A14000D08B
:100DA00001212943084301061B1B000ADB1D02D554
:100DB000002070BC7047DB05181880180029F8DA8D
:100DC000401C4900F5D170BC40084000704710B588
:100DD000002B08DA0024401C614192185B411A4341
:100DE00001D14008400010BDF0B51FB482B00546E7
:100DF0000C0003D0084610F0ADFB02E010F0AAFB97
:100E000020300246009021462846FFF7A1FE049BB1
:100E1000059A04460F4618431143084314D0184658
:100E200010431BD0009840210A1A18460599FFF775
:100E30009FFE05460E46009A05990498FFF788FE26
:100E4000084305D0012004E02046394607B0F0BD34
:100E50000020C11705430E432C43374300990E98D9
:100E60006305401A7905E40A00220C43FD0A0A30A2
:100E700002D500200146E9E70105101969410C9CE3
:100E80000D9D00196941FFF7A2FFDFE74A00090342
:100E90000123090B1B0519430A4B10B5520D9A4249
:100EA00002DA0020014610BD064B34339A4203DCBF
:100EB0009A1AFFF75DFE10BD034BD218FFF748FEEC
:100EC00010BD0000FF030000CDFBFFFF10B500299F
:100ED00004DB0124E40740428C412146002B04DB63
:100EE0001C460123DB075242A341994200D19042A4
:100EF00010BD0000064C0125064E05E0E36807CC56
:100F00002B430C3C98471034B442F7D3FFF7DCF87E
:100F1000FC4801001C49010000487047201F0100E7
:100F200010B50446FFF7F8FF0068005DC007C00F6A
:100F300010BD0000F3B58DB000200A9001200B9089
:100F4000002608460C300C46099062690121099878
:100F50009047051E2ED0252D2DD0216A88470028C8
:100F600018D06269012109989047216A88470028B2
:100F7000F7D1411E62690998904700E0761CA1698B
:100F80000D988847216A88470028F7D1E1690D98B4
:100F90008847DAE7A1690D9888470746A84201D13A
:100FA000761CD2E7E1690D9888477F1C02D10A9828
:100FB000002877D049E1002762693D463946099803
:100FC00090472A280CD16269012109989047012590
:100FD00006E00A214F433F18303FEBD41020054371
:100FE0006269012109989047014630390A2903D2E4
:100FF0009B498F42DEDCECE7E90600D4994F6C2870
:101000000AD04C2810D0682824D06A282ED0742802
:101010000CD07A280AD00DE0626901210998904726
:101020006C2823D004211CE02020054362690121A3
:1010300009989047A760656065284FD026DC58283E
:1010400039D01ADC452849D012DC252834D0412873
:10105000B0D143E06269012109989047682802D025
:1010600008210D43E6E70120C002DEE70220DCE7AD
:10107000462833D047282CD130E05B2870D0612837
:101080002CD063286CD0642823D161E06F284FD026
:1010900009DC662822D0672820D0692826D06E284F
:1010A00017D12EE0CDE070284DD073286FD0752871
:1010B0004ED078280DD154E0A1690D988847054697
:1010C000252800D16CE7E1690D9888476D1C00D197
:1010D0006DE7BAE00A224CE00A2252E001202346E2
:1010E0006A46C0430D9900F050F9A3E0284640211C
:1010F00008436060A807234601D5002239E000229A
:101100003FE0E80700D020E72068011D216000686B
:10111000290501D5067018E7290701D5068014E7CF
:10112000A90703D5F117066041600EE706600CE7DA
:101130002846402108436060A807234601D50822BD
:1011400017E008221DE0484928460840606016E084
:101150002846402108436060A8072346BCD5B9E76C
:1011600015E02846402108436060A80707D52346BC
:1011700010220120C0430D99C046C0465AE02346C4
:1011800010220120C0430D99C046C04652E0002104
:101190000C910B460091632802D05B2807D043E0F6
:1011A000E80601D40120A060012000903CE06269C3
:1011B0000121099890475E2805D101200C90014635
:1011C0006269099890472169002906D10B4601AA56
:1011D0008F00491CD3510829FADB002835D021693A
:1011E00000290ED1C117C90E09184A11930001AA8E
:1011F0009A1849094901411A01201368884003439C
:10120000136062690121099890475D28E5D10C9827
:10121000002808D0002001AB81005A58401CD2435E
:101220005A500828F8DB01AB01202246C0430D9933
:10123000FFF710F800280ADA401C06D10B980028A6
:1012400003D00020C0430FB0F0BD0A98FBE7E907C8
:1012500002D10A99491C0A91361800200B9074E6B5
:10126000CCCCCC0CFFFFFF7FF1F7FFFFFFB5087878
:1012700089B01546FF2805D0491C2D2804D000222E
:10128000002407E000240BE00122F9E70A235C4375
:101290000419491C0878FF28F8D1002A00D06442BC
:1012A000002004902A7801462D2A01D02B2A0FD144
:1012B0006D1C2D2A02D00022049209E00122FBE7D6
:1012C00000260A2233466D1C00F0DDF93818714102
:1012D0002F78FF2FF4D10C9AA218069202460A43E7
:1012E00004D0FF23069A9133DA4205DA00210998E7
:1012F0000A4606C00DB0F0BD0024B74AB54D2646DB
:10130000079200F00DFA029006980391002801DA86
:10131000474200E0074639050020AF4A001C514112
:101320000191009012E0F80707D022462B46304684
:101330000799FFF797F90646079122462B46104674
:101340001946FFF78FF904460D467F10002FEAD1AA
:101350000698019B0028009A0399029806DAFFF785
:10136000E9F93246079BFFF7E5F905E0FFF77AF95F
:101370003246079BFFF776F9049A002A02D0012231
:10138000D2075140099A03C2B4E7FFB591B00020DB
:1013900009900025ED432E209E685C681F46019051
:1013A000B9696D1C129888470090396A88470028EF
:1013B000F6D10098401C0AD00D20C0018443002EB5
:1013C00012DD00982B2809D02D280DD103E0002034
:1013D000C04315B0F0BD012080020443B9696D1C03
:1013E00012988847761E009003A9600501D52D202C
:1013F00000E02B206A461073491C0CA80F91029044
:101400000AE0B9696D1C12988847009001204002DB
:1014100004431398761E0560002E02DD00983028E4
:10142000EFD001990098884245D18020044308E01C
:101430000998401E09900120400204431399681C3A
:101440000860B9696D1C761E129888470090302894
:10145000EED030E00199884205D1200603D48020E7
:101460000443761E1DE0009810F05AF9002825D09C
:10147000012149020C43009807AA0F990332303822
:10148000761E914208D208700F98401C0F902006DB
:1014900007D50998401E03E0200602D40998401C95
:1014A0000990A00502D51399681C0860B9696D1CE4
:1014B000129888470090002ECCDC59E0002E57DDB2
:1014C0000098652801D0452852D1A00550D50320A9
:1014D00000028443B9696D1C761E129888470090FB
:1014E000002E0CDD2B2804D02D2808D1FF20013040
:1014F0000443B9696D1C12988847761E0090E00578
:1015000001D52D2100E02B21029801700298401C8A
:101510000290019025E00120400204430EA90298A8
:101520000131761E88420ED20098029930380006AA
:10153000000E087003D10299019881420AD90298DD
:10154000401C029006E0E00501D5244801E0234854
:1015500040420990B9696D1C129888470090139811
:101560000560002E04DD009810F0DAF80028D2D1D2
:10157000F969129888470F99FF200870029903AA09
:10158000087000200A900B900CA90AA8099BFFF78D
:101590006DFEA00502D40120C0431AE724200442B6
:1015A00009D0E00713D138680B9A0A99031D3B60F4
:1015B000006806C00BE00B990A98FFF77DFA014618
:1015C000E00704D13868021D3A60006801602846CF
:1015D000FFE60000000014400000F03FF1D8FFFFDC
:1015E000F7B582B0029C00272078641C154601974D
:1015F000302802D0002D15D015E020780127641C7A
:10160000782804D0582802D0002D09D00BE0002DF6
:1016100001D0102D07D1002710252078641C02E08E
:10162000082500E00A250026009610E00099012711
:1016300069430818020C294680B2714300908E1845
:101640003804864201D3012001902078641C294689
:1016500000F056F80028E9DA0398002805D0002F9A
:1016600001D0641E00E0029C04600198002806D0AE
:101670000FF088FF02210160C81E05B0F0BD00997F
:1016800030040843F9E7F0B51FB486B0002000909D
:10169000019002900698069980B204900798090C70
:1016A00002040014114307900027089D0998069131
:1016B0003E463C4603900398A9B20204000C0390F6
:1016C00004982D0C1543484300212246FFF740FAA9
:1016D000C719714110340E46402CECDB3846029A93
:1016E000FFF736FA009A019B801800905941029842
:1016F0000191103002904028CCDB00980BB0F0BD77
:101700003A2800D23038202302469A43412A01D396
:1017100010463738884201D30020C043704700008C
:101720000EB5054A02920022009213460192FFF77D
:101730005BFB03B000BD00003304000070B58C18E3
:101740000578401C6B075B0F01D10378401C2A1100
:1017500006D10278401C03E006780E70401C491C3C
:101760005B1EF9D12B0705D40023521E0DD40B703C
:10177000491CFAE70378401CCB1A921C03E01D7841
:101780000D70491C5B1C521EF9D5A142D8D3002014
:1017900070BD000010B52148016A8A0715D44A07B8
:1017A00015D4C90732D01E498A89002A15D0531E84
:1017B0008B8182688C6904C48C610A691B040DD01A
:1017C000002A22D10121016010BD022100E0042184
:1017D000C16113488021416110BD0A69012A09D104
:1017E000026801239A430260C361FF206830993088
:1017F0000C4A106001204861CA69002A05D0886936
:1018000009898B00C01A904710BD10BDFF226832B5
:10181000054806A109A30DF017FBC04608D00140FA
:10182000A095010280E200E0742E01004144435F74
:1018300049525148616E646C65720000556E65785E
:101840007065637465642041444320696E746572F9
:10185000727570740D0A000070B582B00023019398
:10186000444801688A6A4C6813252540132D02D12B
:10187000CB689B07DB0F4361930772D453070AD4ED
:10188000D30711D1130724D5048F838E1C1B102C72
:101890000EDD102310E0042088620220032142A202
:1018A0000EF02EFB02B070BD0120886202B070BD48
:1018B000048F1B1B1C0610D0DBB20024058FC66AE8
:1018C00075192D5D0D74641CA342F7D1048FE318C4
:1018D0000387D20607D400212FE04B6A0824A343D4
:1018E0004B62D206F7D5CB68C28E448F141B5B04C3
:1018F000DB0EA34201D3438FD31ADAB2002A16D0EB
:10190000097D438F046BE1540199012A10D0012312
:101910001C46890145582D7D41184E8F9B19096B36
:10192000CD54641CE3B201999A42F2D800E0002140
:101930008B01C3185C8FA2185A878A0181184B8FBC
:10194000CC8EA3420BD301230B618058002242624C
:10195000CA6B002A03D03A31098801A8904702B027
:1019600070BD02208862044804A1084A08A30DF053
:101970006BFAC046749001028D2E01004145535F01
:1019800049525148616E646C65720000CE020000DD
:1019900041455320696E707574206F766572666C70
:1019A0006F770D0A00000000414553206F75747079
:1019B000757420756E646572666C6F770D0A000031
:1019C000F0B581B001243F2900D993E00346806837
:1019D000456B2D688E0001A7BE59B7461B1B000042
:1019E000371B0000131B0000131B0000F51A00003A
:1019F000F51A0000F51A0000F51A0000F51A0000AB
:101A0000F51A0000F51A0000F51A0000F51A00009A
:101A1000F51A0000491B0000651B0000F51A0000C4
:101A2000F51A0000F51A0000F51A0000F51A00007A
:101A3000F51A0000F51A0000F51A0000F51A00006A
:101A4000F51A0000F51A0000F51A0000F51A00005A
:101A5000F51A0000F51A0000F51A0000F51A00004A
:101A6000F51A0000F51A0000F51A0000F51A00003A
:101A7000F51A0000F51A0000F51A0000F51A00002A
:101A8000F51A0000F51A0000F51A0000F51A00001A
:101A9000F51A0000F51A0000F51A0000F51A00000A
:101AA000F51A0000F51A0000F51A0000F51A0000FA
:101AB000F51A0000DD1A0000DD1A0000DD1A000032
:101AC000DD1A0000DD1A0000DD1A0000DD1A00003A
:101AD000DD1A0000DD1A0000DD1A0000434800692D
:101AE0000024022809D001280DD0002802D103CA01
:101AF00004F0B6FF204601B0F0BD03CA04F0A2FF17
:101B0000204601B0F0BD03CA04F0C0FF204601B07A
:101B1000F0BD022931D0022430E0344D00242C6184
:101B20006C619849354A01F06FFE6869401C686134
:101B3000204601B0F0BD01F0A1FE284602F00EF9EA
:101B40000024204601B0F0BD284909690C234B430D
:101B50002749CA58C918496801F056FE0024204692
:101B600001B0F0BD0024204604F048FF0128C1D197
:101B70001E483030204900241CE001241B490F6915
:101B80000C26314679431A4A51188968214208D0F7
:101B900000247D1C15490D614C61042D10D315499D
:101BA00006E012494869401C4861032812D32949BC
:101BB00000241846224602F081F8204601B0F0BD0C
:101BC0006E430B498A598919496801F01DFE204668
:101BD00001B0F0BD0E20009000240A2228462146C4
:101BE00002F05CF8204601B0F0BDC046E499010265
:101BF000241F01002426010004260100F2390100FF
:101C0000B0B504290FD804468068C04679440979E4
:101C100049008F44020A0E1C1700104910A201F05F
:101C2000F3FD0020B0BD0120B0BD01F027FE002073
:101C3000B0BD00250321284604F0F0FE06492046E9
:101C40002A4602E003490022204602F037F800202D
:101C5000B0BDC04614260100942601008813000080
:101C6000415445300D0A0000B0B582B001240A2964
:101C700010D883687944097949008F440E290505F5
:101C80000B0B0B0B0B0B1A00194909680024224699
:101C900002F014F8204602B0B0BD50681449086044
:101CA000144915A2184601F0AFFD0024204602B0E9
:101CB000B0BD0024019403CA09A201AB02F01CF9D3
:101CC0000228E7D1019804F0FDFE204602B0B0BD25
:101CD000184601F0D3FD0024204602B0B0BDC04636
:101CE0002B4353513A2025642C252A0D0A0000006D
:101CF000009B01028813000041542B4353510D0AED
:101D000000000000B0B582B00546002404F0D4FE07
:101D100001280DD108498C60E86B426853684B601C
:101D2000009401926A4601F0C9FF204602B0B0BD9E
:101D3000E443204602B0B0BDC8930102B0B50546E9
:101D4000881E02280AD3A868012913D0002915D1BA
:101D50000C490DA201F058FD0020B0BD0220014643
:101D600004F05CFE064900242846224601F0A6FF46
:101D70002046B0BD01F082FD0020B0BD0120B0BD05
:101D8000E42501008813000041542B4346554E3D85
:101D9000300D0A00B0B5E0B00324E1016D462846DD
:101DA0000FF0C0FB204621462A460EF0A9F800207D
:101DB00060B0B0BDF0B597B00820149064201390C7
:101DC0002548109002200E904B20C0011690234D04
:101DD00028461430129001270F97B8021190032063
:101DE0000EA906F059F90026F443002802D0204637
:101DF00017B0F0BD0C35284601F0BEFF0028F6D123
:101E000080200C9016490B910A90164809901648AC
:101E100008901648079016480690392005901548F6
:101E20000490154803900D95144D03A9284601F020
:101E300055FD0028DBD1009501970F4C104911A2E8
:101E4000124B204601F0EEFE1149204601F01EFF24
:101E50003446204617B0F0BD80C001025C970102F5
:101E600080C4010200C50102452F0000952F00002B
:101E7000152F0000A4270100149A010290C9010245
:101E8000842501004149523738304500A42601001D
:101E9000951D000010B50348002404700EF0BCFF2F
:101EA000204610BD189F010280B501F053F90020B3
:101EB00080BD0000F0B58DB00E4600270C970B9743
:101EC0000A970997089707970697059702908068E1
:101ED0000490406B0068019004F08AFD04465BA109
:101EE00005220392FEF788F95A4D00281ED05AA108
:101EF00005222046FEF780F9002817D058A10522B8
:101F00002046FEF779F900280FD059A10522204676
:101F1000FEF772F9002809D057A105222046FEF7E6
:101F20006BF9002807D156A500E04FA505A8202190
:101F30002A4602F0B3F801203F2E00D936E0C04611
:101F40007E4436797600B7443340474A57313131C1
:101F5000313131313131653031313131313131313E
:101F60003131313131313131313131313131313161
:101F700031313131313131313131313131311F1F75
:101F80001F1F1F1F1F1F1F1FBE48416A04290CD19E
:101F9000039A426287620C2050433D490A58081850
:101FA000416805AB049801F02FFC38460DB0F0BD38
:101FB000B44C00206062A062CD49364A049801F01A
:101FC00023FCA06A401CA062EFE7049801F056FCD5
:101FD000019801F0C3FEE8E7AA48406A05E0A94974
:101FE000486A01220243032A1CD1A649421C4A62C4
:101FF0008F62062ACFD30BE0A2494A6A012013461A
:102000000343052BD2D1501C48628F62062803D3AC
:102010001E490DE09B48406A0C2141431C48425830
:102020004018BDE7886A401C8862032805D316491A
:102030000022029801F042FEB7E70E200090002136
:102040000A220198029B01F029FEAEE734363030B7
:10205000300000001A3A01003436303032000000FF
:102060003436303031000000554E494E45540000A2
:102070003436303036000000343630303300000063
:1020800043544E455400000084250100D42501002E
:10209000541F01009A39010070B5022956D30F2947
:1020A00007D1784C217A012905D1002222728F496B
:1020B0004AE0012070BD866801F084FE002004F033
:1020C000A5FC012803D10020032104F0A7FC002572
:1020D000284604F093FC012804D130346A490022D8
:1020E000204631E0304600F0EBFD00282ED030468F
:1020F000FFF708FE002829D004F09AFC012807D138
:102100005F498D60F06B4268E26252684A601AE093
:10211000022004F073FC012808D159498D61F06B4D
:102120004268E26252684A6110310CE0022004F019
:102130006DFC01280AD152498D62F06B4268E2625F
:1021400052684A6220312A4601F0B8FD002070BD75
:1021500010B582B003460120272931D87944097986
:1021600049008F442C132D2D162D2D2D2D2D2D2D69
:102170002D2D2D2C2D2D2D2D2D2D2D2D2D2D1C2DA1
:102180002D2D2D2D2D2D2D2D2D2D2D2904F0DCFF68
:1021900015E0DF490022184601F090FD0FE0002015
:1021A000019003CA08A201AB01F0A6FE012806D1E6
:1021B000019805F0E5F802E00248012101720020D3
:1021C00002B010BDE49901022B51495552433A2007
:1021D00022636C6F736564222C25640D0A00000075
:1021E000B0B502294AD30F2914D18568002004F024
:1021F0000DFC012803D10020032104F00FFC002472
:10220000204604F0FBFB012806D1D94830301E4996
:10221000002231E00120B0BD2846FFF773FD002801
:102220002CD004F005FC012808D115498C60E86B1E
:102230004268CF4BDA6252684A601CE0022004F028
:10224000DDFB012809D10E498C61E86B4268C84B5F
:10225000DA6252684A6110310DE0022004F0D6FBC8
:1022600001280BD106498C62E86B4268C04BDA62E8
:1022700052684A622031224601F020FD0020B0BDA4
:1022800040900102E49901020426010080B5022970
:1022900005D3042905D19E49002201F00FFD00203D
:1022A00080BD012080BDC046B0B50546881E02280D
:1022B0000AD3A868012913D0002915D10C490DA211
:1022C00001F0A2FA0020B0BD0220032104F0A6FB19
:1022D000064900242846224601F0F0FC2046B0BD05
:1022E00001F0CCFA0020B0BD0120B0BD24260100D1
:1022F0008813000041542B4346554E3D310D0A00D2
:1023000010B50F290BD001291DD000291DD1FFF7D1
:10231000C1FD0020022104F081FB002010BD044615
:10232000002004F06BFB012803D10020022104F0FF
:1023300075FB002004F06AFB012804D10449002247
:10234000204601F0BBFC002010BD012010BDC0469E
:1023500014260100F0B581B00124322928D80546A1
:102360008768786B0668C0467944097949008F44CC
:102370002F3F1919191F1F1F1F1F1F1F1F1F221F4C
:102380001F1F1F1F1F1F1F1F1F1F1F1F1F1F1F1F5D
:102390001F1F1F1F1F1F1F1F1F1F1F1F1F1F1F1F4D
:1023A0001F1F26001E4900242846224601F086FCF5
:1023B000204601B0F0BD1B48017800291FD0184904
:1023C00000242846224601F079FC204601B0F0BDE9
:1023D0000024FC623969384688470028FAD0114841
:1023E0000470FC62FFF756FD0E20009001220EE003
:1023F000304601F0B3FC0024204601B0F0BD0121BD
:102400000170FFF751FD0E20009000240522304698
:1024100021462B4601F042FC204601B0F0BDC046EB
:10242000A4250100049B010210B586B003460120DB
:102430003B2900D956E0C0467944097949008F44C8
:10244000505051513351515151515151515151519C
:10245000515151515151515151515151515151516C
:10246000515151515151515151515151515151515C
:102470005151515151391D1D1D1D1D1D002005902B
:1024800003CA02AA009218A205AB01F035FD02288A
:1024900027D1039A029817A1FDF7AEFE002820D19C
:1024A000059804F06DFF1CE0B5490022184601F0C4
:1024B00005FC16E0002002900590049003CA05AACE
:1024C000019204AA00920DA202AB01F015FD0328AF
:1024D00007D1049A0599029805F01EF8029804F0B5
:1024E000BDFF002006B010BD25642C2025700D0A0C
:1024F00000000000434C4F53454400002B5245431D
:10250000454956452C25642C25643A0D0A2565005D
:10251000F4250100012901D80020704701207047EF
:10252000B0B50546881E03280BD2104604F088FA81
:102530000F48C16A00242846224601F0BFFB20460E
:10254000B0BDAC6801290BD000290ED104F052FABD
:102550000346084908A2204601F056F90020B0BD04
:10256000204601F08BF90020B0BD0120B0BDC0466F
:10257000E49901028813000025730D0A0000000091
:1025800070B582B001240F293DD803468568686B79
:102590000668C0467944097949008F4407141E34FF
:1025A0003434342F373434343434434E66480024C2
:1025B00004708461C461012101716649664A28463C
:1025C00001F022F91FE0284601F058F9304601F0E9
:1025D000C5FB0024204602B070BD5B480024047196
:1025E0008269042111430278002A2ED0052958D18E
:1025F000016A491C016259D2624961E0524B187864
:102600000024002831D0204602B070BD4E4B18780F
:10261000012816D103CA183351A201F06DFC002025
:1026200002B070BD48480024846101210171007826
:102630004849002812D1484A11E0434E3079002819
:102640001BD00024204602B070BD052932D10024E1
:10265000012101708461C46101713E493F4A2846ED
:1026600001F0D2F8204602B070BD03CA183340A270
:1026700001F042FC204602B070BD002004F0C6F913
:10268000012803D10020032104F0C8F900242046CA
:1026900004F0B4F9012816D130362D490024304613
:1026A0004BE000210162C169491CC1610E2000900C
:1026B00000241CE0C169491CC161652915D330495A
:1026C0000024184639E02846FFF71CFB00289AD062
:1026D00004F0AEF9012812D11C4900248C60E86B8B
:1026E0004268F26252684A6027E00E20009002229F
:1026F0003046214601F0D2FA204602B070BD0220D9
:1027000004F07CF9012809D1104900248C61E86BA0
:102710004268F26252684A6110310EE0022004F011
:1027200075F9012800D06EE7084900248C62E86B37
:102730004268F26252684A622031224601F0BEFAD3
:10274000204602B070BDC046E499010240900102EB
:102750000426010088130000B6390100C1390100C8
:102760002B43475245473A20252A2C256400000078
:102770002B435245473A20252A2C256400000000AF
:10278000F4250100B4250100B0B584B001243B2933
:1027900000D937E0134605468068C0467944097978
:1027A00049008F444B5532322F2F2F2F2F2F2F2F91
:1027B0002F2F2F2F2F2F2F2F2F2F2F2F2F2F2F2F29
:1027C0002F2F2F2F2F2F2F2F2F2F2F2F2F2F2F2F19
:1027D0002F2F2F2F2F2F2F2F2F2F1D1D1D1D1D1D75
:1027E0000024039403CB01AA00921C4A03AB01F01E
:1027F00083FB022806D1029A019819A1FDF7FCFC7F
:1028000000280FD0204604B0B0BD1848006804F07E
:10281000B7FD174900242846224601F04FFA20460A
:1028200004B0B0BD1148006804F0AAFD10490022B0
:10283000284601F043FA204604B0B0BD0B490B60B6
:102840001E210CA200F0E0FF0024204604B0B0BD21
:1028500001F014F80024204604B0B0BD1A3B01007A
:10286000434C4F5345204F4B00000000089B010292
:10287000C425010041542B434950434C4F53453D1F
:1028800025640D0A00000000F0B589B0044601205F
:102890003B2900D9AAE01646A7687A6B1568C0469E
:1028A0007944097949008F44536AA071A1A1A1A17B
:1028B000A1A1A1A1A1A18AA1A1A1A1A1A1A1A1A11F
:1028C000A1A1A1A1A1A1A1A1A1A1A1A1A1A1A1A1F8
:1028D000A1A1A1A1A1A1A1A1A1A1A1A1A1A11D1DF0
:1028E0001D1D1D1D0027089703CE06AA0092414A10
:1028F00008AB01F001FB022877D13F480568089832
:10290000854272D1079A069E3CA130460592FDF79A
:1029100073FC002847D03DA13046059AFDF76CFCBA
:10292000002840D03CA13046059AFDF765FC002800
:10293000314E5AD1284604F03DFD7068401C70604D
:1029400003283CD303207060306804F0BBFC36E001
:1029500029480660304604F009FD059026480068C5
:1029600004F0D8FC04902448006804F0DFFC0499CB
:10297000019102900598012827D02EA026E0384624
:1029800000F07CFF284601F0E9F92EE01A4D286896
:1029900004F010FD6868401C686003280FD3002213
:1029A0006A6022490DE0144E7760284604F018FD55
:1029B000306804F057FE002801D01B4900E00C49A4
:1029C0000022204601F07AF90FE019A000901A4980
:1029D0001AA23846334600F017FF0E20009000215F
:1029E000B4222846234601F059F9002009B0F0BD71
:1029F000C42501001A3B0100D4970102414C524505
:102A000041445920434F4E4E45435400434F4E4E90
:102A1000454354204F4B0000434F4E4E45435420F6
:102A20004641494C00000000642601008425010055
:102A300054435000554450008813000041542B4328
:102A4000495053544152543D25642C222573222C65
:102A5000222573222C25750D0A000000B0B582B026
:102A600014468A1E022A12D38568012917D000292C
:102A70001CD1204604F040FC00901E210EA22846E6
:102A8000234600F0C1FE0024204602B0B0BD094933
:102A90000024224601F012F9204602B0B0BD2846BB
:102AA00000F0ECFE0024204602B0B0BD0124204618
:102AB00002B0B0BD7426010041545E4845415254F5
:102AC000434F4E4649473D312C25642C25750D0A50
:102AD00000000000F0B583B014468A1E022A1CD301
:102AE0008568012921D0002926D1164F3C60204657
:102AF00004F0F4FBFDF76CFB0646386804F0EEFBCF
:102B00007108009101901E210FA22846234600F073
:102B10007BFE0024204603B0F0BD09490024224674
:102B200001F0CCF8204603B0F0BD284600F0A6FE28
:102B30000024204603B0F0BD0124204603B0F0BDC0
:102B4000C42501000C9B010241545E48454152548A
:102B5000424541544845583D25642C25752C257324
:102B60000D0A0000F0B585B0044601203B2900D9CC
:102B700085E0A5687944097949008F443F547F5B1B
:102B80008080808080808080808080806080808065
:102B90008080808080808080808080808080808035
:102BA0008080808080808080808080808080808025
:102BB00080801D1D1D1D1D1D0020049003CA02AA3A
:102BC0000092304A04AB01F097F9022856D12E4802
:102BD00085680498854251D1039E029F2BA13846F7
:102BE0003246FDF709FB00283AD02AA13846324682
:102BF000FDF702FB002841D128461DE0224CA260CF
:102C0000104604F09FFB002838D001F0DEFAE060A7
:102C1000002833D0A36840680090234923A22846A7
:102C200000F0F2FD2AE018480021C160284600F0BB
:102C300025FE23E01448806804F0A2FB19E000F0B0
:102C40008DFE012804D11048C16803C900F08EFF31
:102C50000D48C0680CC81349284600F015FE0DE069
:102C6000284604F06FFB0028074907D0C96801F027
:102C700082FA0B490022204601F020F8002005B01E
:102C8000F0BDC0461A3B0100D497010253454E44A3
:102C9000204F4B0053454E44204641494C00000014
:102CA000C4250100204E00008813000041542B432E
:102CB000495053454E443D25642C25750D0A0000AE
:102CC000F0B583B0074601F07DF80026304604F0E9
:102CD00043FB032835460BD10421284604F0B2FCFF
:102CE000F86B51492A4600F0E9FF304603B0F0BDC9
:102CF00002970024204604F02FFB0428254609D122
:102D00000298C06B49492A4600F0D8FF2646304653
:102D100003B0F0BD0027384604F01EFB05283D46F1
:102D200009D10298C06B40492A4600F0C7FF3E46D1
:102D3000304603B0F0BD01970125284604F00CFB96
:102D40000328029FC8D00125284604F005FB04286B
:102D5000D6D00125284604F0FFFA0528019FE0D0CF
:102D60000225284604F0F8FA0328029FB4D0022571
:102D7000284604F0F1FA0428C2D00225284604F0BF
:102D8000EBFA0528019FCCD0254C2068401C03217C
:102D9000FDF7B6F90D46084604F0DEFA0628029F54
:102DA00008D1284604F0CEFA002803D001F00DFA2D
:102DB00000282AD1681C0321FDF7A2F90D46084618
:102DC00004F0CAFA062808D1284604F0BBFA002805
:102DD00003D001F0FAF9002817D1681C0321FDF790
:102DE0008FF90D46084604F0B7FA0021CE430628B5
:102DF00000D07AE7284604F0A5FA002800D174E74D
:102E000001F0E3F9002800D16FE72560F86B054970
:102E10002A4600F053FF0026304603B0F0BDC046FE
:102E2000109B010284260100442601005426010063
:102E300080B58AB00620042108F078FE4B20C0013E
:102E400009900820079064200690B448143005903B
:102E50000648039002200190012002908002049015
:102E6000032001A905F018F90AB080BD80C0010255
:102E7000B0B582B001220F293ED803468068446B6A
:102E80002468C0467944097949008F44071F2527E3
:102E9000343535353535353535350A152749002270
:102EA00004E02649CA68092A20D8521CCA6016497B
:102EB000164A00F0A9FC1EE0002003F09FFD012847
:102EC00019D11E4830300E49002212E000F0D6FC25
:102ED000204600F043FF0EE00D4908E00E20009070
:102EE00000210122204600F0D9FE04E0054900221D
:102EF000184600F0E3FE0022104602B0B0BDC04606
:102F000004260100E425010088130000CD390100EA
:102F10009425010080B5032005F0A6F880BD0000CF
:102F20000648416B0020002905D0054A914203D094
:102F300049680029FAD1704701207047E4990102DD
:102F4000D4250100B0B514460D460846114600F0E0
:102F5000BAFF012816D1285D002813D1002C0BD010
:102F60006019401E00780A2806D10320084A01464D
:102F70002B460CF0C5FF05E00320054A01462B4611
:102F80000CF0BEFF03202946224605F059F9B0BDDA
:102F900063390100F0B585B0054604A8002404702B
:102FA000E743002D12D0EA68002A0FD0686A002893
:102FB0000CD0A86A002809D0401EE96A814200D3DB
:102FC0008EE004A928469047002803D03C462046BE
:102FD00005B0F0BD514EE86A411CE962696A049A85
:102FE0000A54E86A696A002202920A54E86A0928C7
:102FF00006D1696A09224848FDF7F1F800283ED059
:103000003078411E022908D800F0DCFEB168401A71
:103010004349884264D8414E30780A2820D001289C
:1030200023D16E6A3A213046FDF7C8F8002847D010
:10303000019002980390E96A03AB304639A200F090
:103040005BFF02284CD10398002849D00A21334A5B
:10305000117001990818696A401AC01C50602FE06D
:103060007068E96A81422BD13AE004A800780A2806
:103070000FD00D2814D101202863E86A1AE001203E
:10308000307000F09FFEB0603078411E0229BBD93D
:10309000C3E7296B012904D102202863E86A03E011
:1030A000296BE86A022905D1022817D10298E86243
:1030B000286305E0012803D1686A00783E280FD014
:1030C000A86AE96A401E81420AD2EA6804A9284631
:1030D00090470028114E00D17DE777E702982863DA
:1030E000E96A686A00F0EFFE01280FD16B6AE86AAE
:1030F000002806D0C018401E00780A2801D10DA271
:1031000000E010A2032001460CF0FAFE0348047010
:10311000204605B0F0BDC046A63201005C97010212
:10312000DC0500002B524543454956452C252A2CE9
:1031300025643A005B415420526563765D20257317
:10314000000000005B415420526563765D202573CA
:103150000D0A000010B5064C2078002108F0A2FCF2
:10316000044806F047FD2078012108F09BFC10BDC3
:10317000E696010260E31600B0B50F2001F0ECFB0B
:10318000194D6870287033282AD120243721204611
:1031900001F02EFC2120032101F02AFC22204021F5
:1031A00001F026FC2320082101F022FC3020AA2176
:1031B00001F01EFCA94802210187322001F018FC11
:1031C0003320012101F014FC5F21204601F010FCA6
:1031D0000F2001F0C1FB28700A2006F00BFDB0BDE6
:1031E0009E480021C187B0BD04960102F0B581B0B0
:1031F000364C212100916172354909886170354F43
:10320000FA886271BD6ABD61334B1B782370090A6D
:10321000A170110AA171B978814207D10AF06CFE40
:103220006421FCF757FF3981B978BD6A2B484843C0
:103230002B4940180A21FCF74DFF4519FD620AF0A1
:10324000F1FD40190BF04AFA06460D462548007B71
:103250000BF0D0F8244909882222A15482B2D20B63
:10326000801802B2D0175210B2186841130E009D98
:103270006355130C202563553B6DA3761D0AE57637
:103280001D0C25771B0E637723462233090A5970DC
:10329000A277BA64F864BA65F865100AE0770AF0B4
:1032A0002BFEF861FB6A2821012220460EF0C0F8AF
:1032B0000AF022FE786108F0FDFF0028FBD104200F
:1032C00008F0B0FB002001B0F0BDC0463ED40102C2
:1032D000E098010268990102BC980102800A1B0073
:1032E00040C20C00B6900102C698010270477047B8
:1032F000F0B589B056480068FDF718FB04460D4646
:103300005448406AFDF7C4FB02460B462046294656
:10331000FDF710FA02460B4600244F492046FDF700
:1033200093F90590049106204C49085EFDF7FEFADA
:1033300002900191012007904002039048494831D2
:10334000484F06E0554A10517F1C891C241D642CEF
:103350007CD0387805284448F4D106970891434832
:1033600001593F4E316142480359B3604148005909
:10337000B061414A1259326200275D1A35637369A0
:10338000F1689941079B00DB3B46002B01D0039B72
:10339000C918334E7163F369716A101A9941079A1B
:1033A00000DB3A46002A01D0039A8918FDF7E0FABB
:1033B00002460B4605980499FDF754F9FDF740FBCA
:1033C000274A9062D162401BC10F40184010106024
:1033D0001546FDF7ABFA294A294BFDF743F9A863D7
:1033E000E963284A284BFDF73DF93A46274BFDF79C
:1033F00039F93A46264BFDF783F805460E4618483C
:103400000564416428463A46224BFDF751FA0028EC
:103410000899069F98D10022284631461E4BFDF799
:103420005DFA089900288FD1088800B2FDF77EFA6E
:1034300002460B4628463146FDF762F8029A019B88
:10344000FDF75EF8FDF7D8FA08997BE709B0F0BD03
:1034500028970102802001000000F03F6AA90102C4
:103460001896010238980102FFFF0100CC9F01026B
:1034700030A001022CE0010290E00102699006698F
:103480009006903F52257997532ED33F0000594024
:1034900000003E4000408FC0006AF84058D2010250
:1034A000B0B582B0194C2068056801A900200870E9
:1034B00007E090470198401C01A90870C0B2082895
:1034C00022D2012211048140294209D02268516090
:1034D00080002018826A002AECD001A80121E8E7C8
:1034E000130283402B4201D0022104E082402A4291
:1034F000E0D00321134622685360800020188268C0
:10350000002AD7D001A8D4E702B0B0BDD4920102FE
:10351000FEE7000010B509480168CA69202313437B
:10352000CB610269032A08D1012293050C689C43F0
:103530000C605102C26E0A43C26610BD489301027C
:1035400081B010B581B00393002807D0C16A00296B
:1035500004D003AB0093C46A0021A04701B010BCA3
:1035600001BC01B00047000080B502460848006871
:10357000002807D091B2120C03889A4203D0406908
:103580000028F9D180BD002200F0F4FA80BDC046C9
:103590008CC90102F0B581B05C4C2068856BE807EE
:1035A00007D0E168002904D0002088472068012165
:1035B0008163A80707D52169002904D00120884725
:1035C000206802218163680707D56169002904D05A
:1035D00002208847206804218163280707D5A16954
:1035E000002904D003208847206808218163E80669
:1035F00007D5E169002904D00420884720681021FC
:103600008163A80607D5216A002904D005208847D0
:10361000206820218163680607D5616A002904D0EB
:1036200006208847206840218163280607D5A16AC3
:10363000002904D007208847206880218163012663
:10364000E80507D5E16A002904D037020820884739
:1036500020688763A80507D5216B002904D077026D
:103660000920884720688763680507D5616B0029B2
:1036700004D0B7020A20884720688763280507D549
:10368000A16B002904D0F7020B20884720688763CC
:10369000E80407D5E16B002904D037030C208847E4
:1036A00020688763A80407D5216C002904D077031C
:1036B0000D20884720688763680407D5616C00295E
:1036C00004D0B7030E20884720688763280407D5F5
:1036D000A16C002904D0F7030F2088472068876376
:1036E000E80307D5E16C002904D03704102088478F
:1036F00020688763A80307D5216D002904D07504CD
:10370000112088472068856301B0F0BDD89301027D
:1037100002480068411E88417047C046D4980102A3
:10372000F0B58DB0002862D00446406800285ED015
:10373000A06840285BD8E56A002D58D0074620468F
:1037400040300026039003E0019E4AE0039848E0E1
:10375000402101220691FCF71FFDAE4202963ED2A7
:1037600000203146019009900398069B3E46002EAA
:10377000EAD0606A0491405C07900998401C05906B
:103780000021042708916518EA5C012A17D10A96DE
:103790006268D3191B1F1B68099E9E5D07988642AD
:1037A00008D1059D5B5D002B0A9E22D00898401C25
:1037B000089003E0403500222A70A668069B08376F
:1037C000491CB142DFD308980028BFD00499491C96
:1037D000E06A8142059809900398C8D301E00398F4
:1037E0003E463746E56A029E761CAE42B0D30DB027
:1037F000F0BD616A0B91E16A0C91D1590BAA204688
:1038000000F09CF80DB0F0BD81B0B0B583B00D46AE
:103810000446079307AB02938069E1690DF082FECD
:10382000206265480078002803D1216AA06900F071
:103830009FF96369A169226A204698470146A06BF7
:10384000002905D069460C600021224B0A460CE095
:1038500000F084FA7D2081002846FCF73BFC0246FC
:10386000A06B69460C6000211B4B00F0D3FA0020CE
:1038700003B0B0BC02BC01B00847C04680B5806B45
:1038800000F06CFA002080BD70B582B00D46044691
:10389000466911461A46B0470146A06B002907D079
:1038A00069460C6000210B4B0A4600F0B3FA0EE0AB
:1038B00000F054FA7D2081002846FCF70BFC0246FC
:1038C000A06B69460C600021034B00F0A3FA0020B6
:1038D00002B070BDC1390000D739000070B50D4687
:1038E0000446802100F0C0FA2868E06368686060E0
:1038F000A868A060E868E060286920616869606184
:10390000A869A061E86900262662E061286A606211
:10391000686A2663E662A062A86A6063204638305F
:1039200000F02AFA002802D0F643304670BD214844
:10393000016821600460304670BDC04670B5144611
:103940000D460646881E032802D8B06B00F006FA22
:10395000F06B2946224600F00DF970BD164801783B
:10396000012048407047C04670B512480468002CDA
:103970001FD0114E11A5216920468847002815D176
:10398000307800280DD1E16A606A00F09CFA0146A7
:10399000606A012903D0E16A00F0E8F8284600F0E7
:1039A000E3F82046FFF7BCFE0020E0622468002C0C
:1039B000E1D170BD88C9010280C901020D0A000071
:1039C00010B50446806B00F0C9F9E06B05210022B8
:1039D00000F0D0F810BD10B50446806B00F0BEF9C1
:1039E000E06B0421002200F0C5F810BDF0B581B0F5
:1039F00000910646C7680468A01C3946FCF76AFBBC
:103A000000257068814201D1ED430BE0601C39460E
:103A1000FCF760FB316032695143B06808180099C7
:103A2000FCF7A8FB284601B0F0BDB0B50124002585
:103A30000560446008300EC0B0BD70B50E46044647
:103A4000C1680068401CFCF745FB002560688142A6
:103A500002D1ED43284670BD22695043A168411848
:103A60003046FCF787FBE1686068401CFCF732FBDE
:103A70006160284670BDB0B5002400280DD0054611
:103A800000688842FDD3401A286068684018E968D9
:103A9000FCF720FB69602046B0BDE4432046B0BD82
:103AA000B0B5002400280ED00546006840182860F4
:103AB000EA689042FDD8A86840181146FCF70AFB56
:103AC000A9602046B0BDE4432046B0BDF0B583B048
:103AD000164602460027F843002E22D01C46002B33
:103AE0001FD00D46D168136899421AD9CB1AAB4240
:103AF00017D39268019252198A423A4607D9019A1D
:103B00008A1A0292029A52199342029A09D3029295
:103B100001981018FCF7DEFA316002984019206015
:103B2000384603B0F0BD4068704780687047024671
:103B30000020002A04D0106050609060D16070476F
:103B4000C0437047002803D001684842484170478D
:103B500001207047002805D00168C068411A48421A
:103B6000484170470120704700207047002070478F
:103B700000207047F0B583B014460D4606464088D5
:103B8000012818D1306900280CD0A90040580178CC
:103B90002D2910D0F368716809686A461160506079
:103BA00010A205E0F36870680068694621C115A29B
:103BB0003046FFF7C5FC7768FB6830462946224649
:103BC0009847012808D00AE0C368304629462246B3
:103BD00098477F68012802D178680028F4D103B0A3
:103BE000F0BDC04646534D3A252D387320535441FD
:103BF00054453A252D323873204556454E543A25C2
:103C0000730D0A0046534D3A252D38732053544105
:103C100054453A252D323873204556454E543A25A1
:103C2000750D0A00F0B581B0002828D01E460C465C
:103C30000546079B0698009000206862A862E8622B
:103C4000104909886B8029800F4B1F686C60009BAE
:103C5000AB602B460C33C4C3A861E8612862481CE2
:103C60000849088008480560002C08D06C600021D5
:103C700028460A46FFF77EFFA468002CF6D101B063
:103C8000F0BDC04610CD01028CC9010202460020E1
:103C9000002A01D0D1627047C043704710B582B08E
:103CA00004AC24881B881B041B196C462360024B40
:103CB00000F0B0F802B010BD69350000F0B597B063
:103CC0001646029105464268002A30D001966A6085
:103CD00001210024284616462246FFF74BFF3046B6
:103CE000029FBE4232D003A85021FCF75CFA324654
:103CF0007268002F0CD003AF029811C74068083FCC
:103D0000824209D0394608313C4600280F46F4D19A
:103D1000002A019EDBD10AE0019E3868686000211C
:103D200028463246FFF726FF7F68002FF5D102981C
:103D30008468002C08D06C60002128463246FFF7CA
:103D400019FFA468002CF6D117B0F0BD0021284659
:103D5000019E3246FFF70EFFE9E700000146002012
:103D60001F2901D9C043704718224A43344901230F
:103D70008B5089188860704710B50021CC4300280B
:103D80000BD00A4A1368002B09D01832491C20298D
:103D9000F8D306D106A0FFF7E7FE204610BD0123A9
:103DA000136001600024204610BDC04610CA010205
:103DB00074696D65722049442069732066756C6C66
:103DC0000D0A0000264800687047C04670B52024E0
:103DD0001B4D234E2868022817D13068A968EA686D
:103DE000401A904211D96969002907D02879002822
:103DF00007D0022028603068A86004E00120286015
:103E000003E001202860286988471835641EE1D145
:103E100070BDC046F0B5044600201F2C01D9C04338
:103E2000F0BD059D18266643054C0227A751A4192D
:103E300021710B4909682646083626C66361F0BD24
:103E400010CA010206480168491C01600548416822
:103E500002680023521C02604B4143607047C04619
:103E6000C4AD0102C8AD010280B5FCF79CF980BD6C
:103E7000B0B50278002A24D0441C0021084601E095
:103E8000573A08E023460001D5B2302D0C4611D335
:103E9000392D02D8303A14460CE0412D0C4609D396
:103EA000462D01D8373AF6E71446613CE4B2062CB9
:103EB000E6D30024E2B280185C1C1A78002AE1D113
:103EC000B0BD0020B0BD10B50246012000290DD0C4
:103ED0000023D45C202C02D37F2C04D307E00D2CCC
:103EE00001D00A2C05D15B1C8B42F2D310BD0020FF
:103EF00010BD002010BD000081B0F0B584B0099362
:103F000000230393002800D1C2E0002A00D1BFE0C3
:103F100009AB03931678002E00D1A8E05623DB43AB
:103F2000009300231D46002900D1A2E0252E3FD199
:103F3000971C52781446643C0023142C43D8C04686
:103F40007C4424796400A7440A99A3A3A3A3A3A350
:103F5000A3A3A3A34CA3A3A3A3A3A3A35F0002971C
:103F6000039A131D0393126801920122002317463E
:103F70001E460478FF0703D02D2C01D1164607E01A
:103F80002746303F092F09D80A275F433B19303BAA
:103F9000491E401C00270029EBD13946029A019C9A
:103FA000002C03D0012E00D15B4223606B1C06E085
:103FB0000378B3425BD1491E521C401C2B46167835
:103FC000002EAFD164E02A2A62D13A780378934276
:103FD00004D0491E401C0029F8D100216B1C3A4630
:103FE000EDE7039A131D03933E7812680023C45C27
:103FF000B44233D0491E5B1C0029F8D13C46C71897
:104000000021002A2ED12EE00297039A131D03935C
:1040100012680023009E0778302F18D33A2F02D25F
:10402000344627340BE0612F03D3672F344606D381
:104030000DE03C46413C052C09D8344620341B0198
:104040001B19DB19491E401C0029E4D10021029CE8
:10405000002A00D013606B1C2246B0E73C46C7180C
:10406000002A00D009C26B1C22463846A7E700236D
:104070000EE0252E0BD15178652908D103990A1D30
:1040800003920968002900D008606B1C00E02B46F1
:10409000184604B0F0BC02BC01B0084781B010B5AE
:1040A00081B00C46039303AB00930DF03BFAA042A2
:1040B00000D3601E01B010BC02BC01B0084770B54F
:1040C00004460020002A1BD0002C19D0002B17D04A
:1040D00014600120022B13D32578002D10D0641C0E
:1040E00001208D4205D1651E00262E708500545199
:1040F000401C984204D2661C2578002D3446F0D12D
:1041000070BDB0B504467821FCF758F8002805D1F9
:1041100058212046FCF752F8002828D04278002A7F
:1041200023D0841C0021084623460001D5B2302D3F
:104130000C4613D3392D01D8303A0EE0412D0C46F0
:104140000CD3462D01D8373A07E01446613CE4B25F
:10415000062C01D3002401E0573A1446E2B280183D
:104160005C1C1A78002ADFD1B0BD0020B0BD20460B
:10417000FCF7E4F8B0BD70B504460026F043002C0F
:104180000DD00D4600290AD0204610300121FFF73E
:1041900072FCA96820342046FFF76DFC304670BDE4
:1041A00070B504460026F043002C0DD00D460029C2
:1041B0000AD0204610300121FFF772FCA968203494
:1041C0002046FFF76DFC304670BD70B50024002816
:1041D00014D00546064610363046FFF7B3FC0128DA
:1041E0000CD028462030FFF7ADFC012806D02C6803
:1041F0003046FFF798FC0C2141436418204670BDFF
:10420000F0B583B000250295019500281FD00C461B
:104210000646074610373846FFF79CFC002816D1A3
:104220003046203002AA01AB2146FFF74FFC0028A0
:104230000DD135683846FFF778FC0C214143B06852
:10424000029A101868506D186C600198A860284692
:1042500003B0F0BD70B505460C20584300249042D1
:1042600011D2121A461829606860AE60EA602846CA
:1042700010301946FFF75BFCE96820352846FFF748
:1042800056FC204670BDE443204670BD04217046B4
:10429000084204D0EFF30983EFF3088203E0EFF361
:1042A0000883EFF309829BB004A8F0C044464D4652
:1042B00056465F4608A8F0C01846F0C86846F0C0E9
:1042C00018690C90202018440D9058690E90986938
:1042D0000F90D8691090EFF310801190EFF31480D5
:1042E0001290094908681390084908681490084911
:1042F0000868159007490868169017931892704639
:10430000199068460AF0BAFF04ED00E00CED00E0F9
:1043100010ED00E014ED00E0F0B581B003260024BC
:104320003046214607F002FC04252846214607F0C6
:10433000FDFB0127304639463A4607F08BFB3046F5
:104340002146324607F01AFC284639463A4607F01D
:1043500081FB02212846224607F010FC01B0F0BD87
:10436000F0B589B008900425284607F05BFB0A27C2
:10437000384605F03FFC284607F064FB032420463E
:1043800007F058FB07900526304605F033FC284619
:1043900007F048FB384605F02DFC284607F052FB95
:1043A000204607F047FB0690304605F023FC2846E0
:1043B00007F038FB384605F01DFC284607F042FBA5
:1043C000204607F037FB0590304605F013FC2846E1
:1043D00007F028FB384605F00DFC284607F032FBB5
:1043E000204607F027FB0490304605F003FC2846E2
:1043F00007F018FB384605F0FDFB284607F022FBC6
:10440000204607F017FB0390304605F0F3FB2846E3
:1044100007F008FB3846019705F0ECFB284607F04B
:1044200011FB204607F006FB0290304605F0E2FB48
:10443000284607F0F7FA384605F0DCFB284607F077
:1044400001FB204607F0F6FA0746304605F0D2FB9E
:10445000284607F0E7FA019805F0CCFB284607F05C
:10446000F1FA204607F0E6FA0446304605F0C2FBB2
:10447000284607F0D7FA0699481E81410A4607994F
:10448000481E8141480080188000059A511E8A41CB
:1044900051004018049A511E8A4180188000039AE6
:1044A000511E8A4151004018029A511E8A418018BB
:1044B0008000791E8F4179004018611E8C410619D9
:1044C0000898002803D0032007F0ACFA02E003208C
:1044D00007F0B8FA0A24204605F08CFB042528468C
:1044E00007F0B0FA204605F085FB284607F09AFA57
:1044F000F0B209B0F0BD70B50446042007F092FA9E
:1045000060B2002803D4032007F08CFA02E00320F5
:1045100007F098FA0A25284605F06CFB0426304679
:1045200007F090FA284605F065FB304607F07AFA66
:10453000284605F05FFB600603D4032007F072FAFB
:1045400002E0032007F07EFA0A25284605F052FB18
:104550000426304607F076FA284605F04BFB304635
:1045600007F060FA284605F045FBA00603D40320B7
:1045700007F058FA02E0032007F064FA0A252846FB
:1045800005F038FB0426304607F05CFA284605F0B3
:1045900031FB304607F046FA284605F02BFBE006D3
:1045A00003D4032007F03EFA02E0032007F04AFAA2
:1045B0000A25284605F01EFB0426304607F042FA7D
:1045C000284605F017FB304607F02CFA284605F080
:1045D00011FB200703D4032007F024FA02E0032094
:1045E00007F030FA0A25284605F004FB0426304679
:1045F00007F028FA284605F0FDFA304607F012FACF
:10460000284605F0F7FA600703D4032007F00AFAFA
:1046100002E0032007F016FA0A25284605F0EAFA18
:104620000426304607F00EFA284605F0E3FA304635
:1046300007F0F8F9284605F0DDFAA00703D40320B7
:1046400007F0F0F902E0032007F0FCF90A252846FC
:1046500005F0D0FA0426304607F0F4F9284605F0B4
:10466000C9FA304607F0DEF9284605F0C3FAE0073C
:1046700003D1032007F0D6F902E0032007F0E2F9A6
:104680000A24204605F0B6FA0425284607F0DAF990
:10469000204605F0AFFA284607F0C4F9204605F099
:1046A000A9FA70BDF0B581B003260025012430467B
:1046B0002946224607F0CEF9304607F0C3F9062610
:1046C000304605F097FA042007F0BCF9304605F0B3
:1046D00091FA032007F0AEF900281BD0681CFA2DD0
:1046E0000546F6D30425284607F09CF903263046F4
:1046F00007F098F90A27384605F07CFA284607F0B3
:10470000A1F9304607F09EF9384605F073FA2046C5
:1047100001B0F0BD032001210A4607F09BF90420F7
:1047200007F080F90024204601B0F0BDB0B5044682
:10473000C00703D1032007F075F902E0032007F05A
:1047400081F90825284607F07DF9284607F06AF91F
:10475000A00703D4032007F065F902E0032007F067
:1047600071F90825284607F06DF9284607F05AF92F
:10477000600703D4032007F055F902E0032007F097
:1047800061F90825284607F05DF9284607F04AF93F
:10479000200703D4032007F045F902E0032007F0C7
:1047A00051F90825284607F04DF9284607F03AF94F
:1047B000E00603D4032007F035F902E0032007F0F8
:1047C00041F90825284607F03DF9284607F02AF95F
:1047D000A00603D4032007F025F902E0032007F028
:1047E00031F90825284607F02DF9284607F01AF96F
:1047F000600603D4032007F015F902E0032007F058
:1048000021F90825284607F01DF9284607F00AF97E
:1048100060B2002803D4032007F004F902E003206B
:1048200007F010F90824204607F00CF9204607F09D
:10483000F9F80724204607F005F9204607F0F2F8BA
:10484000B0BDF0B581B0032700243846214607F0FB
:104850005DF93846214607F069F9012538462946B1
:10486000224607F0F7F8052638462946324607F073
:1048700085F908273846214607F058F93846294671
:10488000224607F0E7F838462946324607F076F91F
:1048900007273846214607F049F938462946224677
:1048A00007F0D8F838462946324607F067F901B0D4
:1048B000F0BD000080B50B2007F0BCF812490A7863
:1048C000002804D0002A12D003F0F0FA80BD012A9B
:1048D000FAD1002008700F49C8830C4908700C48B1
:1048E000012101700BF048FC03F0E0FA80BD07489D
:1048F000012202700A700648002101700BF05CFC76
:1049000003F0D4FA80BDC0461C9001021890010249
:10491000199001026AA9010202484069811E4842B9
:1049200048417047A096010280B5FDF743FA002880
:1049300001D00020C04380BD80B5FEF7F1FA80BDF4
:1049400010B504480F2100242246FFF713F9204632
:1049500010BDC046149A0102F0B581B00746032489
:10496000204607F06FF80425284607F06BF820462C
:1049700007F058F80A26304605F03CF9284607F0BB
:1049800051F83220FFF7B7FDFFF78CFEF8B2FFF7C2
:10499000B2FDFFF787FE204607F054F8284607F0DF
:1049A00051F8204607F03EF8304605F023F9284636
:1049B00007F038F83320FFF79EFDFFF773FE002065
:1049C000FFF7CEFC0746284607F02CF8204607F0F4
:1049D00029F8304605F00EF9284607F033F820464E
:1049E00007F030F8304605F005F9384601B0F0BD63
:1049F000F0B581B0009107460324204607F022F865
:104A00000426304607F01EF8204607F00BF80A256A
:104A1000284605F0EFF8304607F004F83220FFF79B
:104A20006AFDFFF73FFEF8B2FFF765FDFFF73AFEBC
:104A30000098FFF760FDFFF735FE304606F0F2FF05
:104A4000204606F0EFFF284605F0D4F8304606F081
:104A5000F9FF204606F0F6FF284605F0CBF8284679
:104A600005F0C8F801B0F0BD80B50748012101701C
:104A7000064802680A43026005480268002A02D01C
:104A800000200146904780BD16CD01021C10005049
:104A900018CD0102F0B599B0F548017BC67A427B8A
:104AA0000E92F44C221F1368F34A12680692427861
:104AB0000C9202790592C76A04931F4001200F905F
:104AC0007A0200D5BCE03A0200D5BFE0FA0102D577
:104AD0000F9802062260502508968A191826BB01F5
:104AE00002D50F98430623604123079569430A9630
:104AF000354655431426FC0210D50F980405384658
:104B00003746DC4E3460DA4CA469B464D84CE469AE
:104B10007464DA4C241D34603E46074690000B90C6
:104B2000D8040D90681809900E9B73430F98820368
:104B3000B902D04D22D50F9841052960CC480E9678
:104B40001646024681692965C169696509990D980A
:104B500001430898000108180B994018C018C8496B
:104B6000098892794A4380180A301C4605F022FBD6
:104B7000234632460E9EC04988672A600F98C404B7
:104B8000380300D52C60F80302D50F980004286084
:104B90000F984104B80300D52960380400D4E4E13B
:104BA000039402910E9308920D980B990C180A9891
:104BB0000C9941430C910F98C0030B90286008F0AA
:104BC0002DF9002801D005F0D7FA0C98005B410BB5
:104BD00043D1099800190E99401805990901401808
:104BE0000E90E74D287B079B4343E97A0A010D9C11
:104BF0002243D21841188B00D2180A9B4B43D1187C
:104C00006A7B564389190E9E2A791018DF4A12884A
:104C10004243881816903068C000800D10A9C882E1
:104C2000002511957079C0077ED110A80F99818257
:104C3000069C00940020E8A2049B0BF061F978E048
:104C40000F98820522603A0200D43FE70F98C20510
:104C50002260FA0100D53BE73DE707214903084000
:104C6000032149038842089A00D07EE1069707F0A5
:104C700049FD0020169009901590C14CE07A217BE7
:104C800008180A99414380000D9A10434118627B2D
:104C90000E9672438A186178A379079E7343D718DA
:104CA000FA683F26324063789A420C976ED1059697
:104CB0000A9A4A4380580F210A0702400398401E6F
:104CC000C04B1B68DB090340981810900F98C00276
:104CD0000B90B868800767D42C46283C0AF086F809
:104CE00005462068000609D5C3208401786A40077C
:104CF00004D40AF07BF8401BA042F7D905980002C3
:104D0000B96849080140B34803688268B868C40CB0
:104D100020202040DB0700D095E0002310221D4614
:104D20001C460E9E0B9FB1E010A88582B0681190C2
:104D3000069C701D924B1979E20707D1491C197125
:104D4000D97A1A798A4202D31D7100E0D9700178AC
:104D50004278120251188278120489180322914372
:104D6000017035715878401C5870D87A197B081832
:104D70005978884200D85D70D879401ED871596B37
:104D8000002901D010A888477E4DEDE010A80B99AE
:104D90008182F86830406378009000207CA20F99EF
:104DA0000BF0AEF80E9E94E0388A874A024010A8B5
:104DB000C2822022BA5C9307DB0F3C68C3720F9B50
:104DC0001A4082726205D20C0D9B1A431692FA6841
:104DD000130E0372BB69FC697C4D2D682D0C0574A4
:104DE0005204920F427211931394654CA07B0028D9
:104DF00009980E9E0B9F5FD075480068007A0328C3
:104E0000099859D00C98007D08400928099853D179
:104E1000C320840109F0EAFF05460C98406A410767
:104E20000BD4594909680906890F06D109F0DEFF3C
:104E3000401BA042F1D90C98406A4103089888436E
:104E400010A9888237E0D2070E9E0B9F03D108235A
:104E50000022154619E00C9B9A68029C224211D14F
:104E60009A68520C022494430022134615460DE022
:104E70001CD2010228A000503CA10050FC1F0000E1
:104E800018D2010204250022134614460843104399
:104E900018432843204310A9888238420BD10C9B29
:104EA000198A494A0A4010A9CA8219684905C90CD9
:104EB0000D9A11431691324C2921615C002908D0CA
:104EC0003037B84205D010A908461130123109F028
:104ED000A7FAE77A2A48047BE519294800790E9059
:104EE00027484078401C2946FBF7F4F888000D9AC3
:104EF0001043189007996143380110434018204926
:104F0000497B4E4380191C21694340180E990919A9
:104F10001B4B1E4A12884A4380181790099A0C9915
:104F20008A60987B002800D04A629879401C98716A
:104F3000187B99798142069F00D39A715978491C50
:104F40005970D97A0818597888420E4D00D85A708D
:104F5000187A401E18722820185C002804D0996B1B
:104F6000002901D010A88847089A174202D00F984C
:104F7000000328601C480449486019B0F0BDC046D1
:104F80001CD2010228A000503CA1005018D20102FE
:104F900048572045542069647820256420616E6458
:104FA0002045542069647820256420696E20525879
:104FB0002064657363206D69736D617463680D0AA5
:104FC0000000000038200040FF0300009430004043
:104FD00044940102604000404D4143204556542016
:104FE00025782025780D0A00FFFFFF03F0B5A5B056
:104FF0001E460C9208910024239422A90C8016A925
:105000000C8024A909250D80598C0D91FBF762F8BD
:105010002A99012900D0DFE03189012900D0DBE0A5
:10502000318C012900D0D7E00D99002900D1D3E0BF
:10503000224607962C990B912B99069180B20590E8
:105040000F9415A8058090000E900C990C582E46D0
:105050000025204629461746FBF7E4FB0028119659
:1050600036D12C200A9778430899081817A90A46C0
:1050700068C868C2E8C8E8C2E8C8E8C2079F1198D3
:1050800080B280000E5822AD019523A800902046E2
:105090003946059A069B04F0BBFD0F98401C0F9003
:1050A000288800282DD03B8A239913AC039416A896
:1050B000029014A8019015AE009617A824AA04F037
:1050C00081FF2588308811900120149E0A9A05E0FE
:1050D00013A8058014952E4628463A460E9F510087
:1050E0000B9B119C5C52591808830D84D81986605B
:1050F0000F981885521C0D9882426DD024A80588FF
:105100009FE7099616A800250580149524A806880F
:10511000239812902F46109503E06D1CA8B2B04260
:1051200013D8A8B2800017A90C5820461299FBF793
:1051300087FB0028F1D1002FEFD115A8058016A814
:105140000127078014941094E7E715A80288B01A85
:10515000012805D115A80680099F1497119628E00B
:1051600010200799095E0129119221DB551CA8B274
:105170000C18109F0E9B099403E06D1CA8B284428A
:1051800018DDAAB2B242F8D8800017AA10581090C1
:10519000394634461E46FBF745FB33462646099CF6
:1051A0000028EAD115A80580109F14971195E4E70F
:1051B000109F0E9B1C463E4638461299FBF761F93C
:1051C000FBF7ECFB0546052800D3052513A8058051
:1051D00001200A9A274682E725B0F0BDF0B58BB0D2
:1051E0000243159A149C139E2BD0054601A856C065
:1051F000129CD869196A09900A911E469F6B012377
:10520000009309A807AA0146059306F0DDFC716C1E
:105210003846FBF736F90746E06A616BFBF731F970
:10522000002D069613D0044611980199012924D126
:105230000921081A0421069A515E884229D1642561
:10524000B1E000203080207010700BB0F0BDB0884D
:1052500000226425002829D0059269493846FBF7C9
:105260000BFB0028049C039E6FD166493846FBF770
:1052700003FB00281DD05A2567E03C25082800D1F3
:1052800091E05F492046FBF7F7FA002819D0502536
:1052900089E00A291DDB1D293BDC59493846FBF70B
:1052A000EBFA0022002854D05A253AE03346049CF9
:1052B00039E055493846FBF7DFFA002821D0502560
:1052C00043E050492046FBF7D7FA00282ED0462568
:1052D00069E03C25012866D049492046FBF7CCFA15
:1052E0000028D4D147492046FBF7C6FA0028EED162
:1052F00045492046FBF7C0FA002854D143492046CF
:105300006EE042493846FBF7B7FA00281CD1282541
:105310001BE03B493846FBF7AFFA0022002832D0A9
:105320005025049C069B0299039E41E03649204685
:10533000FBF7A2FA002836D134492046FBF79CFA45
:1053400000282FD114252EE037250299059A069BB7
:105350002EE005922B493846FBF78EFA002896D1AD
:1053600029493846FBF788FA0028B0D12749384642
:10537000FBF782FA0028049C069B0299039E059A7B
:105380003BD11E2514E005921E493846FBF774FAFE
:1053900000289CD11C493846FBF76EFA00281DD026
:1053A0003C2500E02325049C069B0299039E059A58
:1053B0002580327000200870307800280CD11868E1
:1053C0001349FBF74BFA002806D12088102803D395
:1053D0000F3820800BB0F0BD0BB0F0BD0B49384644
:1053E000FBF74AFA0028049C069B0299039E059A43
:1053F00001D11425DCE72325DAE72D25D8E7C046BF
:10540000CDCCCC3DCDCC4C3DCDCCCC3C0AD7233CF7
:105410000000204070B588B00C4606464088002841
:1054200020D0FBF77CFA059005A804A901252A469F
:1054300006F034FE3088B188081AFBF765FA03904D
:10544000049903A807AA2B4606F0E8FD5249079DD8
:105450002846FBF711FA002808D0BF20000620607C
:1054600008B070BD0020206008B070BD4B492846D0
:10547000FBF7E6F9002804D03F200006206008B0C2
:1054800070BD47492846FBF7F7F9002801D00020F6
:1054900010E000212846FBF7EFF9002801D0022098
:1054A00008E040492846FBF7E7F9002801D004202E
:1054B00000E0062001957F21C905029180003A494C
:1054C000091801A806AA022306F05CFD06982060D0
:1054D00008B070BDF0B587B00C4605464768002699
:1054E00038463146FBF7D6F9002802D0266007B0CF
:1054F000F0BD049704A803A90126324606F0CEFDAC
:10550000A8682968FAF778FF0290039902A806AA0A
:10551000334606F083FD2049069D2846FBF7ACF98B
:10552000002804D0BF200606266007B0F0BD1B4946
:105530002846FBF785F9002804D03F2006062660A0
:1055400007B0F0BD16492846FBF796F9002801D0B0
:10555000002010E000212846FBF78EF9002801D03A
:10556000022008E00F492846FBF786F9002801D001
:10557000042000E0062000957F21C90501918000EC
:1055800009490918684605AA022306F0FBFC059E96
:10559000266007B0F0BDC046CDCC0C3F295C0FBFE4
:1055A000CDCC4C3ECDCC4CBE4C940102F0B587B076
:1055B0000C4606467F270088002801D0FD0503E041
:1055C000B08800282ED0334DFBF7A9F903907088DE
:1055D000FBF7A5F9049003A802A90126324606F0BC
:1055E0005DFD029904A806AA334606F017FD2A4974
:1055F000069E3046FBF740F9002802D03F20010606
:1056000041E026493046FBF71BF9002802D0BF20B5
:10561000010638E022493046FBF72EF9002805D074
:10562000002024E00020206007B0F0BD1D49304676
:10563000FBF722F9002801D0022018E01A49304671
:10564000FBF71AF9002801D0042010E01749304672
:10565000FBF712F9002801D0062008E01449304673
:10566000FBF70AF9002801D0082000E00A20009684
:10567000F905019180000F490918684605AA02231F
:1056800006F080FC05992846FAF7BEFE206007B0B8
:10569000F0BDC046000080BF000038433333733F85
:1056A0000000C84200007042000020420000A041FB
:1056B0000000C0406C940102F0B59DB015460B91FE
:1056C0007F210391C9051C9102911B9119A9002406
:1056D0008C80199418941794598C0691198C0F91F9
:1056E000DE8B998B0791997805911F882B21CA43EE
:1056F0002799914201DB7F0015E04022D24391427D
:1057000011DC4922D243914202DB7908CF190AE029
:105710005322D2439142EEDA5D22D243914201DB21
:10572000BF0000E0FF000A971396269E597E0029CD
:105730000BD0002132460F46D1709170517011701C
:10574000121D7F1C5C7EA742F6D30C931195259900
:10575000149122990D91159041088C4211D2FD4A65
:105760002346A00084583454270A451C7755250C3D
:10577000871CF555240EC01C34545B1C9CB2A142FE
:10578000EFD82398109001200990009030463146C0
:10579000149A159F3B4606F025FA0D9800060890CE
:1057A000400E139D00D186E068000490002F3FD08A
:1057B000002210461146144606E01C461146159F6D
:1057C000401C82B2BA420ED283B2AB42F8D09200F1
:1057D000149B9A5E0FB2BA42034600DC2346BA42DB
:1057E000EBDC0A46E9E7002F25D0002210461146DF
:1057F000129206E012931146159F401C82B2BA42E3
:1058000014D283B2AB42F8D0A5B2AB420CD0920016
:10581000149B9A5E0FB2BA42034600DC129BBA4256
:10582000139DE7DC0A46E5E7139DE6E7129903E0DE
:105830000024214600E00021129110980183C482C7
:105840008582049FF057FBF75FF87921C9050E9117
:10585000FAF7DAFD1099C86109980743F057FBF78A
:1058600053F80E99FAF7D0FD109F38622004C40B4C
:105870003057FBF749F80E99FAF7C6FD7862601CBD
:105880003056FBF741F80E9C2146FAF7BDFDB86291
:1058900012980004C70BF057FBF736F82146FAF7C9
:1058A000B3FD109CE062781C3056FBF72DF80E9982
:1058B000FAF7AAFD2063119805800C98407E4100FC
:1058C00000278D4228463A46149E1ED30A9880B27D
:1058D0008AB29300F45E84420BDA491C8AB2AA426F
:1058E000F6D9002728463A4681B2691A012910D014
:1058F0001BE0F018119B1980078808040FD0500096
:1059000040008019001F0288084681B2691A0129E7
:105910000BD1A800301811990D80078826E00020CF
:10592000024681B2691A0129F3D00A9989B2079B0C
:105930004B43BB421AD306998A4217D805990029CE
:1059400014D0401C82B2891803E0401C82B29142FC
:105950000CD983B2AB42F8D89200B35EBCB2A3427A
:10596000F3DDB218119B18801788EEE712970B9899
:105970000580119800882B1A002B16DD02210F9A42
:105980001143032942D10E93411C421E10B28142A1
:105990000EDA0E98032824DB0C98808C012820D086
:1059A00019A818A9FFF736FD1FE0002018902BE07A
:1059B0000026F443374608E0B8B2400019AD2B5238
:1059C0007F1C521C10B28142E3DB13B2A342334668
:1059D000F2DD159B98423346EEDA8000149B1B5A89
:1059E000EAE719A818A9FFF7E1FD149E139D0F9A85
:1059F000012A13D0032A11D0022A04D11198008859
:105A0000281A02280ADA0020179034E0022A01D16D
:105A1000022BB8DA00201890012AEBD1681C691E0D
:105A20000FB2B84208DA0C98808C01281DD119A851
:105A300017A9FFF7BBFD1CE00022D343144608E082
:105A4000A5B26D0019AF7E53641C491C0FB2B84259
:105A5000E9DB0DB29D421646F2DD159DAF421646BA
:105A6000EEDABD00149E765BEAE719A817A9FFF7E6
:105A7000D1FC149E139D249F189C17992046FAF779
:105A8000BBFC0F99012900D8204638600D980028EA
:105A900000D1CBE011990888109FB8860888281A91
:105AA000B880129880B2FAF73AFF7921CC052146E6
:105AB000FAF7AAFC2146FAF7A7FCB863119F3888C9
:105AC000002849D081008919091F0988129C0C19E6
:105AD0001599884203D2800080198088041915988E
:105AE0004300534916AA304606F05AFA1698109900
:105AF0004864FAF76CFFA4B2A04201D14D480FE010
:105B0000001BFAF70CFF1C901CA81BA9012206F031
:105B1000C5FA2046FAF703FF01461B98FAF774FC12
:105B2000109908603988491B4A1C92B2032A02D294
:105B30000021159F17E009B20229159F12DB3F21B2
:105B40000906FAF799FE002802990CD109988107F5
:105B500009E0C046402100400020129C159988426F
:105B6000B9D3BCE73449109801610898800E5DD024
:105B7000002F1CD000221146144610464B1B1DB2AC
:105B8000ED135B196B40139D1BB29200B25E534341
:105B90001818A418491C8AB2BA42EFD3FAF7BFFE0C
:105BA00006462046FAF7BBFE002C03D100E0002693
:105BB0000398C0051C901CA81BA901252A4606F0C5
:105BC0006DFA1B9C20463146FAF71EFC01461098E0
:105BD0008160002F119422D0002427462646139579
:105BE0001291B8B2FAF79BFE1299FAF705FC054636
:105BF000A0001499085EFAF787FE01461398C007C3
:105C000085432846FAF700FC01463046FAF7A3FB25
:105C100006467F1CBCB215988442E2D300E0002601
:105C200011983146FAF7F0FB1099C8601DB0F0BD2D
:105C300068A701020000204100004040F0B58FB08D
:105C40000692F74A09AF70CA70C770CA70C70328B6
:105C5000079320D88800F3A10858F649FAF77BFB90
:105C60000446F549FAF777FB0D90F4492046FAF718
:105C700072FB0C90F2492046FAF76DFB0B90F1494C
:105C80002046FAF768FB0A90EF492046FAF763FBD3
:105C90000990EE4969E0042822D0062820D888001F
:105CA000EBA10858EE49FAF756FB0446ED49FAF71E
:105CB00052FB0D90EC492046FAF74DFB0C90EB4956
:105CC0002046FAF748FB0B90E9492046FAF743FBD8
:105CD0000A90E8492046FAF73EFB0990FD4944E066
:105CE0000838022821D88800FBA10858D149FAF7C2
:105CF00032FB0446FC49FAF72EFB0D90FB49204687
:105D0000FAF729FB0C90FF2081052046FAF723FBC8
:105D10000B90F7492046FAF71EFB0A90CA49204625
:105D2000FAF719FB0990FE491FE08800F1A1085815
:105D3000F449FAF710FB0446F349FAF70CFB0D900F
:105D4000F2492046FAF707FB0C90F1492046FAF792
:105D500002FB0B90EF492046FAF7FDFA0A90EE4954
:105D60002046FAF7F8FA0990EC4900942046FAF731
:105D7000F2FAEC4909680E90EB480468EB480168B8
:105D80004808EB4F05463D400022002D08922DD0DB
:105D9000CA01120E07D0280CE90D12D14000E649C5
:105DA000085AE6490AE0C903090E0CD0280AE90B93
:105DB00010D14000E049085A8F2189004018E43092
:105DC0000DE0DC490AE081B27F2905D84800DA49B4
:105DD000085A04E0D94901E08F218900401800B237
:105DE000FAF792FDD649FAF70FFB024602920395A5
:105DF00007252606D34B1A68002A089840D0791C3C
:105E00008A420BD21102090E13D0110C1F46D00D7D
:105E10001FD14800C849085AC84907E01F46110E5B
:105E2000002A13D44800C449085AC2494018E43033
:105E30001FE011041F46090E0ED0110AD00B12D11B
:105E40004800BD49085A8F218900EFE7BE4808186D
:105E50000FE0B84808180CE091B27F2906D8480036
:105E6000B549085A05E0B548081802E08F218900B5
:105E7000501800B2FAF748FDB149FAF7C5FA3B46A7
:105E80000590159F2C40F50E5B69B04919400898A4
:105E900010D0DA02D20E34D0C80B3E210140A64801
:105EA000405AA6494018E43000B2FAF72DFDA44943
:105EB000FAF7AAFA0490149E6800A5A1085EFAF702
:105EC00023FD0146A00009AA1058FAF744FA01463A
:105ED000B8B20128089F019102D1022C0AD9A74F1C
:105EE000052C24D1189808900C2D20D80B2D16D3F2
:105EF000A44918E00027022C089718D08120C70574
:105F000015E01A04120E00D1CAE0080AC90B00D02D
:105F1000CDE040008849085A8F218900C2E7092D49
:105F200000D2C7E096490898FAF715FA08900120C0
:105F30000021B542034600D30B46052C00D308468A
:105F40001799169A1A9C199D1843069B012B12D17A
:105F5000079B402B22D1002840D03846FAF7FBF9A6
:105F600001460198FAF7F7F901460098FAF744FA62
:105F7000059A04998AE0079B402B1FD1002838D04E
:105F80003846FAF7E8F901460198FAF7E4F90146CC
:105F90000098FAF731FA059A049977E0002833D08F
:105FA0003846FAF7D8F901460198FAF7D4F90146CC
:105FB0000098FAF721FA059A049967E000285BD067
:105FC0003846FAF7C8F901460198FAF7C4F90146CC
:105FD0000098FAF711FA059A049957E002981146C9
:105FE000FAF70AFA0399002900D16748059A04993B
:105FF0004CE002981146FAF7FFF90399002900D105
:106000006148059A049941E002981146FAF7F4F9BB
:106010000399002900D15C48059A049936E0C046EE
:106020009C1F0100000068C1000088C166665EC157
:10603000000084C1000084410000B44100004841D8
:10604000000020400000F0C0000084C10000F841C2
:10605000333323C1000050C19A9929C19A9949C18B
:106060009A9949413333CB4166667641CDCCAC40F9
:10607000333393C09A9949C102981146FAF7BCF993
:106080000399002900D14048059A049928601046D8
:10609000FAF7B2F90899FAF7AFF920600FB0F0BD3E
:1060A00099B27F2911D848002349085AFCE62349B0
:1060B0004018F9E6C12001060898FAF74CF9089053
:1060C000062D00D933E7002030E78F2189005818CA
:1060D000EAE6C0463333F341000058C19A9961C1E2
:1060E0009A9969C1000084C10000AC4100003841A8
:1060F000000008C1CDCC80C1CDCC88C133338FC165
:10610000333397C133339741CDCC8C413333F34094
:106110009A9919C0666646C1333397C1CDCCB44154
:106120000000D4410C000040503000406840004066
:10613000FFFFFF007C080000A82301005C050000B1
:10614000919AF63C642000409C0B0000FFFF1F006A
:10615000FAFFFCFFFEFF000002000400060008003A
:106160000A000C000E0010001200140016001800A7
:106170001A001C001E00200022002400000080BF26
:106180000000A0C0000040C00000DCC2F0B5FFB0BD
:10619000ECB017460E460D900021E991E891DC9194
:1061A00099919891979196911491139112919AA81F
:1061B000F49DF39CF29A002E00D1E6E10B9380301F
:1061C000F09B1180099529602546DBAC218095ACB8
:1061D00021800C952980DA917F24E405B994B89444
:1061E000B794B694B594B494B394B294B194B09473
:1061F000AF94AE94AD94AC94AB94AA94A994A894A3
:10620000A794A694A594A494A394A294A194A094D2
:106210009F949E949D949C949B949A940466446647
:106220008466C466046744678467C467046444641E
:106230008464C464046544658465C465046244621E
:106240008462C462046344638463C463046044601E
:106250008460C460046144618461C461B0090B2539
:106260000B2800D3AE011095012B0B9D00D070E1DF
:106270002B89012B00D06CE1298C00290E9200D1D2
:106280008BE16B8C002B00D1FAE1AA8C3021695C88
:10629000002900D188E10892109F5F431196304693
:1062A00039460F93F9F716FF0590FAF72DFB0146D3
:1062B0002046FAF7E6F88321C905FAF7A5F806465D
:1062C00096A8021D119887420A9200D879E155A834
:1062D00011909AA9069196AF15463A46059C234619
:1062E00005F050FE15A80F9006992A46234605F0A2
:1062F00049FE02230D93384631463A4605F08EFE9C
:10630000012308930093E8AA10923846394605F015
:106310005BFCE898DD901198069D29463A46234695
:1063200005F030FE0F9829460A9A234605F02AFE0A
:10633000384631463A460D9B05F070FE089B0093A7
:1063400038463946109A05F03FFCE898DE901198DF
:106350002C4629463A46059D2B4605F013FE0F981C
:1063600021460A9A2C462B4605F00CFE384631464B
:106370003A460D9B05F052FE089B0093384639467D
:10638000109A05F021FCE898DF901198069D2946A7
:106390003A46234605F0F6FD0F9829460A9A234609
:1063A000254605F0EFFD384631463A460D9B05F08F
:1063B00035FE089B009338463946109A05F004FCD8
:1063C000E898E0901198069C21463A462B4605F045
:1063D000D9FD0F9821460A9A2C462B4605F0D2FD8E
:1063E000384631463A460D9B05F018FE089B00934F
:1063F00038463946109A05F0E7FBE898E190119885
:10640000069D29463A46234605F0BCFD0F982946CD
:106410000A9A2346254605F0B5FD384631463A46E8
:106420000D9B05F0FBFD089B009338463946109AFA
:1064300005F0CAFBE898E2901198069C21463A467E
:106440002B4605F09FFD0F9821460A9A2B4605F032
:1064500099FD384631463A460D9B05F0DFFD089B15
:10646000009338463946109A05F0AEFBE898E39061
:10647000119821463A462B4605F084FD0F98214697
:106480000A9A2B462C4605F07DFD384631463A46A1
:106490000D9B05F0C3FD089B009338463946109AC2
:1064A00005F092FBE898E4901198069D29463A463B
:1064B000234605F067FD0F9829460A9A254623468C
:1064C00005F060FD384631463A460D9B05F0A6FDC5
:1064D000089B009338463946109A05F075FBE898FA
:1064E000E5901198069C21463A462B4605F04AFD58
:1064F0000F9821460A9A2B4605F044FD384631464E
:106500003A460D9B05F08AFD089B009338463946B4
:10651000109A05F059FBE898E690119821463A4602
:106520002B4605F02FFD0F9821460A9A2B4605F0C1
:1065300029FD384631463A460D9B05F06FFD089B14
:10654000009338463946109A05F03EFBE898E790EC
:106550007AE010880C9A108099919891DA9E0846FA
:106560000F46099DF59CF9F747FF2860DC982760E6
:106570006060A6600C34DDA80EC80EC42EC82EC400
:106580002EC82EC47FB06CB0F0BDFF20108000215B
:10659000296020807FB06CB0F0BD00220123302143
:1065A000695C002900D076E6DDAA1ACF1AC23ACF7C
:1065B0003AC23ACF3AC20B213046F9F78BFD054675
:1065C00042E000200690059D0796089F11900698CE
:1065D00001460D9C0F9A4A43D219109B5A43119BB6
:1065E000D218D200A35889002E4655AD6B503546BF
:1065F000121DA25815AB5A50401C01B28E42E9DC64
:1066000055A89AAE96AC314622462B4605F0BAFC08
:1066100015A831460A9A2B4605F0B4FC0223204601
:106620000799224605F0FAFC01230093E8AA2046C8
:10663000214605F0C9FA119B9800DDA9E89A0A5095
:106640005B1C0B2B1846C1D1F19EDDA89AA9DCAAD0
:106650000B2305F097FC09210E980F9101800B98F0
:10666000C168DC9C2046F9F7CFFE0146A8B2E69F40
:106670000F281BD808280DD30846F9F76CFE14E044
:10668000FF2010800021099A11600C9908807FB0CA
:106690006CB0F0BD042803D381220846D10502E086
:1066A000412208461106F9F7AFFE01462B20C043F0
:1066B00086420D9704DB0846F9F74DFE014603E0DC
:1066C0004020C043864244DD0E9A0C9C0B98408AC1
:1066D000002811D00B98038A95A80390DBA802909C
:1066E000DAA801900094DDA80D4603F06BFC294662
:1066F0002488DA9E099D68E011910F982080002778
:106700003D46109705E00E9804887F1CB8B2A04261
:1067100011D8B8B28000DDA90C5820461199FAF7BB
:106720008FF80028EFD1002DEDD10C9807800125BE
:106730000F971094E7E7DBA805800F9A90B2201A14
:10674000012811D10C9804800D9FDA973E46099DCF
:106750003AE04920C043864200DA8BE0FF22084637
:106760009105F9F751FEA9E710200B990E5E012E55
:1067700000DA90E0551CABB21846A1B2AAB28A4228
:1067800017D805E00E990C88A1B2AAB28A4210D897
:106790008000DDA90C58204610991F46FAF742F8F0
:1067A0003B46002805D10C9805800B98068A0F956A
:1067B000109430B2C1186D1CA8B28142E2DC109E68
:1067C000DA960F9C099D0D9F11993046F9F759FEF5
:1067D000FAF7E4F8052800D3052095A90880A0B2AF
:1067E0000E990988814218D9401C611E0CB2A04242
:1067F00018DA12A898A9FEF76DFE0E980188481CB9
:10680000491E0CB2A04221DA12A899A9FEF762FE35
:1068100099999898099D0D9FA4E6002198919991C6
:1068200008469FE60022134608E09CB2A40012AF7F
:106830003D515B1C491C0CB2A042DADB8DB20A2D23
:106840001546F2D8A400DDAD2D59EEE7002213461F
:1068500008E09CB2A40012AF3D515B1C491C0CB275
:10686000A042D1DB8DB20A2D1546F2D8A400DDADD1
:106870002D59EEE75320C043864200DB1BE70E464E
:106880000B9881692046F9F7CDFF00280C9C08D1B0
:106890000B98808B07E01446099D0D9F1199109E5F
:1068A00093E70B98C08BFAF73AF801463046F9F7B0
:1068B000ABFD119021E70000F0B58BB01C460993A9
:1068C0000E46034600200A9040480088224F059754
:1068D0000AA9049103940292109C01940125009549
:1068E0000B21414389B230331C4A3046FFF74EFC3E
:1068F0003868079078680890B86806903348008830
:10690000334F009501940297324E30363249334A64
:106910003346FEF76BFB0698F862079838630898D1
:106920007863099800882E4905912E4904912E49D3
:1069300003910297019000962C4B284629462A463F
:10694000FEF74CFC432001060A98F9F75DFDFAF7C3
:1069500025F80BB0F0BDC04630A70102E8DF010208
:10696000F0B589B00F9F0E9C002815D010980790A5
:1069700016480088164E012500950191029608934D
:10698000144B30331449154AFEF730FB089BF7626D
:1069900007983063746303E00D484763C4620025C1
:1069A00018880F4905910F4904910F49039108492F
:1069B0000291019007483030009001210B4B28468E
:1069C0000A46FEF70BFC09B0F0BDC046D4AD01028B
:1069D000ACD4010294A001021C9F0102BCD20102AE
:1069E00060A40102D0AD010270AD010278AD0102D8
:1069F000304870470048704714AE010280003749A4
:106A00000918C86B0022CA637047C046800033492A
:106A10000918886C00228A647047C04680B52F4AE6
:106A2000D369002B01D0126A9847002080BDC04670
:106A30000249087800220A707047C04684C90102E2
:106A40000020704780B5182905D803468A1E0348E0
:106A50001946F9F78FFB002080BDC046D8AD010272
:106A6000B0B502460020022901D2C043B0BD8C1E41
:106A70000F2C07D8044D284611462246F9F77AFB19
:106A800000202855B0BDC046F4AD0102B0B50246A5
:106A90000020022901D2C043B0BD8C1E0F2C07D8A4
:106AA000044D284611462246F9F764FB002028557C
:106AB000B0BDC04604AE01020849087800220A7041
:106AC0007047C046B0B50446044DAA68002A02D0FB
:106AD000E968204690472C610020B0BDE497010290
:106AE000B0B5D44DE869002819D0284800780028AE
:106AF0001BD0012829D127480068CD498A8A9042B5
:106B000024DA2878002804D000202870022002F01F
:106B100047F90020687028621D490870B0BD002048
:106B2000286268701A490870B0BD2878002803D11F
:106B30000120287002F034F915480121017000206D
:106B400028626970C04313490860B0BD01246C70AD
:106B50002A6A531C2B62C98A884209DD132AF4DB96
:106B6000287800280DD12C70204602F019F908E091
:106B7000132AEADB2878002803D12C70204602F083
:106B80000FF90020286202480470B0BD6899010224
:106B9000E59601028C99010280B5124801681F2216
:106BA0000A40026003200840022812D10E48026801
:106BB000D30D02D0FF231B06D2180C4B1A600C4ACF
:106BC00012680C4B1A6080680B4A1080000C0B4A4C
:106BD00010801A488268002A02D0826800209047FC
:106BE00080BDC0467420004064400040D0D2010205
:106BF00078300040D4D20102F8A00102A2D40102F0
:106C000080B50D48016889070FD5052101600B4843
:106C1000C178002908D00021C170C168002903D0C3
:106C2000C26841680020904780BD054805A10B4A15
:106C30000BA308F009F9C0462C040040349401026B
:106C40000C3D01005048595F54494D45525F49522F
:106C50005148616E646C6572000000008D0A00008E
:106C6000556E657870656374656420696E746572CD
:106C7000727570740000000070B50446401E012853
:106C800014D80320084011D13F2040030818050BF9
:106C9000281980280AD8164E317801204840294604
:106CA00004F0EAF8641E6D1C002CF5D170BDC046DE
:106CB00080B50020014603F027FE002800D080BDEB
:106CC0000B480121017080BD70B516460C46054683
:106CD000FF22F9F761FA05483118054802780120CA
:106CE00050402A46234603F06FFF70BD00E00704C2
:106CF00068A901020120000370470120400370478A
:106D0000F0B585B048484949016005F0DBFF484DC2
:106D1000E98A4A2247488152AA8A4823C252AB884C
:106D20008362AC7A0471AC89C48102824182A98DEC
:106D30000187049383864A1E91414900C161A88B53
:106D40003B2801D83C20A8830020E883288B3A49BF
:106D500008804120800068806C8C0F202246024011
:106D60007D21C900260B4E43B6182205170F642259
:106D70005743F6192406270F0A246743F6192F4FA5
:106D80003E80AE8C374607402B46350B4D43ED1900
:106D900037053F0F5743ED193606360F6643AD19D9
:106DA000274E3580DD8C2E4606402F0B4F43BE19F3
:106DB0002F053F0F5743F6192D062D0F6543751903
:106DC000204F3D801D8D28402E0B4E433018290545
:106DD000090F514340182906090F614340181A4E04
:106DE0003080032419A220462146049B09F088F82C
:106DF0000F484088C1B20091030A18A220462146DC
:106E000009F07EF80D4803880D48008839883288DB
:106E1000094D2D8800AE27C619A22046214609F04B
:106E20006FF805B0F0BDC046009601026584000011
:106E30006AA90102B8980102AC960102A496010267
:106E4000A6960102A8960102AA960102C9E8B1B865
:106E500049443A202578202E0D0A0000B9CCBCFE0A
:106E6000B0E6B1BE3A5557422D3447B3B5D4D8CA6F
:106E7000D6BBB7205625642E25642E200D0A0000AF
:106E8000B7FECEF1C6F7B5D8D6B73A2025642E2581
:106E9000642E25642E25643A25642E0D0A00000018
:106EA000F0B583B030480068C16B0901890F01D08B
:106EB00003B0F0BDC16BC06B2C4D05404800400FC6
:106EC0000826029686400227384602F0C3FD01904C
:106ED0007043C10B4A1B26485043F9F711F9044689
:106EE00007F0F4FE032123A238461F4F00912346EA
:106EF00009F006F8F88A002817D0019840012946C1
:106F0000F9F7E8F846431822324001200F2A0146DB
:106F100000D8002173095B181B4CA3420DD8194DF2
:106F2000ED1A6D050F2A0CD80CE038680021C160FD
:106F3000112002F07FFD03B0F0BD5D1C6D050F2A2E
:106F400000D956422A0C029D2E4009018919A342FC
:106F500002D80098000400E040040818801839683E
:106F6000086303B0F0BDC046C4940102FFFF1F00D8
:106F700040420F0052434F33324B2070706D20253A
:106F8000640D0A00FF070000FE7F0000B0B582B06C
:106F9000154908688269D2070CD00122C2610D69C7
:106FA000002D07D000686C46214607F02FFC002119
:106FB0002046A84702B0B0BDB0B582B00A49086803
:106FC000026C92070ED5026C012313430364CD6853
:106FD000002D07D000686C46214607F017FC002101
:106FE0002046A84702B0B0BDC4940102064801681B
:106FF000032291430160016801220A43026000F00C
:107000004FFB07F085FEC0462800004080B50D49C3
:107010000868002810D5224802680423032A01D0FA
:107020001A4300E01A460A601E490A68002A02D084
:1070300041680020904780BD03A00CA19E2211A3AF
:1070400007F002FF2C100140696E636C7564652FB8
:10705000647269766572732F6D6B5F736C656570B2
:107060005F74696D65722E6300000000534C4545E6
:10707000505F54494D45525F49525148616E646CAE
:1070800065720000556E6578706563746564207381
:107090006C65657020696E7465727275707400003D
:1070A0000C900102A8D40102B0B582B00446007869
:1070B000002811D0094D01A908702868416A0029EB
:1070C000FCD101A901220020034609F0DBFC611C70
:1070D000607800280C46EED102B0B0BDFC940102ED
:1070E000F0B50C784D782D022C198D78C9780902ED
:1070F000491909040C1981000E4D6C509478D5780B
:10710000167852780C4F7B50120292192B021B19E1
:107110001B049A18094B5A50059A13785278084C58
:10712000079D65504000074908181102C9184822F8
:107130008152F0BDCC9F010290E0010230A001021B
:107140002CE001021896010210B5CE4C21680629E8
:107150000FD8012002468A4058210A4209D02060F7
:107160000020A0602369002B03D062690020022167
:107170009847C3482258062A12D801210B4693404B
:10718000582213420CD0215020180021816003693D
:10719000002B05D0AD20C0002258012002219847C5
:1071A00047482258062A11D801210B4693405822FD
:1071B00013420BD021502018002181600369002B5D
:1071C00004D003482258022001469847002010BDF1
:1071D000BC0A0000F0B581B00024022803D9E443C2
:1071E000204601B0F0BD17460B46094E46430948FC
:1071F0008519284618302A2107A2FCF74FFF4220A4
:107200002F52032003498851204601B0F0BDC046EB
:107210005405000094AE010225730000F0B585B05E
:10722000E04D2C68002C0CD0DD4FDE4CE659002ED2
:107230000CD0234FE659002E0DD00020C04305B0DE
:10724000F0BD01AC0FC400272E4608E001AE0FC60A
:10725000E619012703E001AE0FC6E6190227D04C5C
:1072600030462146FCF700FE022030607C4329199D
:10727000029D4D60CF6003980861049848610846FC
:107280004430CC310122560210233246FCF7E2FF93
:10729000E4480019B32189004118012D05D1B83007
:1072A00001233246FCF7C1FB04E074301023324660
:1072B000FCF7D0FF01980760002005B0F0BDC04684
:1072C000A80A000001460020022901D9C0437047E6
:1072D000E24A4A43E24988507047C046022806D82D
:1072E000E6494143E64840180249401870474B20A0
:1072F00080007047D4040000022802D94B2080008F
:107300007047DE494143DE4840184D21090140588D
:107310007047C046032801DB03487047D749414303
:10732000D748401818307047193B0100022806DC86
:10733000D2494143D24840184221405A7047002068
:107340007047C046032801DB00207047CB4941430A
:10735000CB48401844307047022804DCC7494143F9
:10736000C7484058704700207047C046022805DCD7
:10737000C2494143C24840184068704700207047E6
:10738000B0B50024E14302280FD8BC4A4243BC4BAD
:107390009D58042D09D0991801220A600B69002B11
:1073A00005D04A690221984721460846B0BD2046CB
:1073B000B0BDC04610B50024022801D9E04310BD7D
:1073C000AE494143AE4A0723535051180B69002B75
:1073D00003D04A69002421469847204610BDC04684
:1073E000F0B581B00024022803D9E443204601B05F
:1073F000F0BD0546A1486843A14906220A500F186E
:10740000384644303946CC310122560210233246E8
:10741000FCF720FF786801280CD1B32080003918D0
:107420003846B83001233246FCF7FFFA3B69002B9F
:107430000CD1DBE7B32080003918384674301023B4
:107440003246FCF707FF3B69002BCFD07A69012158
:1074500028469847204601B0F0BDC04610B500242C
:10746000022801D9E04310BD84494143844A5118A0
:107470000B69002B02D04A6903219847204610BDB2
:107480005405000094AE0102F0B583B01746002405
:10749000E24302281AD8002B18D00D467749414301
:1074A0007748461870680128029312D1002F0AD03D
:1074B000B836002429193046FCF7BFFA002825D138
:1074C000641CA742F6D1029807600022104603B060
:1074D000F0BD019274363046FCF777FE002811D0DB
:1074E00003464268BA4209D2196828461D46F8F791
:1074F00041FE2B466868029908600194304619469F
:10750000FCF739FE019A104603B0F0BD0298046002
:107510000022104603B0F0BDF0B581B00446002053
:10752000C343022C02D9184601B0F0BD15460E46E1
:107530001B4A62431B498F187968012910D1002D1D
:1075400028D01C460090B83738463146FCF74EFA32
:10755000002821D1761C6D1EF6D1009801B0F0BD37
:107560000090743738462946FCF74AFE00280CD0B4
:107570000446006831462A46F8F7FCFD38462146A5
:10758000FCF70EFE009801B0F0BD07A02146FCF705
:10759000EBFA009801B0F0BD204601B0F0BDC04646
:1075A0005405000094AE0102536F636B65745B2554
:1075B000755D205265637620427566666572204669
:1075C000756C6C0D0A000000F0B583B015460746D7
:1075D0000022D043022F19D8002D17D000AB07C3CB
:1075E0000F4878430F490E18443630462946FCF7B9
:1075F00007FE00280CD00446006801992A46F8F7D7
:10760000B9FD30462146FCF7CBFD029803B0F0BD32
:1076100005A03946FCF7A8FA009803B0F0BDC046B3
:107620005405000094AE0102736F636B65745B25B3
:10763000645D2073656E64206275662066756C6C8F
:107640000D0A000002460020022A04DC0B4B5343C3
:107650000B4AD1507047C0437047C04654050000E4
:1076600094AE0102022801D900207047034941432A
:1076700003484018034940587047C046540500006D
:1076800094AE0102CC04000080B504480168491C96
:1076900001600069002800D0804780BD14E001022D
:1076A0000148024901607047709001020026B8034A
:1076B00010B5C5480024446110300221024A234617
:1076C000FFF7ACFD204610BD7D77000070B584B09B
:1076D000FDF732F9012814D1FCF774FB204D6969DC
:1076E000022914D0002909D12978002921D0A969BB
:1076F000411A062902D300212970A861002004B094
:1077000070BD174800214161002004B070BDE969D7
:10771000421A1449144B9B8B9A4202D20A78002ACF
:10772000ECD0E8610020087000F006F9002004B0F9
:1077300070BD01266E61AB88E88829896A8900AC32
:1077400007C4B102094C0AA22046FCF7A7FC28692D
:10775000AA892146FFF73EFD2E70002004B070BDBF
:10776000A0960102449301026AA9010280C50102A8
:1077700025752E25752E25752E257500F0B58DB035
:10778000032909D87944097949008F4401070F1565
:107790005948416901290AD00DB0F0BD56484169E8
:1077A0000129F9D1022141610DB0F0BD52480021FB
:1077B000416101700DB0F0BD002500954E4C20696F
:1077C0004E494F4A6B46FFF75FFE0028E4D1032085
:1077D0004CA2014608F094FB48484DA10A22F8F754
:1077E000FEFC002812D045484CA10F22F8F7F7FC08
:1077F0000028D1D141482C2101AA0C23FCF75FFCC1
:107800000298FCF735FB60870DB0F0BD3B482C219A
:1078100001AA0C23FCF753FC0498FCF729FB6087B2
:1078200080B2684EB1888142B6D10298FCF769FCFB
:10783000E062039801794279120251188279C37982
:107840001B029A18120451188278C378077840787E
:107850000002C0191B029A181204101820626162FB
:107860000598FCF705FBA0870698FCF74AFCE08723
:107870000798FCF746FC4027E0530898FCF741FCCA
:1078800042216054E16A491E062901D80122A270F2
:10789000062926D87944097949008F440318111C18
:1078A000221E1500E08FB082E05BF082A08FB18DC8
:1078B000814216D01E4902220A60B0851D4800E0B0
:1078C0001A48012101700CE00120B08709E0184836
:1078D0000560B58505E0B58703E0C0B23C214143B2
:1078E000B1830120A07000F027F807F073F925623A
:1078F0006562A5700DB0F0BDA096010280C50102C1
:10790000FF030000CAD5B5BDCAFDBEDD0D0A0000EB
:1079100024696E7374727563742C0000246D657332
:10792000736167655F7265706C792C00E496010283
:10793000D498010238900102F0B5C7B0214CA0885C
:107940001490214D68781390FBF7E2FE1290A08D01
:107950001190687810901D4800780F90A08A0E90C2
:10796000E08A0D901A48C0C81A490A684968AB787D
:10797000194C24682035089209910A950B930C94B0
:107980001298009011980190109802900F9803900F
:107990000E9804900D9805A9C1C11398002801D034
:1079A0000F4A00E00D4A15ADC8212846149B09F086
:1079B0009DFD0246044800692946FFF705FE47B0D1
:1079C000F0BDC0466AA90102A0960102C09801025A
:1079D00048990102409901028C9901022532010067
:1079E000E431010080B582B00E4908680022C2600F
:1079F0000192CA68002A02D0016801A8904702B02B
:107A000080BDC04680B582B0064908690022C260C8
:107A100001220192CA69002A02D0016801A8904798
:107A200002B080BD1C930102F0B582B0144C2078E6
:107A3000009000281DD0134B24330025019504E04D
:107A40009B1C6D1C0098854215D262196026905DC2
:107A5000471C97550928F3D80199C8B222181C88E9
:107A600097554000074A10188484054C491C019121
:107A7000E6E7002001900198207002B0F0BDC046FA
:107A800068990102449A0102F0B589B009F052FCEC
:107A9000E94C607809F0F4F9E8498A8807A88280FF
:107AA0000A88498809048918079105F08DF96078DA
:107AB000052804D00222E249092804D104E0012269
:107AC000DF49092800D0891849792078621C09F01B
:107AD0009BFA607A06F0A0FCDA48DB4904F078FCF7
:107AE000DA4C20780026002806960AD0D8491A31A8
:107AF000D84A034610CA0C80891C5B1EFAD1460086
:107B0000D24CD54DA872D54800886871D4490978FF
:107B100029706178E970000AA871481C60702846D5
:107B20000B30CB4F39464C3103913246F8F722FBEC
:107B300070190B3039461A313246F8F71BFB2020FA
:107B4000687206982071E0886870000AA870C320E7
:107B50000690840106F0D0F90319BC48C362BB4803
:107B6000007881000D3101222846059209F060FC61
:107B7000B6498862B548C46A06F054F90019B34C96
:107B800006F0ACFD05460E46AB48007B06F032FC25
:107B900081B2C90B401800B2C11740102818A06567
:107BA0007141E16506F0A8F9A06104F083FB0028AB
:107BB000FBD106F0A1F9E0617D20060100273846DF
:107BC0003946324609F0E8FBA062677125460698FF
:107BD000040206F091F9297861434118A248081877
:107BE000421C01D19F480818984C206306F084F984
:107BF0006063216B884204D39C4A8918884200D86C
:107C000097E006F079F9606306F076F9E06104F038
:107C100051FB0028FBD106F06FF920626079022841
:107C20004FD001287DD100206071914D697A2129C2
:107C300071D16979AA7912025118884A1288914241
:107C400069D1874909782A788A4264D16978AA7803
:107C500012025118A181E278002A40D02278002A2D
:107C60000BD07B4B4C3300201C888C4204D09B1CD7
:107C7000401C8242F8D11046744CC0B2E081236EA1
:107C8000A16BA26D7A4D2C46223400946F4C019169
:107C9000029229461A311E352A46FFF721FAE08959
:107CA000E178884208D34100694A5118A2894C23DF
:107CB000CA522178491C21700521654A11546C482B
:107CC00024E0002060710146324609F065FBA062A5
:107CD00006F012F9206206F00FF9A06121E04C20B5
:107CE0005B4A11520598207005201070236EA06B1E
:107CF000A16D2A46223200920190029129461A3142
:107D00002A461E320020FFF7EBF928469621F8F7A5
:107D10004AFA0020208200200146324609F03CFB4E
:107D2000A062226B606B51495118904200D365E705
:107D300067E7A06DE16DFBF7DBFAA77020780028FC
:107D40002FD044484C213D463C46414B05E0891C20
:107D5000001DFAB26D1C95421AD25E5D002EF6D05F
:107D6000761E5E55A3000693F6B22246414CE650BD
:107D7000374B5E5A5300404CE6527F1C334B9F708A
:107D800003683E4C069EA3511446314B541CDEE75B
:107D900005922E48C77007700497F8B2022806D2E1
:107DA00028E0E77805970497F8B2022822D30598CF
:107DB000441E0021069403E0491C069CA14219D0F0
:107DC0002E4A10682C4B2B4F0FE0156050605D88D9
:107DD0001E885E801D8060CF083F3E607D60641E0F
:107DE000121D9B1C3F1D002CE6D05568A842ECDC00
:107DF0002846F4E704980006059C10D062001E494E
:107E00000398F8F7B7F9A20012481C49F8F7B2F93D
:107E10000F4A184802C81170521C641EFAD10B4850
:107E200083890C4800680090032015A2014608F0E1
:107E300067F809B0F0BDC046C4900102B41F01004C
:107E4000FCA001023901010051EB0000E89601029B
:107E50003898010258D2010206EA0102E0980102B4
:107E6000BC98010201CF030000CF03000026B80335
:107E7000A8D301020CE90102D4E9010270E9010270
:107E8000BBF9D5BE4944A3BA25582CBEE0C0EB3A95
:107E90002025640D0A00000080B5002008F0AAFA31
:107EA00080BD80B5012008F0A5FA80BDF0B581B095
:107EB00003F040FD164CE060A178002901D001B02C
:107EC000F0BD21790029FAD10121217100281BD0B0
:107ED0008D02281AA168814216D0614E2F46A068F3
:107EE000305C21698847A068401CA060681EA168BA
:107EF000814201DD0020A060E168A068022F03D369
:107F0000691A7F1E8842EAD10020207101B0F0BDBD
:107F1000F0950102B0B5294C2368002B07D0022B45
:107F20000DD0012B39D109F0D1F900F00FFC09F087
:107F3000ABF92368022B1FD0012B18D02DE0204D68
:107F4000287800282FD003201EA2014607F0D8FF72
:107F50000020287009F0BAF900F06EFD1C4D287061
:107F600009F092F928780028E3D001202060194810
:107F700000214181012310E011480178002909D135
:107F800014494A89531C4B81152A03D301220270DC
:107F90000020488108F040FF2368032014A2014616
:107FA00007F0AEFFB0BD0B48408914210B1A032027
:107FB00009A2014607F0A4FFBBE7C046D49801021E
:107FC00038900102BFAAC6F4CBD1CBF70D0A00004E
:107FD000BD98010268990102B5C8B4FDBDF8C8EBAF
:107FE000CBD1CBF7C4A3CABDA3BA25640D0A000048
:107FF000555742D7B4CCACA3BA25640D0A00000093
:1080000080B505480068022805D809F05FF9FFF738
:108010003BFD09F039F980BDD498010270B50E25F9
:1080200000242846214603F081FD0D20214603F05F
:108030007DFD0124204608F0E5F804262846314657
:1080400003F074FD0920314603F070FD204601F075
:1080500047FBA2020249034B204608F0D1FB70BD4A
:1080600018CE0102390A010080B5032810D8002972
:108070000ED07C224243BF488018C268012A07D133
:108080002030FBF7DAFC002801D00020C04380BD7F
:108090000020C04380BDC046F0B589B00022D54362
:1080A000032800D9ABE00C46002900D1A7E00095D9
:1080B000216A0727534DA9420EDC574DA9421ADD0C
:1080C000564A91422FDC4B22D501A9423ED01202E2
:1080D00091424BD1042246E04B4A914217DD4B4A74
:1080E00091422ADCE1221203914231D0494A914265
:1080F0003CD10C2237E04B252E01B14233D06A012E
:10810000914227D0AA01914230D102222BE0E122F4
:108110005502A94220D09502A9421FD0D202914215
:1081200024D109221FE04B225202914218D0E122B1
:10813000120291421AD1062215E0E1225203914225
:1081400010D0334A914211D10D220CE003220AE0F3
:108150000A2208E0012206E0072204E0082202E0E9
:10816000052200E00B22D1002D4A57587C214143C3
:10817000804A505056182068B0606068F060A1686E
:108180003161E2687261002505950323049303952C
:10819000029501970695079501231B020893012874
:1081A00007D000280AD18818009A8018B161F061C0
:1081B00004E0304620300123FBF737FC2069706370
:1081C0006069B063E069B067A069F063706801A995
:1081D00008F042FA2068012806D83046403023468D
:1081E00010330ECBFCF736F86068012807D1301D3C
:1081F0007036006801220B4B314608F001FB28461F
:1082000009B0F0BDFFC10100FF0F0E00FF1F1C00F1
:1082100080841E0040420F007F250000FF95000073
:10822000E41F0100510A0100B0B50C467C2148430F
:10823000504A15182846FBF717FE6C600020B0BDA9
:10824000F0B583B00024E743032800D98EE00E4642
:10825000002900D18AE01546002A00D186E07C2161
:108260004143444841188868022832D001283AD056
:1082700000282BD1EFF31080C00702D1EFF310805C
:1082800072B602910846403001902946FBF7B8FFCC
:10829000002863D0014601980F46FBF781FF38683C
:1082A00031462A46F7F766FF0198FBF78EFFEFF39A
:1082B0001081C90703D1EFF3108172B662B602993B
:1082C0004D6806C82C4B284608F0DCFB204603B05E
:1082D000F0BD4868002431462A46234608F0D2FB08
:1082E000204603B0F0BDEFF31080C00702D1EFF3DA
:1082F000108072B602910846403001902946FBF783
:108300007FFF00281ED0014601980F46FBF748FF6B
:10831000386831462A46F7F72DFF0198FBF755FFDD
:10832000EFF31081C90703D1EFF3108172B662B683
:1083300002994D6806C8104B284608F0A3FB20465A
:1083400003B0F0BDEFF31080C0070FD1EFF3108042
:1083500072B662B63C46204603B0F0BDEFF3108023
:10836000C00703D1EFF3108072B662B63C462046D8
:1083700003B0F0BD90BE0102550D0100B0B582B052
:10838000602833D0622843D0642854D101A82F49F3
:108390000180EFF3108072B600242046214602F0DF
:1083A000B3FA2B4D002805D10120020300202946F5
:1083B00002F004FA103501AA02232046294602F0F1
:1083C000DBFE62B623A0FEF76FFE64201B490C5251
:1083D00006F000FC1A4801F00DFCBFF34F8F19485E
:1083E00019490160BFF34F8F00BFFDE760201349BB
:1083F00000220A5206F0EEFB114801F0FBFBBFF32E
:108400004F8F104810490160BFF34F8F00BFFDE749
:1084100062200A4900220A520A8006F0DBFB084863
:1084200001F0E8FBBFF34F8F064807490160BFF337
:108430004F8F00BFFDE702B0B0BDC0466AA9010280
:10844000A08601000CED00E00400FA05AAAA0000D5
:1084500000D00204BDF8C8EBC9FDBCB6C4A3CABDB8
:108460000D0A0000F0B5D1B0A74EA8490A78002A3D
:1084700025D0F28B002A22D1A54FBA68082A00D94C
:1084800090E0930001A4E3589F46C046B1840000E9
:10849000A5850000A5850000B5850000DF850000EA
:1084A000E9850000F3850000C3850000FD8500001C
:1084B000552800D0BBE00120B86051B0F0BD49782C
:1084C000002900D1B7E0924D6A7996498854A9797C
:1084D000A871E971521C6A710A2800D0ABE00D291D
:1084E00000D0A8E003A8019037A800902C463034B3
:1084F0008C488D491DAB2246F7F78EFEE8608BA1B4
:1085000005222046F7F76BFE00282AD1F08B0028C1
:1085100005D0032087A2834B014607F0F1FC1DA87C
:108520000024214609F0ABFCA861E961824B224698
:10853000F8F7BEF9002814D1804800F0F7FF1DA815
:108540000024214609F09BFC2862696237A8214675
:1085500009F095FCA862E96203A8F7F7EFFE28612D
:1085600000E0286900266E71002806D07448067065
:10857000744801210170744806806A489621F7F713
:1085800012FE1DA864242146F7F70DFE37A82146E8
:10859000F7F709FE03A82146F7F705FE6E71EE8096
:1085A00051B0F0BDAA2838D1012A36D10220B860D6
:1085B00051B0F0BD0421B9600021B970787051B09C
:1085C000F0BD3979534A5054481C38717978491FA5
:1085D000C0B281422FD10820B86051B0F0BD052251
:1085E000BA60887051B0F0BD0621B960B87051B062
:1085F000F0BD0721B960387051B0F0BD7A78062A15
:1086000002921AD3531F0025424A2C46565DA419E4
:10861000A4B26D1C9D42F9DB10E0032807D1022AA9
:1086200005D10120F8700320B86051B0F0BD0020E2
:10863000B870B860787051B0F0BD00242018029A6C
:10864000821888781118BD7849193C780919FA7888
:10865000002A00D0C91C2C4EC9B2FF2935D10128EF
:1086600009D0022831D11E2D36D1FFF7D7FC0120C9
:10867000F08351B0F0BD284A9471032010719070BE
:10868000AA2050705520107068085071651DD57073
:10869000400031181646D01D2246F7F76BFD301DFD
:1086A000E11CEAB2D21C037892B2D218401C491ED7
:1086B000F9D1A019D143C171090A0172093401200D
:1086C00000233146224608F0DDF90020B870B8607A
:1086D0003871787051B0F0BD70190E4E3146224697
:1086E000F7F748FD3078012802D12846FFF746FE0B
:1086F00006F070FABFF34F8F084809490160BFF3D5
:108700004F8F00BFFDE7C0466AA901021890010221
:1087100020990102B4CD0102149B01020CED00E08E
:108720000400FA051CCD010281310100474E474784
:1087300041000000257300000000F03FD1AD0102B0
:108740002C940102E7960102D2AD0102F0B589B086
:1087500008F0F0FD9A489B4903F03AFE9A4E002437
:108760003471F47005F0C8FBF061042003F06AF97D
:10877000964D6A6820460694214608F00DFE05F0E5
:10878000BBFB0446306327204101686848430A2147
:10879000F7F7A0FC70630119481C00D00846B063CD
:1087A00005F0AAFBF063B16B894C884202D309192A
:1087B000884233D9874F884D05F09EFBF06303F064
:1087C00079FD00280AD0FCF775F805F095FBF063F9
:1087D000B16B8842F3D909198842F0D2F0780128A8
:1087E0000FD138782978814211D1787A20280ED19A
:1087F0007879B979090208187849898D884206D1B3
:1088000033E0724842680020014608F0C5FDB16BB4
:10881000F06B8842D0D309198842CDD8012528466B
:1088200001F0E8F9284608F0E1FD3079002816D17A
:108830006B4806F04FFA6F4C2378032077A201466D
:1088400007F05EFB2078411C2170062807D3794889
:10885000022101600698207070815C480570042038
:1088600003F0E0F8002009B0F0BD012030715C4851
:10887000623006F02FFA05F03FFBB061B87AB070B5
:10888000024605907879B97909020C18F4803946C6
:108890000B315500534802912A46F7F76BFCE91952
:1088A000059F0B314F4832302A46F7F763FC002F03
:1088B000069872D04948808904904B480368002587
:1088C000484A039326E0B11860230027CF54510093
:1088D000464A51188C8400B2F8F728F83A46444BBF
:1088E000F7F7C0FE08900791706AF8F71FF83A464C
:1088F0003F4BF7F7B7FE02460B4608980799F7F784
:10890000FFFDF8F779F87062059F364A039B6D1CEE
:10891000BD4227D06800115A8B42F8D11118488EF9
:10892000049A80184886317800290ED02F4B2433C2
:1089300000221F88A7420DD09B1C521C9142F8D1E7
:108940000B460A46172908D9BDE700231A461729FE
:1089500003D9B8E7D3B21729B5D88B42B3D1491C94
:108960003170B0E7002F0FD01F4801680020029C33
:10897000227863781B029A18914207D0A41C401CED
:108980008742F5D1384608E0002006E0C4B2204610
:10899000FAF72CFCB078A04201D1FAF727FC154871
:1089A00000210170052030560C498B8D716A0091B1
:1089B0000190032010A2014607F0A2FA2EE7C0465C
:1089C00011010100A9EA0000689901023890010232
:1089D000007C312510D30102BC9801026AA9010272
:1089E0001A3F00009C9A0102E0980102449A010299
:1089F0000000E03F0ED30102B1EAC7A94944A3BA7F
:108A000025582CBEE0C0EB3A20256420D0C5BAC55D
:108A1000C7BFB6C8A3BA25642E0D0A00B2E2BEE0F5
:108A2000CAA7B0DCA3ACBCC6CAFDA3BA25640D0AB4
:108A300000000000D4980102F0B587B008F07AFC7D
:108A4000904C607808F01CFA8F498A8805A88280CB
:108A50000A88498809048918059104F0B5F96078F5
:108A6000052804D002228949092804D104E0012202
:108A70008649092800D0891849792078621C08F0B5
:108A8000C3FA607A05F0C8FC8148824903F0A0FC73
:108A9000814C0026E67005F02FFAE061042002F018
:108AA000D1FF7E4D3046049631462A4608F074FCCC
:108AB00005F022FA7A49206361634118481C00D00E
:108AC0000846A06305F018FAE063A16B754E884272
:108AD00002D38919884234D9734F03F0EBFB002885
:108AE0000AD0FBF7E7FE05F007FAE063A16B8842C6
:108AF000F3D989198842F0D205F0FEF9A061E07837
:108B000001280FD138786949097881420AD1787AE9
:108B1000202807D17879B979090208186449898D24
:108B200088421CD005F0E8F9E061002001462A46A1
:108B300008F032FCA16BE06B8842CED389198842E1
:108B4000CBD80125284601F055F8284608F04EFC00
:108B5000049C042002F066FF204607B0F0BD554893
:108B600006F0B8F805F0C8F9A061B87AA07002461E
:108B700002907879B97909020D18E58039460B31F0
:108B800056004D4800913246F7F7F4FAF119029F6A
:108B90000B31494832303246F7F7ECFA002F62D0F9
:108BA000464803680026444A019326E0A118602342
:108BB0000027CF545100424A51188D8400B2F7F774
:108BC000B5FE3A463F4BF7F74DFD04900391606ABE
:108BD000F7F7ACFE3A463B4BF7F744FD02460B462F
:108BE00004980399F7F78CFCF7F706FF6062029F81
:108BF000314A019B761CBE4224D07000115A8B4230
:108C0000F8D11018408E217800290ED02C4B243337
:108C100000221F88AF420DD09B1C521C9142F8D1FC
:108C20000B460A46172908D9C0E700231A46172918
:108C300003D9BBE7D3B21729B8D88B42B6D1491CA8
:108C40002170B3E7002F0ED01C4801680020009D62
:108C50002A786B781B029A1891420AD0AD1C401CEE
:108C60008742F5D100E000273846FAF7BFFA012421
:108C70006FE7C5B22846FAF7B9FAA778AF42F3D042
:108C8000012466E7B6900102BA1F0100FCA00102B0
:108C900011010100A9EA00006899010280841E0008
:108CA0000098E00E007C312510D30102BC9801022F
:108CB0006AA901025C3F00009C9A0102E09801024F
:108CC000449A01020000E03F80B582B0002001908C
:108CD0000448C268002A02D001A80021904702B0CF
:108CE00080BDC0468C950102F0B583B000242046BB
:108CF000FDF7DEFFFEF701F8274EB060FDF7FAFF43
:108D00007060264F0BE001A8C1888088084319D104
:108D100001A8408824180834B068844235D201ADD7
:108D2000082128462246FDF7CFFF28880028EAD0F0
:108D3000B8422AD001AD0421284600F045FFA98899
:108D40008842E5D03460B06884420CD201AD022183
:108D500028462246FDF7B8FF2888B84203D0A41C55
:108D6000B0688442F2D370682118491E404208401E
:108D700030600DD00024254601202946FDF77CFFF8
:108D800003CE4D19083E8542F6D3346003B0F0BDE2
:108D90000024346003B0F0BD50970102FFFF0000D3
:108DA00010B5054C6070FEF7C7FD6078022801D150
:108DB0000020607010BDC046A0960102F0B585B0DD
:108DC0001F4604920646C8170C1844400A2C03910B
:108DD00014D301250A212046F7F77CF96D1C632C7A
:108DE0000446F7D804998D4200D329460A9C002FE7
:108DF00009D00398002808D4002207E0012504992F
:108E00008D42F2D2F2E7002205E001220423234042
:108E10009B081343FA1A0223234004980028029463
:108E200012D1002B10D0F468002C62D403980028D3
:108E300025D40298400734D57068B5686F1C874206
:108E40002FD830682B2423E0E407ECD1002A0AD184
:108E5000E9E7376820203855B560F068441CF460B5
:108E6000521E002CDFD49142DDD27768B468651CB5
:108E7000BD42EED9F468521E002CF4D5D3E740422F
:108E800003907068B5686F1C87420AD830682D243B
:108E90004455B760F068441CF4600025ED43A842D7
:108EA00027DB002B1CD00120029B1840049B184399
:108EB00016D1002A03D113E0521E002C0ED4914289
:108EC0000CD27068B3685D1C8542F5D830683024D8
:108ED000C454B560F068441CF460EDE7002C08D47D
:108EE0000092029801900A2230460399049B00F0F8
:108EF00003F805B0F0BD0000F0B587B01F46154679
:108F00000290012406919142009407D3012406980F
:108F10002946F7F7DFF8641CA842F9D20D980C9A9D
:108F2000BC42039700D3039400990140002A0091AA
:108F300009D00029029C25D12021800705D40846AC
:108F4000002F11D004E0029C1CE03020002F0BD039
:108F5000084609E023685854A260E168491CE160B2
:108F60003246721E00290DD4039991420AD2164648
:108F70006368A1684A1C9A42ECD9E1683246721EC5
:108F80000029F1D5E068002859D40590012401E0BA
:108F90007F1E6C43022FFBD2069821461646F7F738
:108FA00099F83246A842F4D2029880680490069F4D
:108FB0000195069738462146F7F78CF8049D691C01
:108FC000029F7A68914206D9069F059A019D0592F3
:108FD000002A0ED516E01B4A125C3B685A55B96050
:108FE000FA68521CFA600491069F019D0592002ABE
:108FF00008D460433F1A20462946F7F76BF8AC4285
:109000000446D6D200980028029C059B049D16D0E9
:10901000002E14D0701C01E0002B10D4401E0399C8
:1090200081420CD2691C62689142F5D822682023E3
:109030005355A160E268531CE3600D46ECE707B0AE
:10904000F0BDC046C0220100F0B583B0019002918E
:10905000002923D00025124F2E460AE01348081895
:10906000410F4018C0103872761CB0B20299884285
:1090700014D2019800884B24210100B200F018F8A6
:10908000400061014018F88201B20648814228463A
:10909000E9DB05488142E1DD6420E4E703B0F0BD8F
:1090A000B8980102E40C0000041000001CF3FFFF5C
:1090B000074A904201DD054A801800B24143C817B3
:1090C000400D0818C00A00B27047C04600F0FFFF0C
:1090D000FF07000010B50078012819D1AC480269DB
:1090E000012A04D1614A13680124A34313600329B0
:1090F00005D080214161C269002A05D107E0012124
:109100004161C269002A02D001898069904710BD7F
:10911000FF222E32024803A107A305F095FEC046A8
:10912000742E01006164635F646D615F63616C6CE8
:109130006261636B00000000556E65787065637452
:10914000656420646D61206368616E6E656C0D0AF4
:1091500000000000F0B58DB00D460124EFF3108142
:10916000214002D1EFF3108372B6894E73690F2B41
:1091700006DD102B37D0402B2FD0802B2DD005E0D3
:10918000002B2AD0012B01D110237361B5813581C9
:10919000B061F261002900D162B63179002929D08D
:1091A0000294304C05A90A4604950390E8CCE8C225
:1091B000E8CCE8C2029C204600F08CFD2A480090D2
:1091C0002A4D294608312046039A049B00F0F2FDFF
:1091D0002C60002420460DB0F0BD0029FAD162B603
:1091E00020460DB0F0BD02240029F3D162B620461E
:1091F0000DB0F0BD3178002907D01C4807218161EE
:109200000460002420460DB0F0BD3269B3891749CF
:10921000002B15D0B5693089012A02D0002A03D06D
:1092200003E09FB2874200D10C604F68FF07FCD07B
:109230008F6880C55B1E1F04EED10023B381B5612A
:10924000012A02D10A68A2430A607461F26900240B
:10925000002ABFD0B36931898800181A9047204688
:109260000DB0F0BD00230100D590000008D00140F2
:10927000F0B581B0002856D00446424EF068800711
:1092800054D41325284600F0DDFB284605F0B0FA3B
:1092900027686168012538462840CA07920F1018D0
:1092A000227C1207120E8018627C1207120D8018A1
:1092B000A27C1207120C8018627D13071B0AC018CB
:1092C00012091206801830607D20060200293046FF
:1092D00000D12D48E3681A0A7D2A1A4629D22B4E5E
:1092E000B3422AD200292BD0002A2946254E00D08D
:1092F0001146F6F7EFFE401E80B270602448076109
:10930000E27C0270237D0371224F3E686902A468EB
:10931000012C1BD02C0226433E60002B1ED00121C5
:10932000184A116329E0012001B0F0BD022001B00C
:10933000F0BD3246154EB342D4D333460029D3D1C3
:109340001A46002A29460F4ED2D1D2E73F242401E3
:10935000A6437618F0363E60002BE0D1002A0CD0F0
:10936000FF2212020C4B1C6894430122D203A21864
:109370001A60304A1160304A1160012141610020B9
:1093800001B0F0BD00D001400026B80380841E006B
:10939000A09501022C06004008E400E070B500280A
:1093A00001D0012070BD0C461625284600F04AFB6E
:1093B000284605F01DFA002C05D01B481830142251
:1093C0002146F6F7D7FE28211748415C002915D021
:1093D0004168002916D403220B469343144A9C5833
:1093E0008D07ED0EFF26AE40B4439C501F220A406D
:1093F000012191400F4A11600F4A11600121016162
:10940000002070BD8A07D20EFF2393400F220A402E
:10941000083A03218A43054954589C43545001217A
:109420000161002070BDC046749001021CED00E097
:1094300000E400E080E200E000E100E080B5684880
:109440000021017061480078C001614909788901F3
:10945000014360480078400108435F4909780901E9
:1094600001435E480078C00008435E49097849001E
:1094700001435D4800780843C0B2FBF757F980BD4F
:1094800080B55748012101705148007880014F494B
:109490000978C90101434F480078400108434E490B
:1094A0000978090101434D480078C00008434D493F
:1094B0000978490001434C480078084304210143DE
:1094C000C8B2FBF733F980BD5A21014A50527047A8
:1094D00094A00102F0B581B013490A78002A13D094
:1094E000052A01D104220A709300CD18561C0023CE
:1094F0001C462F686F60F917DB194C412D1F761E33
:10950000012EF6DC084902E00022134614464860AA
:10951000521C0A70C11718186141D2B20023F6F725
:1095200003FE01B0F0BDC046C0950102F0B581B0A8
:109530000446007841424141217024480078C0012E
:1095400023490978890101432248007840010843F2
:10955000214909780901014320480078C0000843E7
:109560001F4F3978890001431E4D28784000084379
:109570001D4E31780143C8B2FBF7D8F87D20C000FA
:1095800000F038FB20784142414121700F480078BB
:10959000C0010F490978890101430E480078400154
:1095A00008430D490978090101430C480078C000BF
:1095B000084339788900014328784000084331780E
:1095C0000143C8B2FBF7B2F801B0F0BD189F010229
:1095D000E69601021D9001029CEA0102D1AD010252
:1095E000199F01025CA301025DA30102B0B5094D00
:1095F00028600224002120460A4602F02BFA0121AD
:109600000522204602F0BAFA2A680321204602F019
:1096100099F9B0BD149F01025C219D48002242527D
:1096200082847A2141840284C2830283C2820282BC
:10963000114941608260C2603D21490441834182F9
:10964000090C8183818270475C219148002242523B
:1096500082847A2141840284C2830283C28202828C
:10966000054941608260C2603D21490441834182D5
:10967000090C8183818270474C37373770B5854834
:109680004C21016001252C02601C00F05BF93220A6
:1096900000F0B0FA00F044F9284600F04BF92846F3
:1096A00000F05AF800F036F90C4800F04BF90026AB
:1096B0003046314600F056FA2846314600F052FA5C
:1096C000204600F03FF9022000F03CF948342046E3
:1096D00005F032FB05F090FB70BDC04601020000B2
:1096E00010B50446072106F069FA0148046010BD70
:1096F0009496010270B505200424214602F016FA62
:109700000620214602F012FA0A20214602F00EFA43
:109710000920214602F00AFA00240121204602F025
:1097200005FA022520462946224602F027FA0B2692
:1097300030462146224602F08DF93046294622461F
:1097400002F01CFA70BD000002480168012291433A
:10975000016070475800004002490A680240824296
:10976000FBD1704704600040B0B5494D28688107BF
:10977000484C0ED528797F21084022688A4310186A
:10978000206023680B4002200321434A06F0B8FB07
:10979000286880040ED55E20285C7F21084062681E
:1097A0008A431018606063680B40022003213B4A23
:1097B00006F0A6FB172000F045F93948016802229F
:1097C0000A4301218A43026036483749016037481D
:1097D0000021C17181791F2529408171817A427CE4
:1097E000837C1B029A18C37C1B04D218037D1B06C2
:1097F000D2182F4B9A4218D1427B837B1B029A18B6
:10980000C37B1B04D218037C1B06D218294B9A4237
:109810000BD1C27A037B491E122906D81902891876
:10982000254A914201D1202101720178CA0602D154
:109830001022114301701C3C2068202188432060C5
:109840001E481F49016041680029FCD503F020FA39
:109850000446022003211BA2234606F051FB0A20E6
:10986000C441032C05D8022003211DA206F048FBA9
:10987000FEE71848C1680F229143C1600168164A8B
:109880000A40026019200001144948600D60B0BD13
:10989000FCA0010248000040BC2E0100A62E0100E1
:1098A000040200400C060040AF6B100A6B00014040
:1098B0004D383650312E32360734000000600040FB
:1098C000FE1C0080436869702049443A20253038E6
:1098D000780D0A00C8600040FEFFC3FF0C04004082
:1098E0004F6C642063686970206D6F64656C2069DB
:1098F00073206E6F7420737570706F72746564205E
:10990000627920746869732053444B2121210D0A28
:109910000000000080B5172000F08CF8002080BD0A
:1099200010B51724204600F08DF8204604F060FFA3
:10993000002010BD0121C9070143014801607047A3
:109940000060004010B5C1B2000AC2B202290CD0BA
:10995000012913D0002930D1911E7F4802291BD242
:109960000121032A2AD0490429E07B484168002AC2
:109970001FD00246203A1143416010BD764801686D
:10998000D31E022B10D3012A29D0002A41D1012253
:1099900092079143016010BD002A16D101214907A9
:1099A00002688A43026010BD0123042A1FD05A04B2
:1099B0001EE0012292079143416010BD0904194A3B
:1099C0007F32C36A13405918C16217498A699207E6
:1099D000FCD50121490702680A43026010BD052237
:1099E000120791430246203A0A43026010BD1A044E
:1099F000836A0C4C1C40A21882620B4A131F00247D
:109A00001C600A4B0A4C1C600D235B0214681C434B
:109A10001460054A93695B06FCD5052212071143C1
:109A2000016010BD80FFFCFF1402004004010040F3
:109A3000FF0F000001218140474802688A4302600D
:109A40007047C04601218140434802680A430260D2
:109A50007047C04610B5052811D8C0467844007933
:109A600040008744020E192434393B490A680868CB
:109A7000C0003CD53A4820390A425DD03BE0002086
:109A800010BD35490A680868C00035D534480B4612
:109A9000203B1A4237D134E02F490A680868C000D9
:109AA00036D52F480B46203B1A424CD135E02A4987
:109AB0004C680120C0030A680B46203B1C421AD0A8
:109AC0000C68E4003BD5264C1A423CD03AE02248D0
:109AD00000680120C00310BD1F490A680868C00063
:109AE0001ED51F480B46203B1A4220D11DE01B48C3
:109AF00020390A4220D010BD18480B46203B1A429C
:109B000001D10120C00349688900890FC84010BDF8
:109B100012480B46203B1A4215D10120C00312E027
:109B20000E480B46203B1A4201D10120C003496870
:109B30000903890FC84010BD0120C00310BD074CA8
:109B40001A4200D020464A689200920FD0404968DD
:109B50000901890FC84010BD20000040006CDC02E4
:109B60000026B80304282CD8164AC0467844007949
:109B700040008744020A121A2100032000071368DC
:109B800083438807800818181AE0032080061368AA
:109B9000834388070009181812E003208004136823
:109BA00083438807000B18180AE0FF20000213689F
:109BB00083430802181803E01068FF2398434018F5
:109BC0001060704724000040B0B5002200290CD07E
:109BD000074B047895B22D0A65406C001C5B12029D
:109BE0006240491E401C0029F3D190B2B0BDC0466E
:109BF000C020010000280AD030B407252C02CD2552
:109C00006419604340091238001FFDD830BC70470A
:109C1000F0B583B01F4616460D460146E86802912E
:109C2000F6F7F2FB04460F2E11D8082E04D3204677
:109C30002146F6F790FB09E0042E02D38120C105EE
:109C400001E0412001062046F6F7DEFB04460999B3
:109C5000089E2B20C043874205DB20460F46214645
:109C6000F6F779FB0DE03F20C04387420BDA49202D
:109C7000C04387420CDBFF200F4681052046F6F7E4
:109C8000C3FB39460446688A0880346003B0F0BDDF
:109C900001915320C043874206DB20462146F6F758
:109CA0005AFB0446688A10E0A8690299F6F7D6FDC7
:109CB000002801D1A88B00E0E88BF6F730FE0146C2
:109CC0002046F6F7A1FB0446002001990880346085
:109CD00003B0F0BDF0B581B005460120072D66D870
:109CE0000C46002963D04A4F38680169C90736D14C
:109CF00005263046FFF7A6FE304604F079FD03CF77
:109D00000369012213430361002918D403200B4681
:109D100083438E481E588807C00EFF278740BE43E6
:109D200040278740374389481F501F200840824002
:109D30008748026087480260354800680FE08A075C
:109D4000D20EFF2696400F230B40083B03218B4386
:109D50007D495F58B743402696403E435E506901B7
:109D60004018012109024218E369DB069B0CA56932
:109D7000ED00EDB2EB18536062685207520B236896
:109D80005B075B099A18A3685B079B0CD218E36812
:109D90005B075B0DD21823695B01DBB2D2186369E4
:109DA0009B07DB0ED218802313434350002001B0E1
:109DB000F0BDC046F0B581B0002A23D00546083575
:109DC000134C2668F668EE40F50702D0022001B079
:109DD000F0BD069D8600A619B560400124682018D4
:109DE000009301231D02461977680724A743776073
:109DF000F16032610099B16041591943415100202D
:109E000001B0F0BD03A00AA174220DA305F01CF857
:109E1000D4920102696E636C7564652F6472697611
:109E20006572732F6D6B5F646D612E6300000000BF
:109E3000646D615F7472616E73666572000000002C
:109E4000496E76616C6964207472616E73666572C6
:109E5000206473742061646472000000000158493A
:109E6000085840687047C046F0B581B005460120EB
:109E7000012D4CD80C46002949D0002D03D0012DCE
:109E800004D10F2000E00E20FFF7DCFDA668012EB4
:109E900004D0002E4FD1E08900284CD12901294857
:109EA00043580020D860F507AD0F27686668B607ED
:109EB000360F76192569EA07920EB618022F04D0DC
:109EC000012F03D10122164300E040361D4F9E6052
:109ED000E2681A6079188D606269CA604968002971
:109EE00017D403220B469343184A9C588D07ED0E56
:109EF000FF26AE40B4438026AE4026439E501F222C
:109F00000A4001219140124A1160124A116001B0C9
:109F1000F0BD8A07D20EFF2494400F230B40083B6C
:109F200003218B4308495D58A543802494402C436A
:109F30005C5001B0F0BD08A00FA1492212A304F0AB
:109F400083FFC0461C9301021CED00E000E400E02A
:109F500080E200E000E100E0696E636C7564652FEB
:109F6000647269766572732F6D6B5F6475616C5F87
:109F700074696D65722E63006475616C5F74696DE0
:109F800065725F6F70656E00636F6E6669672069EA
:109F90007320696E76616C69640000000001084AF4
:109FA00010580160816880220A4382607047C04671
:109FB00000010349085881688022914381607047FD
:109FC0001C930102F0B58DB0019315460E460A9020
:109FD0001298002408900480149F3C8013980990E4
:109FE0000460159804900480FF2081053046F6F740
:109FF0000BFA0290304603963146F6F7ACF92B4641
:10A000003D460690274607950B9311E0118018886E
:10A0100080002858099908600120079D28800520A4
:10A02000049908807F1CBCB21888844200D9A0E043
:10A0300028880028F6D1A0000A9D2E58304606999F
:10A04000F6F7FEFB002817D030460399F6F7F8FB29
:10A0500000280B9B079DE5D1089A1780099D2E606B
:10A060001888011B012934D11080198889000A9AA7
:10A0700051582960059035E0089A178009980660C4
:10A080000B9B1988081B0128C0D00C960198251835
:10A090007E1CB0B28542BFD389B2B2B28A420ED81A
:10A0A00080000A990C5820460C99F6F7BBFB0B9BD5
:10A0B000002804D109980460089806800C94761C46
:10A0C000B0B28542A8D3198889B2B2B28A42E7D920
:10A0D000F5E70C96019962187D1CA9B216468A42D2
:10A0E00005972CD2059884B2A5000A9E7259002CBF
:10A0F000104609D0A819001F016810460C92F6F707
:10A100002AF90C9A062C07D80446A819416810466B
:10A11000F6F721F90C902046079D0299F6F79EFB71
:10A1200000280B9B07D10C980299F6F789FB0B9B33
:10A13000002800D076E701202880032070E780B255
:10A14000AAB282420FD888000A990C5820460C996E
:10A15000F6F768FB0B9B002805D109980460089866
:10A16000058005950C946D1CA9B28E42BAD318884F
:10A17000E5E70DB0F0BD00000A490A680A48024050
:10A180000A60FD214900094A1268515C002908D083
:10A1900007490A6C02400A64012000060A688243EB
:10A1A0000A60704700040040FFFFFF7F44940102F3
:10A1B0002000004000207047F0B583B00D460446F3
:10A1C0007C26464350488719F869396AF5F782FFBB
:10A1D000A84200D892E0019502940121EFF310808B
:10A1E000084002D1EFF3108272B63C4610343B694E
:10A1F0000025062B0CD80A469A40D3065B0F06D1E1
:10A2000061231A4275D00D46002803D003E00225D1
:10A21000002800D162B6002D02D0284603B0F0BD60
:10A2200000943C462034384880591021C1613E4694
:10A23000143604F0DBFD05463868C069C00605D554
:10A2400004F0D4FD401B31888842F5D90621029DD7
:10A25000284600F00BFF206801994143B8690918AE
:10A2600038688160172179563C461734002909D592
:10A27000C16920220A43C2610121F9668905026889
:10A280000A4302600521284600F0F0FE207840B223
:10A2900000250028C1D42B4800687D24E100F5F793
:10A2A00019FF61014143029800F0B2FE04F09EFDE7
:10A2B00004463868C069C00705D004F097FD001B4C
:10A2C00031888842F5D904F091FD04463868C169A7
:10A2D000890706D504F08AFD001B31888842F5D92C
:10A2E00038680121009A116053498161284603B002
:10A2F000F0BD0321216000288CD08CE7034804A125
:10A30000084A09A304F0A0FD48930102EC2E0100C5
:10A31000666C6173685F626C6F636B5F65726173BB
:10A32000650000005D020000626C6F636B20696471
:10A3300078206973206F7665722072616E67650D93
:10A340000A00000028E00102F0B583B002907C21F1
:10A350004143934A5418E56EEAB2511E02291FD2B6
:10A3600029040126090E18D001960092022100F05E
:10A370007DFE2746143704F039FD06462068C16982
:10A38000890606D404F032FD801B39888842F5D94D
:10A390002068007DC007019E08D0304603B0F0BDA4
:10A3A000032A36D100922804000E36D020466C30A5
:10A3B0002D0C0021019101602746143704F016FD91
:10A3C00006462068C069C00705D004F00FFD801B59
:10A3D00039888842F5D904F009FD06462068C1692C
:10A3E000890706D504F002FD801B39888842F5D91B
:10A3F000206811498161E9B20120002911D00329A7
:10A400000099019E00D006202061226F002A0ED103
:10A41000C3E70026304603B0F0BD0126304603B046
:10A42000F0BD0099019E2061226F002AB5D002A8DC
:10A430009047304603B0F0BD000093EB70B50028A4
:10A4400001D0012070BD7825CD4E705D00280ED062
:10A4500000240921204600F009FE0F20FFF7CAFB67
:10A460001520FFF7E7FA74553461204670BD0420CB
:10A4700070BDC046F0B581B00C460078484EF1681A
:10A4800081422CD1032C54D1706EB16E884261D9B7
:10A4900000240621204600F0E9FD3068F16D81605E
:10A4A0002046214600F0E2FD354660352CCDF068AF
:10A4B0003168B48C414F00975B1BA34200D81C4607
:10A4C000A3081431FFF776FCB06E0019B066306E49
:10A4D00000193066F06D0019F06501B0F0BDB1688B
:10A4E000814255D1032C45D1F08CF16D0918F165ED
:10A4F000316E09183166B16E0818B066716E81420E
:10A5000038D900240621204600F0B0FD3068F16DF6
:10A5100081600121204600F0A9FD316EB068F38C06
:10A520003268264C009414329B08FFF743FC01B0BC
:10A53000F0BD30681021C16104F058FC0546306858
:10A54000C069C00616D504F051FC401BB18A884290
:10A55000F5D90FE030681021C16104F047FC0546D1
:10A560003068C069C00605D504F040FC401BB18AC4
:10A570008842F5D90120C107326813688B43136004
:10A58000F16E22040A4300021043F06601B0F0BDF0
:10A590004D200201034804A1844B04F055FCC04641
:10A5A00048930102EC2E0100666C6173685F646D74
:10A5B000615F63616C6C6261636B000075A4000095
:10A5C000F0B581B000786E4DAA68824200D0D0E02C
:10A5D00001263002032942D16A6DAA66AB6DAC6ACE
:10A5E000A418EB652C66AB6C5B1CAB646B6E934282
:10A5F00035D95E30FFF7FEFA686CA96C02293AD3B0
:10A60000814238D1E88C696D081868650020062100
:10A6100000F02CFD2868E96D81602F6D04F0E6FBE9
:10A6200004462868C069C00705D004F0DFFB001BA2
:10A63000A98A8842F5D904F0D9FB04462A68D06972
:10A64000800706D504F0D2FB001BA98A8842F5D901
:10A650002A687420285C012841D0F10440E0F20708
:10A660002B681C6894431C60EA6E09041143014383
:10A67000E96601B0F0BD0229FBD38142F9D2E88C32
:10A68000696D09186965A96D0818A865002006217B
:10A6900000F0ECFC2868E96D8160EF8C04F0A6FB0B
:10A6A00004462868C069C00705D004F09FFB001B62
:10A6B000A98A8842F5D904F099FB04462A68D06932
:10A6C000800706D504F092FB001BA98A8842F5D9C1
:10A6D0002A687420285C012822D0F10421E0310589
:10A6E000334B3B405918012802D01920400601E0A5
:10A6F0000720C00608182F4940185060002F0DD0C1
:10A7000004F074FB04462A68D069800706D404F07C
:10A710006DFB001BA98A8842F5D92A682B6D1FE0C2
:10A720003105234B3B40C918012802D019204006AF
:10A7300001E00720C00608181E4940185060002F8D
:10A740000DD004F053FB04462A68D069800706D474
:10A7500004F04CFB001BA98A8842F5D92A68EB8CCF
:10A76000296EA868144C00941432FFF723FB01B043
:10A77000F0BD044804A10C4A0C4B04F065FBC04634
:10A7800048930102EC2E0100666C6173685F646D92
:10A79000615F77726974655F6E62797465735F6318
:10A7A000616C6C6261636B0072040000D32E010067
:10A7B000FF3F000000808000C1A50000F0B587B019
:10A7C00004460126880E14D01546002A11D00F46E3
:10A7D0008120C004401B88420BD37C206043F04999
:10A7E00008180590818C38460691F5F773FC00290E
:10A7F00002D0304607B0F0BD28460699F5F76AFC4E
:10A800000029F6D1059880693E1A30460699F5F779
:10A8100061FC0746039670190190069E3146F5F7D4
:10A8200059FC0546C01B04900598006A0290314609
:10A83000F5F750FC049981420FD20026BD42D8D9C9
:10A840002046394600F018FB2046FFF77DFD002822
:10A85000FAD17F1CAF42F3D3CBE700900398029D5F
:10A860002946F5F737FC0646284670430399081A2F
:10A87000019800D0761C2946009D7543F5F72AFC07
:10A880000590029941430198401A03900699F5F703
:10A8900021FC0490AF420BD22046394600F0ECFA7E
:10A8A0002046FFF751FD0028FAD17F1CAF42F3D3B9
:10A8B00005988642069D009F0CD220463146FFF740
:10A8C0007BFC2046FFF740FD0028FAD1761C059856
:10A8D0008642F2D30398A84203D20026304607B03E
:10A8E000F0BD059847430025E919204600F0C4FA59
:10A8F0002046FFF729FD0028FAD16D1C0026049898
:10A900008542F1D375E7C046F0B585B0002803D085
:10A910000124204605B0F0BD7822A14FB85C002884
:10A9200003D00024204605B0F0BD0492002905D0D4
:10A93000384614300CC90CC01CC91CC00020F86675
:10A9400015242046FFF77EF8204603F051FF3868B3
:10A950001021C16104F04AFA04463868C169C90689
:10A9600007D504F043FA001BB98A8842F5D9386844
:10A9700000E0B98ABA7D1207120B5218F97DCB0795
:10A98000DB08D2188B07DB0F5B05D218CB06DB0F79
:10A99000DB05D2184B07DB0FDB06D2188B06DB0F6B
:10A9A0005B07D2180907C90F89071143016000240A
:10A9B0000A21204600F05AFB3220FFF71BF908213C
:10A9C000204600F053FB04F011FA05463868C169CF
:10A9D000890606D404F00AFA401BB98A8842F5D9E0
:10A9E0003868017D0A46C23A5342534174257B556B
:10A9F0000904027D12025118007D0B180220032663
:10AA000068A2314605F07CFA785D0128039619D1D9
:10AA1000F87D029000260621304600F027FB072132
:10AA2000304600F023FB012102988143785D012824
:10AA300047D138688901017506757521795C01294E
:10AA400038D048E00020032100F010FB04F0CEF9DC
:10AA500006463868C169890606D404F0C7F9801B28
:10AA6000B98A8842F5D93868007D46080122F87D08
:10AA7000014631431640C90701D0304036D0029517
:10AA8000002506212846019200F0F0FA07210095E2
:10AA9000284600F0EBFA019846400298385C0128FD
:10AAA00013D13868B1010175009901757521795C80
:10AAB000012910D114307621795C4A424A41510073
:10AAC00008E038680675490003E0386800990175A8
:10AAD000710014300170374800687D21C900F5F716
:10AAE000F9FA28214143002000F092FA7720385CDF
:10AAF000012803D102200021FFF734F804F076F991
:10AB000006463868C069C00705D004F06FF9801B9D
:10AB1000B98A8842F5D904F069F906463868C169EE
:10AB2000890706D504F062F9801BB98A8842F5D9F5
:10AB30003868D049816117203856002829D57868AF
:10AB4000002816D40146039A91431C4A8B58850766
:10AB5000ED0EFF26AE40B3438026AE401E438E501E
:10AB60001F210140012088401549086015490860EF
:10AB70000FE08107C90EFF228A400F230340083BE4
:10AB8000039883430C481D58954380228A402A43EA
:10AB90001A500120049978543861204605B0F0BD60
:10ABA000489301026A656465635F69642025780DD6
:10ABB0000A00000028E001021CED00E000E400E0D3
:10ABC00080E200E000E100E0F0B593B07C270A905D
:10ABD00047439348C619980704D0F07D40240440A9
:10ABE00000D017E10125880E2ED0002B2CD081201B
:10ABF000C004C01A884227D309920122EFF31084BF
:10AC0000144002D1EFF3108072B630461030059038
:10AC10003069002506280891069310D80794144639
:10AC20008440E106490F04D161210C4203D015464E
:10AC300004E0022502E00221059B1960079C002C1C
:10AC400000D162B6002D02D0284613B0F0BD3446C4
:10AC500017347348C05910210491C1613746143725
:10AC600004F0C4F805463068C069C00605D504F094
:10AC7000BDF8401B39888842F5D92078400665D454
:10AC80000297B78C069C20463946F5F723FA0790C1
:10AC900039464143601A039035462435A74200D80F
:10ACA00094E0039800281CD006210A9C204600F05E
:10ACB000DDF9288807994843089940183168886069
:10ACC00000272046039C394600F0D0F9079B099ADB
:10ACD00028885843C0193168097D11547F1CA74248
:10ACE000F6D330680499C16104F080F80446029DEF
:10ACF0003068C069C00605D504F078F8001B2988C3
:10AD00008842F5D904F072F804463068C069C0077B
:10AD100005D004F06BF8001B29888842F5D904F0AF
:10AD200065F804463068C169890706D504F05EF805
:10AD3000001B29888842F5D930680121059A1160E5
:10AD4000B24981610025284613B0F0BD03200025DB
:10AD5000089FF7650999316606997166B566F066D0
:10AD60000120C00731680A6802430A6006210A9C74
:10AD7000204600F07BF9306887602046294600F0C5
:10AD800075F93A4F0BAA0A921BCF1BC21BCF1BC2ED
:10AD9000B48CF0680A99FEF79DFFF0683168344A78
:10ADA0000092069A944200D31446A3081431099ADB
:10ADB000FFF700F8B06E0019B066306E001930660B
:10ADC000F06D0019F065284613B0F0BD002404E0D2
:10ADD000641C0798844200D363E706210A9800F0B8
:10ADE00045F9288860430899401831688860002731
:10ADF0000A98394600F03AF928880028099AE7D0DD
:10AE0000604310183168097DC1557F1C288887422E
:10AE1000F6D3DDE7034804A1064A07A304F014F8BB
:10AE200048930102EC2E0100666C6173685F7265E5
:10AE300061640000C603000054686520444D412051
:10AE400072656164206C656E6774682073686F75E5
:10AE50006C6420626520746865206D756C7469701F
:10AE60006C65206F6620340D0A000000602301002D
:10AE700075A40000000093EBF0B583B00D460446C6
:10AE80007C26464351488719F869B98CF5F722F9B1
:10AE9000A84200D894E0019502940121EFF31080BC
:10AEA000084002D1EFF3108272B63C4610343B6981
:10AEB0000025062B0CD80A469A40D3065B0F06D114
:10AEC00061231A4277D00D46002803D003E0022503
:10AED000002800D162B6002D02D0284603B0F0BD94
:10AEE00000943C462434394880591021C1613E46C3
:10AEF000143603F07BFF05463868C069C00605D5E7
:10AF000003F074FF401B31888842F5D90621029D69
:10AF1000284600F0ABF8208801994143B869091828
:10AF200038688160172179563C461734002909D5C5
:10AF3000C16920220A43C2610121F96689050268BC
:10AF40000A4302600421284600F090F8207840B2BD
:10AF50002C4600250028C0D42B4800687D21C9005C
:10AF6000F5F7B8F820492D314143204600F050F85C
:10AF700003F03CFF04463868C069C00705D003F001
:10AF800035FF001B31888842F5D903F02FFF0446B6
:10AF90003868C169890706D503F028FF001B31888E
:10AFA0008842F5D938680121009A116017498161FA
:10AFB000284603B0F0BD0321216000288AD08AE72B
:10AFC000034804A1084A09A303F03EFF4893010285
:10AFD000EC2E0100666C6173685F736563746F7259
:10AFE0005F657261736500002B0200007365637416
:10AFF0006F7220696478206973206F7665722072A1
:10B00000616E67650D0A000028E00102000093EB05
:10B01000F0B583B001917C220290424353498C18D1
:10B020002546143503F0E2FE06460221029800F0A0
:10B030001DF803F0DBFE07462068C169890606D4C7
:10B0400003F0D4FEC01B29888842F5D92068007D12
:10B05000C00708D06420FEF7CDFD03F0C7FE801BBB
:10B0600001998842E1D903B0F0BDC046F0B585B082
:10B07000049104467C2060433C490F183D4614353A
:10B0800003F0B4FE06463868C069C00705D003F077
:10B09000ADFE801B29888842F5D903F0A7FE06463D
:10B0A0003868C069800705D503F0A0FE801B298899
:10B0B0008842F5D91421049B5943DC2060432C4A73
:10B0C0001018039002914018018A8268C47C74268B
:10B0D000BE5D012E0DD10191012B02990CD0012BE7
:10B0E0000DD07526BE5D012E0ED0019E072B0ED110
:10B0F0000EE00E4602990BE00222012BF1D138241A
:10B100007526BE5D012EF0D10326072B00D0019ECF
:10B11000184B334024069207D20A1219D218039B07
:10B120005958C907490C52184168CB071B0CD21853
:10B13000837C5B075B0BD218C0684007000A1018BD
:10B140003A685060002E0ED001290CD103F04EFE5B
:10B1500004463868C069800705D403F047FE001B29
:10B1600029888842F5D905B0F0BDC0464893010250
:10B17000A8240100FF3F0000F0B59DB00D46012658
:10B18000890E2FD0002B2DD011928121C90410934C
:10B19000C91AA94226D30121EFF310840C4002D131
:10B1A000EFF3108272B67C220F904243E74814926C
:10B1B0008718384610303B690026062B0DD80A4602
:10B1C0009A40D3065B0F07D161231A4200D16FE387
:10B1D0000E46002C03D003E00226002C00D162B6FC
:10B1E000002E02D030461DB0F0BD0290BD6500219A
:10B1F000139179651098401E12904019B964B9698D
:10B200000D916E1A1199B962FD6238637E63F98CF3
:10B210000E913046F4F75EFF0446B863129830187A
:10B220000E9E3146F4F756FF109B011B4A1CF86333
:10B2300039647A64139A0029194608D07043591961
:10B240000D9BC91A0A1A7443581B801901193846F4
:10B2500048300E90384644300D90384640300B90C0
:10B2600038462630059038465830139038465430CA
:10B270001290F9643A651498B44908581021C161D4
:10B280003846143014903846503004903D464C35C2
:10B2900003F0ACFD04463868C069C00606D503F06B
:10B2A000A5FD001B149909888842F4D9F87D400651
:10B2B0000C9500D574E201230E9803600D98016887
:10B2C00000290F9800D1CDE23A4674320A92DA048E
:10B2D00007921A0509921922520606920722D206EF
:10B2E000089216E09A4800687D21C900F4F7F2FE42
:10B2F000109941430F9C2046FFF78AFE20460C9D83
:10B300000E9A11684B1C13600D9909688B4200D985
:10B31000A8E20B9A1268012A55D0002A00D0A8E0B2
:10B320002E6812990C6813990D6806211091FFF789
:10B330009DFE386885601198051903F057FD044695
:10B340003868C069C00706D003F050FD001B14998F
:10B3500009888842F4D903F049FD04463868C16978
:10B36000890707D503F042FD001B1499098888421C
:10B37000F4D938680A990A78012A089900D0069900
:10B38000012A099A00D0079A3346724C234013438E
:10B390000B4371490B434360002EA3D003F026FDFD
:10B3A00004463868C069800706D403F01FFD001BFF
:10B3B000149909888842F4D93868297801756D1C78
:10B3C000761EFAD18EE7012B00D0C7E02E681299C5
:10B3D0000C6813990D6806211091FFF747FE386835
:10B3E00085601198051903F001FD04463868C069AD
:10B3F000C00706D003F0FAFC001B149909888842A4
:10B40000F4D903F0F3FC04463868C169890707D50D
:10B4100003F0ECFC001B149909888842F4D93868C1
:10B420000A990A78012A089900D00699012A099AEE
:10B4300000D0079A3346474C234013430B434649F9
:10B440000B434360002E69D003F0D0FC04463868FB
:10B45000C069800706D403F0C9FC001B1499098851
:10B460008842F4D93868297801756D1C761EFAD1A6
:10B4700054E0012B00D0C9E02E6812990C68139992
:10B480000D6806211091FFF7F1FD3868856011986D
:10B49000051903F0ABFC04463868C069C00706D044
:10B4A00003F0A4FC001B149909888842F4D903F026
:10B4B0009DFC04463868C169890707D503F096FCEE
:10B4C000001B149909888842F4D938680A990A78C7
:10B4D000012A089900D00699012A099A00D0079AF2
:10B4E00033461C4C234013430B431B490B4343601F
:10B4F000002E13D003F07AFC04463868C069800738
:10B5000006D403F073FC001B149909888842F4D90F
:10B510003868297801756D1C761EFAD10C480068D0
:10B520007D21C900F4F7D6FD109941430F9C2046B8
:10B53000FFF76EFD20460C9D2A68139B1968891839
:10B540001960129B196889181960D9E6489301029D
:10B5500028E00102FF3F0000008080008B4200D005
:10B56000CEE604990E6812990C6813990D680621AD
:10B570001091FFF77BFD386885601198051903F07D
:10B5800035FC04463868C069C00706D003F02EFCBD
:10B59000001B149909888842F4D903F027FC04465B
:10B5A0003868C169890707D503F020FC001B14998E
:10B5B00009888842F4D938680A990A78012A0899D2
:10B5C00000D00699012A099A00D0079A3346D44C34
:10B5D000234013430B43D3490B434360002E00D158
:10B5E00080E603F003FC04463868C069800706D48F
:10B5F00003F0FCFB001B149909888842F4D93868D1
:10B60000297801756D1C761EFAD16BE6129A1268C4
:10B61000119CA618139A15688B425FD104990C6887
:10B6200006210391FFF722FD3868856003F0DEFBF9
:10B6300005463868C069C00706D003F0D7FB401B39
:10B64000149909888842F4D903F0D0FB10900C9D1E
:10B650003868C169890708D503F0C8FB1099401AFA
:10B66000149909888842F3D938680A990A78012A16
:10B67000089900D006991091012A099A00D0079ADA
:10B680002346A7490B40134310990B43A5490B438D
:10B690004360002C14D003F0A9FB10903868C069F7
:10B6A000800707D403F0A2FB1099401A1499098867
:10B6B0008842F3D9386831780175761C641EFAD156
:10B6C0009A4800687D21C900F4F704FD03994143BD
:10B6D0000F9C2046FFF79CFC204611E605990C883C
:10B6E00006210391FFF7C2FC3868856003F07EFBFA
:10B6F00005463868C069C00706D003F077FB401BD9
:10B70000149909888842F4D903F070FB10900C9DBD
:10B710003868C169890708D503F068FB1099401A99
:10B72000149909888842F3D938680A990A78012A55
:10B73000089900D006991091012A099A00D0079A19
:10B74000234677490B40134310990B4375490B432C
:10B750004360002C14D003F049FB10903868C06996
:10B76000800707D403F042FB1099401A1499098806
:10B770008842F3D9386831780175761C641EFAD195
:10B780006A4800687D21C900F4F7A4FC039941438D
:10B790000F9C2046FFF73CFC204605990A88CCE622
:10B7A0005E4815A90A4678C878C278C878C20125CB
:10B7B000E8073A68136803431360B868FEF78AFA2B
:10B7C00002200026139C2168BA6AF9653A6610992E
:10B7D0007966BE66F8660C980068129A11680918B6
:10B7E00011600E9B19684A1C1A60226810182060AC
:10B7F000002900D0F6E410953846603013903C469E
:10B800005C3438460830129006210F98FFF72EFC62
:10B810003868216881600C980068119003F0E6FA9E
:10B8200004463868C069C00706D003F0DFFA001B81
:10B83000149909888842F4D903F0D8FA0446109D77
:10B840003A68D069800707D503F0D0FA001B149935
:10B8500009888842F4D93A687420385C01282DD0D0
:10B86000E9042CE003F0C2FA04463868C069C00756
:10B8700006D003F0BBFA001B149909888842F4D95A
:10B8800003F0B4FA04463868C169890707D503F0A4
:10B89000ADFA001B149909888842F4D9386801214F
:10B8A000029A116022498161002630461DB0F0BD28
:10B8B00004210160002C00D191E491E42905119C40
:10B8C000174B2340591801280C9D02D0192040061F
:10B8D00001E00720C0060818124940185060002CEB
:10B8E0000ED003F083FA04463A68D069800707D483
:10B8F00003F07CFA001B149909888842F4D93A684D
:10B900002B681398016812980068074C0094143251
:10B91000FEF750FA30461DB0F0BDC04620230100AE
:10B92000FF3F000000808000C1A5000028E0010268
:10B93000000093EB3920C00001490968085870479E
:10B94000D4920102F0B5032920D8C0467944097980
:10B9500049008F4401080F15012181404F4B1B689E
:10B960005963D96212E0012181404C4B1B68196375
:10B97000D9620BE001218140484B1B68596304E008
:10B9800001218140454B1B6819639962830043493B
:10B99000CB18DA608A68002A29D14A68002A16D4AE
:10B9A000032314469C43174BE5589607F60EFF27D2
:10B9B000B740BD438027B7402F43E7501F231340B4
:10B9C00001229A40104B1A60104B1A600FE0930747
:10B9D000DB0EFF259D400F241440083C03229443B6
:10B9E000074AA658AE4380259D403543A550012205
:10B9F000824008680262886810438860F0BDC046D3
:10BA00001CED00E000E400E080E200E000E100E086
:10BA100010B501242046FEF715F8204602F0E8FE96
:10BA2000002010BD012181401C48006842688A4303
:10BA300042607047194909680968C14001200840FF
:10BA40007047C046012181401448006842680A439B
:10BA500042607047012907D0002910D1012181409F
:10BA60000F4802680A430FE0012181400B4800683B
:10BA70004368002A0DD00B434360016170470121E8
:10BA80008140074802688A430260044800684161B7
:10BA900070478B43436001617047C046D8930102F1
:10BAA0000801004080B5114A1170114A10708001E0
:10BAB000C90101430F480078400108430E49097845
:10BAC000090101430D480078C00008430C4909787A
:10BAD000890001430B480078400008430A4909786F
:10BAE0000143C8B2F8F722FE80BDC046189F01028C
:10BAF000E69601021D9001029CEA0102D1AD01020D
:10BB0000199F01025CA301025DA301020122824090
:10BB10000548002903D0016811430160704701689E
:10BB2000914301607047C04600010040124A072857
:10BB300009D880000F238340814019401068984342
:10BB40000843106070470F280AD8800020380F2360
:10BB500083408140194050689843084350607047C3
:10BB6000800040380F2383408140194090689843FB
:10BB7000084390607047C04634000040F0B543076A
:10BB8000DC0E0726A640C3089D000E4BEF187D680B
:10BB9000B5433E1D002908D03560012282400129AD
:10BBA0000CD1186810431860F0BD0121814018685D
:10BBB00088431860A24015433560F0BD1868904373
:10BBC0001860F0BD0C01004010B582B014460A4662
:10BBD00001460498009301900820234600F092F853
:10BBE00002B010BDB0B584B014460A4601460898AC
:10BBF00002250095019302900720234600F052F998
:10BC000004B0B0BD70B500285BD031490A78314925
:10BC1000002A03D14A68012313434B6042880388FA
:10BC20001B049A180B46183B1A60828883891B04F0
:10BC30009B180C460C3C23600B46083B84681C6038
:10BC4000446903232340057CAD00EB188569AD07EB
:10BC50002D0D5B19457C2D035B19C569AE07B60A2E
:10BC60009B19867CB6059B190E1F3360036A122B45
:10BC700004D107240C60541EA2410AE0032C05D114
:10BC8000012D03D807220A60012202E006220A6081
:10BC90000122114C002525700F2464012034C57C3D
:10BCA0006D0225401B069B0BD218C3791B07DB0EC8
:10BCB000D21880790007C00D101840191439086097
:10BCC00070BD064806A1862209A303F0BDF8C04650
:10BCD00014CD01021810005016CD0102C93B01001D
:10BCE0006C73705F656E67696E655F72756E00007C
:10BCF000506172616D65746572206973206E756C38
:10BD00006C000000F0B58BB0109E34043ED00D46A0
:10BD1000D64C2140012701977F06B9423CD11146FC
:10BD20002140B9423FD11C40BC4243D1119902ACE1
:10BD30000027E781E780668027802782A774E17467
:10BD40009908A181A908A1800A90099708970797E7
:10BD5000900880B204902046FFF754FFAA4800786C
:10BD6000002801D00BB0F0BDAB480168C90708D16D
:10BD70000168C90705D10168C90702D10168C9076F
:10BD8000F3D07F48019901700BB0F0BDB8480D4960
:10BD9000AF22C14B03F058F80095B5480949B022CD
:10BDA000754B03F051F80092B1480649B122724B2D
:10BDB00003F04AF80093AE480249B2226E4B03F0FA
:10BDC00043F8C0469F3B0100F0B58DB00392139E2F
:10BDD000340446D00A46A54C2140012502956F0641
:10BDE000B94244D103992140B94247D11C40BC42D9
:10BDF0004CD11499129D04ACE17429492182002789
:10BE0000E781E780668027809908A1819108A18059
:10BE10000B95012D01D16121CF43A7740C90022015
:10BE20000A9009900398800880B206902046FFF798
:10BE3000E9FE75480078002801D00DB0F0BD7648C5
:10BE40000168C90708D10168C90705D10168C90798
:10BE500002D10168C907F3D04948029901700DB0B9
:10BE6000F0BD83480D49FB228B4B02F0EDFF0092A1
:10BE70007F480A49FC22404B02F0E6FF03980090FD
:10BE80007B480649FD223C4B02F0DEFF00937848D8
:10BE90000249FE22384B02F0D7FFC046AC3B0100FE
:10BEA0008E8E0000F0B58BB0119E340447D00D4645
:10BEB0006E4C2140012701977F06B94245D11146BA
:10BEC0002140B94248D11C40BC424CD11299109F2C
:10BED00002ACE174294921820021E181E180668080
:10BEE00021809908A181A908A1800997012F01D07B
:10BEF000712100E06121C943A1740A9003200890D8
:10BF00000790900880B204902046FFF77BFE3E48E1
:10BF10000078002801D00BB0F0BD3F480168C90788
:10BF200008D10168C90705D10168C90702D10168B4
:10BF3000C907F3D01248019901700BB0F0BD4C480D
:10BF40000C49D522544B02F07FFF0095484809491F
:10BF5000D622094B02F078FF009245480549D722C6
:10BF6000054B02F071FF009341480249D822024B71
:10BF700002F06AFFBB3B0100E93B0100868600003E
:10BF800016CD010210B582B014460A4601460020C3
:10BF90000093019004202346FFF7B4FE02B010BDC9
:10BFA00010B584B014460A46014600200090019363
:10BFB000029004202346FFF707FF04B010BD0000E5
:10BFC00070B50D46064604242046FDF73BFD20468D
:10BFD00002F00EFC0B4805600B480670002E0ED0D8
:10BFE0000A48016880220A437F218A4302600120B7
:10BFF00000030749086007490860074804600020FB
:10C0000070BDC04618CD010214CD01020CE400E061
:10C0100080E200E000E100E01C100050B0B582B00A
:10C02000144602461148204001256D06A8420DD154
:10C03000180413D0174801600020009301900620D7
:10C0400011462346FFF75EFE02B0B0BD0094FF220A
:10C050008C320748074908A302F0F6FEFF208C3017
:10C06000421C034803490C4B02F0EEFE0300FCFFA8
:10C07000C93B0100913B0100447374206164647208
:10C0800065737320257820697320696E76616C6909
:10C090006400000008100050073C010080B582B029
:10C0A0000B46014600200092019003200A46FFF74C
:10C0B00029FE02B080BD0000002801D0042100E06C
:10C0C0000221C54A5172411E8841800103490A6814
:10C0D00040239A43101808607047C04650A0005093
:10C0E000F0B583B002912E49CD7A0E7B7719874245
:10C0F0004FD908990191182545434126F604BF0000
:10C10000BE19745B34490C4057033C199B07D90C8A
:10C110006418324B1B681B7A745375196C8803269C
:10C12000B60326409B079B0C9B193F24044018191B
:10C13000029CA3061B0DC0186880012A184E13D854
:10C14000707B14224243307B5023434324011B194C
:10C150009A18F37AC0181C234343D01880081E4A4B
:10C16000104007430F432F800198686001F0C4FE20
:10C17000A860E8681A4908403030E860286908403B
:10C180002721715C4018286100F044FE686103B00B
:10C19000F0BDFF228832034803A108A302F054FE39
:10C1A0001CD20102583C01006D61635F63735F63E1
:10C1B0006F6E7374727563740000000043532069DE
:10C1C0006E646578206973206F7665722072616E87
:10C1D00067650D0A00000000FF070000449401029B
:10C1E0000000F0FF2820D84900220A547047C046BA
:10C1F000F0B581B0009314460D460746062630463A
:10C20000FDF720FC304602F0F3FA26211D48475482
:10C210000021017041708171017181704171C170A3
:10C22000C17102224272C16201634163816304737E
:10C230004273C572009A561C134A1680017241203F
:10C24000C00401214903F3F7AEFF502060432901E8
:10C25000081861198A00801818224A438018B2B25F
:10C260004A438018094940180949884204D200F01D
:10C27000B5F8002001B0F0BD064807A19A2209A335
:10C2800002F0E2FD1CD2010218D2010228000802CD
:10C2900001200802583C01006D61635F696E69749A
:10C2A00000000000454D206F766572666C6F770D5B
:10C2B0000A000000A448C179002901D0012070477C
:10C2C000007A411E88417047F0B583B002912A4937
:10C2D0004B7B834248D9CB7A0C7BE31818245C4310
:10C2E0009B00E3184124E4041A1914240190054624
:10C2F00065430026565100925519EE882E4F0B4685
:10C300007A1C3240F54E3688497A711A2B4E0E400F
:10C31000B618EE803740997BEF80AA88284F1740E7
:10C320004A424A4191007918264A8918A980264F25
:10C330000F402D1D029801280AD124490E400921E1
:10C34000C902711869800121C9037918298000E0A8
:10C350002F800198444300980019074A918C41822C
:10C36000118C018203B0F0BD3520C200034804A146
:10C3700009A302F069FDC0461CD20102583C01002D
:10C380006D61635F6C696E6B5F646573635F636F40
:10C390006E737472756374004C696E6B20646573A0
:10C3A0006320696E646578206973206F76657220FA
:10C3B00072616E67650D0A00FFFBFFFFFF0300005F
:10C3C00003D0FFFFE80F0000EF1F0000FF83000015
:10C3D000BE4A5063916370471CD20102F0B581B030
:10C3E0004348CC21016003214160B8490A7BD30452
:10C3F000404C1B19CC7AA218541E1C4318235343DB
:10C4000092009A184B7B14255D43521992012243E6
:10C41000012463061343436100228262C262026305
:10C4200042638263C26342650267334B1A605A609B
:10C430009A60324B1A601A619A61DC61304C1C625E
:10C44000304C251D1D6325460C3D5D632546283D6A
:10C450009D632D4EDE631C645C642C4D2F461C379F
:10C460009F642746143FDF64103C1C65284C5C65C4
:10C47000284C9C650C369E67274CA5634035E563C8
:10C48000DA651A665A669A66DA661A67234DDD67B8
:10C4900002258561224DC561C325AD03CD620A63C6
:10C4A000D2435A601F4A1368FF25AB4326254D5DD2
:10C4B000AD072D0EEB1813601B4A102313601B4AA7
:10C4C0001360272260238B5419498160C160016188
:10C4D00021607D210901016641661649C164164942
:10C4E00041641649016400F085FC01B0F0BDC0460E
:10C4F00004A000500000F8FF94A0005034A10050A8
:10C50000FF185A0030040040041000401C20004076
:10C510005430004060400040B8A1005014001400A6
:10C52000FF3F3FFF04E400E080E200E000E100E0C4
:10C53000DC05DC053F0270020133D007D007D007CD
:10C540002921C64A505470471CD20102F0B58BB065
:10C55000079208910146C14FB8780991FFF7B4FEE0
:10C5600078793A7B79790691824200D89FE0FB7A0C
:10C570009A181823534392004124E104049152185D
:10C58000D2187B7B14214B43D2185024604315589A
:10C5900001230A93DB022E469E4316504E4B2B403E
:10C5A00005937D7B03914D433E7B7443F97A0B01E8
:10C5B0001B195B1971181C24029461435918A84B6C
:10C5C0001B88069C5C430919C904490D059BC918C1
:10C5D000115010180799416038787979089A0092BB
:10C5E0000322099BFFF77CFDF87A397B091838781C
:10C5F000814263D983000993049AD45C0894F7219B
:10C600002140D154D1184D788E7836027619CB78E6
:10C610001B04F31807900A9886051E43330CCB7051
:10C62000FB7A387BBC784D709F4D3540039E664346
:10C63000C018029B4343981940029C4B03405C196D
:10C64000200A8870200CC870F023089D2B401B1D09
:10C650003D7B0895FE7A099D5355C8700620079AC0
:10C6600050438019089A801848701F22D202224035
:10C670000243100A88707879401C7871387B797988
:10C68000814201D3002179713978491C3970F97AD6
:10C6900008183978884201D80020387028200A9973
:10C6A0003954387A401C3872387A0BB0F0BDA72064
:10C6B0004200D2480649074B02F0C6FBA7204200C1
:10C6C0007A32CE487349744B02F0BEFB1CD2010291
:10C6D000783C0100213C010000F0FFFF18D201026C
:10C6E0000320000605490A6882430A600A6802437B
:10C6F0000A600348012101607047C0461C000040E9
:10C700001CA0005080B50120FDF752FC80BD000048
:10C71000F0B587B006930646504C607A504B1B88A4
:10C72000181A0C9DA84200DC89E00F460592012EE4
:10C7300006D156480021C1620169554A8918016035
:10C74000A0783146FFF7C0FDE078E178069A2B46E5
:10C7500000F0AEF82078E178009700220692334688
:10C76000FFF7BEFCE07A217B0818217888426ED959
:10C770004120C20404918800815C0391F7250D409B
:10C78000029285544549455C4549465C3602761916
:10C790004449475C3F04F6190127BF0537433E0C67
:10C7A0004654E67A217BA3783C4A85543E4D3D4071
:10C7B00014275F4389191C234B43D91949023B4B6A
:10C7C0000B405D19290A364BC1542E0C354946548D
:10C7D000F02703990F400599002900D13F1D217BC7
:10C7E000E37A029A87542F4A86540622049E7243A3
:10C7F000D2185118294A81541F22D20215400D43E4
:10C80000290A274A8154E078401CE070E07AE178F8
:10C81000814201D30699E1702178491C2170217B66
:10C8200008182178884201D806982070E079401CC9
:10C83000E071A07A401CA072E07907B0F0BD392009
:10C84000C2001632074808A109A302F0FDFA3920F8
:10C85000C20004480F49104B02F0F6FA1CD2010244
:10C8600018D20102583C01006D61635F74780000CA
:10C870004D4143205458206C656E206973206F76BB
:10C8800065722072616E67650D0A00000804004041
:10C8900090D003008E3C01003F3C010001000802E3
:10C8A0000200080203000802FF07C0FF00F83F0073
:10C8B000F0B589B00893019204914F4DEF7A874209
:10C8C00000D891E0297B502632464A434124E304B4
:10C8D0000693D218CC19A10051181822059254437E
:10C8E0000A19697B142307935943531802900001D6
:10C8F000195804460390504A0A40A97AC9025118AF
:10C9000008988205D2088A181A514C4911402A7B8E
:10C9100000965643384CE57A2C0106982418A7193E
:10C92000354E5419A5007D19059844432819747B88
:10C93000079D6C430519049FD2194148048854434C
:10C940002A19089CD204520D51181D4603981950FB
:10C9500000F06AFA0146707A001902043E460CD0D3
:10C9600080B2C000002900D1801E029FA52149008D
:10C97000F3F7B0FB1F21014001E00021029F3801C5
:10C980002818427983791B029A18C3791B04D2189C
:10C990002C4B1340437109045918090CC171002C28
:10C9A00020D0154835460646007B009B4343F17A6C
:10C9B0000A01069F3A43D21841188B00D218059BF2
:10C9C0004B43D118727B079B5343C91840191C4A2B
:10C9D0001288424388180199884203D0019922465F
:10C9E000F3F7C8FB09B0F0BDFF225C32034804A195
:10C9F00009A302F029FAC0461CD20102583C0100EA
:10CA00006D61635F74785F646573635F636F6E739A
:10CA100074727563740000005458204445534320D9
:10CA2000696E646578206973206F76657220726123
:10CA30006E67650D0A000000FF0700E000F8FFFFC9
:10CA400018D20102EFFFE00082B0FCF717FE0520CC
:10CA500000252946FFF76AF806202946FFF766F801
:10CA60000A202946FFF762F809202946FFF75EF8F9
:10CA70000124204603F0C6FB284603F0C3FBFCF765
:10CA800039FE2046FCF72CFE01F032FE01F02AFEB2
:10CA90006D4801686D480068890308D403210907BF
:10CAA00008402107884202D0FCF7B6FD06E0FCF7FB
:10CAB0001BF9FCF7C9FD0020FDF7C0FCFCF754FE94
:10CAC0000025284604F0DEFC032661A230463146EC
:10CAD00003F016FA30462946FBF7A6FBF7F724FFCA
:10CAE000FAF7E6FDFEF794FF5F4F381DFCF7C0FB39
:10CAF000F7F712FCF6F740FBF7F7A3FE04263046E3
:10CB00002946FFF713F8304621462A46FEF7A2FFD2
:10CB1000052230462146FFF731F820462146FEF730
:10CB2000C1FF674E30462430504A01902146FCF741
:10CB300011FBFAF7E5F8A2024D494E4B204603F0EF
:10CB40005FFE01F0B3FBF6F705FB4B4A204621469A
:10CB500002F090F8494802F0BDF84948FCF746FD5C
:10CB6000B87800280DD104E0FBF7A0F9B8780028C8
:10CB700007D1F7F7D1FE002803D1F079002815D1AD
:10CB80003CE0FCF77DFCB079002802D0B571F6F7E7
:10CB90004FF9F7F7D5FEF6F7E7FEF7F717F9FAF7CB
:10CBA00095FDFCF74BFCF079002827D0F571B078A3
:10CBB000411CB1703D2806D30020B07001210198BE
:10CBC0002A4AFCF7C7FAFAF72FFF2E480470F7F746
:10CBD000A3FE002802D0BD70F57007E0F0781E2893
:10CBE000214600D32946B970401CF070F7F72AF9A6
:10CBF0007F20C105B069F3F7AEFBB0610B20FEF7F3
:10CC000019FF3978002810D00029ADD101201E4924
:10CC10000870387000201D49087003F0CDFAFBF74A
:10CC200045F9B8780028ACD1A3E701299CD10020B0
:10CC300038705049C883144908700120134908709E
:10CC400003F09AFA90E7C046180000403000014017
:10CC50005557422073696D706C65206578616D7001
:10CC60006C650D0A000000001C9001024990000054
:10CC700018CE0102390A01001DEC00007C3F0000C3
:10CC8000B9CC0000E6960102189001021990010249
:10CC9000014800687047C0460C00004081B080B574
:10CCA00081B0039303AB009302F0A4FD01B080BCFC
:10CCB00002BC01B0084700000148002181617047B3
:10CCC000B8980102F0B581B0002630463146FDF734
:10CCD0001BFE0125AC022649264F30463A46234624
:10CCE000FDF772FF3988244881423ED064217E528C
:10CCF00062217E5260217E524422BE52FD87BD8752
:10CD000078227A8702223A874322FA86BE83FE81FE
:10CD10001A4ABA817E810A223A81C822FA80184AC8
:10CD2000BA803880FE8306203885F984FF201230CF
:10CD300078848730B88450203E523A83EFF31080D5
:10CD400072B630463146FDF7DFFD00280CD12A03CC
:10CD500000263046064D2946FDF730FD054A30468F
:10CD600029462346FEF708FA62B601B0F0BDC04678
:10CD700000E002046AA90102AA550000E1FF0000D8
:10CD8000341200000020704710B50024002809D09C
:10CD9000002905D003464A0003481946F3F7EAF98B
:10CDA000204610BDE04310BD3C9301020146002027
:10CDB0000A2901DAC0437047014A11807047C04612
:10CDC000C49301020020704780B50188064A118093
:10CDD0008178064A1170C178054A11700079FCF714
:10CDE00073FB002080BDC0462E94010230940102E6
:10CDF000CCD20102044805490160152109044160B3
:10CE0000034981607047C0469C30004041000800E3
:10CE1000340007000748006840697047FD20400063
:10CE200004490968085C7047024800686221405C58
:10CE30007047C0464494010210B50648046806488D
:10CE400000686421F3F75CF90221C94341430819E2
:10CE500010BDC046D0D20102D4D201020A491A2222
:10CE60000A600A4948704878FF210902084A136895
:10CE70008B43800380B2C0181060064820210160F7
:10CE80000548016000207047702000403494010282
:10CE900004E400E080E200E000E100E0F0B5A9B0C9
:10CEA00016460F460546C648002B024600D01A46D5
:10CEB0003921CC003D21C9005118119182421892AC
:10CEC00006D001204202BE491898F3F753F9189A88
:10CED0006120111913910E21119C0A91A170002F4C
:10CEE0000D9501D00A2100E00921592317938300F1
:10CEF000E170784278411399087030781090107082
:10CF0000F17AE17471785170B7789770F178D170D7
:10CF10003579157174795471B1799171F179D17153
:10CF2000317A1172717A5172B17A91727E1EF0B2B9
:10CF300000210328169106D870B28000A1A21058D3
:10CF40006A00805A1690179882001898C01814909A
:10CF5000F81E022804D3012E084604D89D4800E09C
:10CF60009D48031918781290189DA8181790284604
:10CF7000303015902C4656346D2080002950974A49
:10CF8000974B149E33627262B362F2623176F18221
:10CF9000139B597009229A70281841608160C16002
:10CFA0000161109880008F490858F3F771FD012F37
:10CFB00010900F9104D0022F05D17F217E2004E034
:10CFC0007C217B2001E05B215A20159DA9842070E3
:10CFD00003200C90A080012666701F200B90A88271
:10CFE0001820A8740A46083A179BDA76169B129AFC
:10CFF000D2184A439100189A9163B702791E8B4266
:10D000000E9109D978486080342068847748288256
:10D0100077481399088339E07F2B10DD802B18D0D7
:10D0200031028B421BD071028B4227D16E49618045
:10D0300068846F4813990883CF20C00025E0202B17
:10D0400017D0402B1AD16848608004206884694852
:10D050001BE06548608006206884674815E06248E8
:10D06000608010206884624813990883C520C0003E
:10D070000BE0624860800220688404E00420688439
:10D08000812040006080FF2002302882104600F09E
:10D09000D7FE1298102806D0402808D108201499ED
:10D0A000C876072000E004201799887002E01798DE
:10D0B0000C9981701898169A8078C11E02290CD399
:10D0C000022811D001280CD12672BA4200D90026BC
:10D0D0006672BA4213D8F44812E00D20000211998A
:10D0E00008800120800201E00C9800022081BA42F1
:10D0F00001D8EE4800E0FA20179988600EE0FA2087
:10D1000017998860139800780028119901D0E84891
:10D110004880E848139A1083E7480880A88CF3F702
:10D1200019FC0026E54B3246F3F79CFA02460B4603
:10D13000E3493046F3F7FEFAE24B3246F3F792FA50
:10D14000F3F75AFC0746E080DF493046109A0F9B00
:10D15000F3F7F0FADD4B3246F3F784FAF3F74CFCC1
:10D1600078434042800B608116990E98814208D91D
:10D170000C20149FB872D648179988831220189AE9
:10D180000EE0480A189A149F01D00D2003E0080A07
:10D1900000D1DBE20A98B872CE4817998883122032
:10D1A000F872D078052844D8784400794000874444
:10D1B0000227402C3339C848B881C8482FE0C04600
:10D1C000D4900102D0220100D0220100E02201000F
:10D1D000E0220100C01F0100C71F010030750000E0
:10D1E000102700008020010005020000FF0600005B
:10D1F000040800000A0400003604000003020000D6
:10D20000B748F881B748388013E0B748F881B74885
:10D210003882B74838600CE0B448B881B5481799EF
:10D22000C88306E0B4487882B448B8800B980006FA
:10D230009064AE483881A748F880B14802882A84B3
:10D24000B0480078E874B0480078119F7875387D50
:10D25000139000285ED0AD490A681023DA413A6085
:10D260000A794B79CF8867801B029A186A840A7AF8
:10D270004B7A8F7AC87A0D7B65701B029A183B0433
:10D28000D21800061018179FF860487B8A7BCB7B6A
:10D290003B77120210186081087C7877487C149ADA
:10D2A0009072887CD072C87C159B1874087D587465
:10D2B000487D11909874C87D0A7E120212181A8453
:10D2C000887DD87418464B7EC375887ECD7E2D022E
:10D2D0002818B880087F4D7F2D022818F880887F95
:10D2E000B877C87FF8772020085C149D2873212028
:10D2F000085C68732A20085C2A314D782D022818B2
:10D300008D782D044019C978090640181899886449
:10D31000119801E0EB7DA87C7D498B700A8080002C
:10D320001F38C882C883139800281FD0222277484C
:10D33000825C034622335B781B029A180A842422FB
:10D34000825C034624335B781B029A18CA84262227
:10D35000825C034626335B781B029A188A83282254
:10D36000825C283040780002801888846948032550
:10D3700069A2294602F0C4FD189F387814907B7882
:10D38000B8780F90FA78B8791390F8791190387AC4
:10D390001090787AB97A0890099100930F980190CB
:10D3A0000292169803901298049013980590119881
:10D3B000069010980790FAA2F8482946149B02F0AC
:10D3C0009FFD3D46643580212846F2F7ECFEB87893
:10D3D000C11E02290ED3012800D18FE1022800D0FE
:10D3E000ABE11691149078787F225043F7494018AA
:10D3F000F74907E01691149078785B225043F14981
:10D400004018F14941182846F2F7B4FE0D9D1898CE
:10D41000C6870E34324602E0641C0F2A0ADA2178ED
:10D420000029F9D0491C8907C90F91400E43C687CE
:10D43000521CF1E71699022907D31499491E0129B4
:10D4400000D97DE14279D24901E04279CF4989187A
:10D450000C78002D00D177E1C1790E91032900D914
:10D460004AE14279062A00D979E149218900411827
:10D470001191E43010900E98401E129019A80019D6
:10D480000F9000231392149403E01898290600D1FA
:10D490005AE1052A5AD8C0467A4412795200974474
:10D4A000455C728598ABC04688130000E20400001A
:10D4B0000C080000060A0000040F000000001041E4
:10D4C00030C1BD41000070400000F0400000D0417C
:10D4D000120C0000140B000012120000140E0000C9
:10D4E0000E160000130D0000121600000E120000B0
:10D4F000140B0E0A12080000101600000E0B00009C
:10D500002E94010230940102CCD20102D8D2010241
:10D510009C940102010800004361736520706172F0
:10D52000616D65746572733A200D0A001693DFB25F
:10D53000002F04D019A801223946F2F72DFE002C45
:10D5400000D191E019A8C019BB498AE0E8B20228CD
:10D5500067D00027022867D06BE00E98022872D1AE
:10D56000E8B2022800D103461693DFB2002F04D0A0
:10D5700019A801223946F2F70FFE002C74D019A821
:10D58000C019ACA16DE0E8B2022800D104231693C3
:10D59000DFB2002F04D019A801223946F2F7FCFDB2
:10D5A000002C61D019A8C0199FA15AE0E8B2022846
:10D5B00000D106231693DFB2002F04D019A8012250
:10D5C0003946F2F7E9FD002C4ED019A8C01992A1F6
:10D5D00047E0E8B2022800D10C231693DFB2002FF7
:10D5E00004D019A801223946F2F7D6FD002C3BD011
:10D5F00019A8C019874934E0E8B2811E4A424A415D
:10D600009700022804D119A801223946F2F7C4FD77
:10D61000002C16D019A8C0197CA12246F2F7AAFD49
:10D620000FE00627022804D119A801223946F2F793
:10D63000B3FD002C05D019A8C01980492246F2F785
:10D6400099FD169710E01693DFB2002F04D019A8A9
:10D6500001223946F2F7A0FD002C05D019A8C01907
:10D6600073492246F2F786FD3C193F2C05D80F98E6
:10D67000C0194021091BF2F796FD1298022818984C
:10D6800001D2002002E0C078411E8841159908703F
:10D69000611E2E46E8B202280CD1179A517019A9C2
:10D6A000119AB8C9B8C2B8C9B8C2B8C9B8C2B8C95D
:10D6B000B8C20DE0179A117019A9109AB8C9B8C26A
:10D6C000B8C9B8C2B8C9B8C2B8C9B8C2C10709D1C7
:10D6D00080073546149C139A169B00D4D5E6022089
:10D6E0008543D2E6FE20354605401898149C139ACF
:10D6F000169B290628D0CCE637A231E0169114906B
:10D7000078780B994143334808181F386F21C94373
:10D710000D9D7A180378D427D3554378D827D3554D
:10D720008378DC27D355002900D170E6C378E02741
:10D73000D3551031001D189FEBE70120404A10E03F
:10D740000024002D00D087E629B0F0BD80290ED33B
:10D750000F20B872104817998883102020E525A261
:10D760000120014602F0CCFB189829B0F0BD102032
:10D77000402904D3B8720849179B998310E5B87201
:10D7800004481799888314200AE5C046C71F010082
:10D79000C01F0100150F0000140B0000010800005D
:10D7A0002564202564202564202564202564202507
:10D7B00064202564202564202564202564202564B8
:10D7C0000D0A0000144601001DF7FFFF2C3D01006B
:10D7D00089FBFFFF1C4501007472785F6D6F646503
:10D7E00020706172616D65746572206572726F720E
:10D7F0000D0A00004E73666420706172616D65747D
:10D800006572206572726F720D0A0000FFFFFFFFE4
:10D8100001FF000080230100FFFFFFFFFF0101FF68
:10D82000FF01FF01FFFF01FFFFFFFF01FFFF01FFFE
:10D830006C290100FFFF01FFA0230100F02201007D
:10D84000CA3C0100002800D1014806490860704721
:10D85000D4900102F0B586B0002805D101480068D7
:10D8600002E0C046449401023121C90004914118EC
:10D870008A791F231A40CD79ED06AD0DAA180D7ACD
:10D88000ED066D0C52194D7AED062D0B52198D7A5D
:10D89000ED06ED095219CD7AED06AD0852194D7C11
:10D8A000ED075219BD4C22600A7B1A404E7BF606EA
:10D8B000B60DB2188E7BF606760C9219CE7BF60664
:10D8C000360B92190E79F606F60992194E79F6067C
:10D8D000B608921962604A6AB14D2A40A2608A6A0B
:10D8E0002A40E2602D22D20087183A7E1A40039324
:10D8F0007E7EF606B60DB218BE7EF606760C92193E
:10D90000FE7EF606360B92193E7FF606F609921950
:10D910007E7FF606B60892190E7CF60792192261F0
:10D92000BA7F1A400597FE7FF606B60DB218049B23
:10D93000C35CDB065B0CD2184B78DB061B0BD218E2
:10D940008B78DB06DB09D218CB78DB069B08D21874
:10D950006261CA692A40A2610A6A2A40E2618A7C3D
:10D9600001252A40CB7CDB079B0F9A180B7DDB0738
:10D970005B0FD2184B7D9B07DB0ED2188B7DDB072C
:10D980009B0ED218CB7D1B079B0D9A180B7E1B0795
:10D990009B0CD2184B7E5B06DB0A13438A7E520631
:10D9A00012091A43CB7E5B075B0813432362CA6AE2
:10D9B00062620A6BA2624A6BE2628A6B226339225C
:10D9C000D200835C1E462E4066635E425E41B30415
:10D9D000AE04744F3C68B443E3183B6083185A7834
:10D9E0002A409C782407E40EA2188C8F6401A218A8
:10D9F0006D4C1440C98FC905490A0919DA78D20754
:10DA0000120A89181A791207120989185A79D20745
:10DA1000D2088918FB4EB1639968F163997904952E
:10DA20002940DA79D207920F51181A7B5207D20E89
:10DA300089185A7BD206920D51189A7B5207D20C44
:10DA40008918DA7BD206920B89181A7CD206520A00
:10DA500089185A7C520792090A43997CC9064908D9
:10DA600051183164D97C039A11401A7DD206920D67
:10DA700051185A7DD206520C89189A7DD206120B83
:10DA80008918DA7DD206D20989187164197E0F24AB
:10DA900021405A7E120151189A7E12038918DA7EAB
:10DAA0001207120A51181A7F1207120989185A7F91
:10DAB00012078918B164997F01942140DA7F120717
:10DAC000120E51183D22D200835C5B075B0D591882
:10DAD000841862781207520C8918A278D206120BA9
:10DAE0008918E278D206D2098918F16421790722CF
:10DAF0000A406179C9008918A2795206920B51181F
:10DB0000E2799207120B8918227AD2078A18BF4944
:10DB10000A60627AA37A1B029A18E37A1B04D2186D
:10DB20004A60E289BA4B13400394228AD2049209D4
:10DB3000D2188A6003463033598CB64A114002939A
:10DB40009A8CD205D20A51185622825C1206891884
:10DB5000B14D2960014656314A788C782402A218CA
:10DB60008C8864056409A218CC78240712196A60AD
:10DB7000CA880C7AA407A40BA2184C7A6407E40A9A
:10DB80001219AA604989E960492189004118FF22D8
:10DB90006632821800921035002207E00030004003
:10DBA000FFFFFF0004040040FF3F000084186427CB
:10DBB000E65D03273E406523E35C9B071B0F9B1933
:10DBC0006626A65DB607B60EF3186726A65DB601F3
:10DBD000F318DBB26826A65DB607B60DF318692602
:10DBE000A65DB607360DF3186A26A65DB607B60C15
:10DBF000F3186B26A65DB607360CF3186C26A65DE7
:10DC0000B607B60BF3186D26A65DB607360BF318EC
:10DC10006E26A65DB607B60AF3186F26A65DB60790
:10DC2000360AF3187026A65DB607B609F3187126F2
:10DC3000A65DB6073609F3187226A65DB607B608C4
:10DC4000F3187326A45DA407E31808C51032802AD0
:10DC5000ACD1019AD243704EB4180B783B404D784A
:10DC6000AD072D0FEB188D78AD07AD0EEB18CD7805
:10DC7000AD01EB18DBB20D79AD07AD0DEB184D79A9
:10DC8000AD072D0DEB188D79AD07AD0CEB18CD79E7
:10DC9000AD072D0CEB180D7AAD07AD0BEB184D7AD7
:10DCA000AD072D0BEB188D7AAD07AD0AEB18CD7AC9
:10DCB000AD072D0AEB180D7BAD07AD09EB184D7BB9
:10DCC000AD072D09EB188D7BAD07AD08EB18CD7BAB
:10DCD000AD07EB18A3641031121DBDD1009B19785C
:10DCE0005A785207520D51189A78D207120D891896
:10DCF000B164059B1968F164D97D5A681202511804
:10DD000031659968454A0A40998A490589187165BB
:10DD1000D9683D4C2140B16519692140F165029EE9
:10DD20003178049D294082785207120F5118C27928
:10DD30009207920E8918427A9207920D5118827AB0
:10DD40009207120D8918C27AD207920C89189A7D0F
:10DD5000D207520C891872789207D20B8918B278C0
:10DD60001207D20A8918F2781207D2098A182C49A8
:10DD70000A60327C737C1B071B0D9A18B37C9B06D0
:10DD80009B0BD218F37C1B079B0AD218337DDB0652
:10DD90005B09D218737DDB071B09D2184A60B27D7C
:10DDA0002A40C38F5B009A188A60826CCA60C26C7A
:10DDB00022400A61F27D7F231340328C5204520AC2
:10DDC000D2184A6102698A614269CA6182690A623B
:10DDD000C2694A62026A8A62426ACA62826A0A63E3
:10DDE000C26A4A63039A927CD201121D0A64027AC3
:10DDF0003A40CA65808F074A10400866002006B086
:10DE0000F0BDC04600300040FFFFFF009C300040E6
:10DE1000FF1F0000FF03000000400040FFFF1F0045
:10DE20000020004004480068806B800803490968AE
:10DE30004900401809307047449401021004004022
:10DE400010B52D21C9004118027A032A04D10079A6
:10DE5000002807D0082006E08378DA1E022A05D2BF
:10DE6000032412E0142088601C203DE0012B02D125
:10DE7000C8228A6012E00479042C01D3462404E00D
:10DE8000032C01D1322400E014248C605B1E022B91
:10DE900004D3022A10D24279154B01E04279154B86
:10DEA0009B181B78402B04D0102B06D1142344243C
:10DEB00005E02A233E2402E04279342348244B80A3
:10DEC0000C80022A06D0062A08D0052A08D118227A
:10DED0004C2301E0142250230B8000E01C224A80D6
:10DEE000C078042803D1142048806420088010BD25
:10DEF000C71F0100C01F0100134800687047C046DB
:10DF000010B5104A107091700F49002813D0506856
:10DF10000861042048619078FF2212020B4B1C68B4
:10DF20009443800380B20019186001204007084A1A
:10DF30001060084A106000200860074901220A604A
:10DF400010BDC04634940102180400401CE400E0F7
:10DF500080E200E000E100E070000040F0B591B028
:10DF6000002801D1C04800688778F91E022913D320
:10DF7000012F21D0022F3CD11021CA4344782146E1
:10DF8000193991423DD800970125B94A28462946BA
:10DF9000234601F0B5FF53E10821CA4344782146E6
:10DFA0002139914218D800970125B14A28462946BF
:10DFB000234601F0A5FF43E10821CA4344782146E6
:10DFC0000939914234D800970125A94A28462946A3
:10DFD000234601F095FF33E1032F3CD0042F43D1BA
:10DFE000C3780125042B00D02DE106462A02042324
:10DFF00043E00125A6A2284629463B4601F080FFC2
:10E000001EE1C3780125052B0AD806462A022846B8
:10E0100098401B21084230D10021052B08462ED004
:10E0200002200090914A2846294601F069FF07E145
:10E030000646C3780021022B1ED3032B1CD0042BD1
:10E0400008460A461BD001250095884A28462946DD
:10E0500001F056FFF4E0C3780125032B00D0FAE06D
:10E0600006462A02032308E0012583A22846294602
:10E070003B4601F045FFE3E00A46012148020F91CB
:10E08000592189007518FD21490071180291314606
:10E0900062313F05D219641E1F2727405C013C19DD
:10E0A0001443044332795207D20C22432B789B0647
:10E0B0005B0BD218B379DB071B0B13436D4D2B6041
:10E0C000F279032310931A40737A9B079B0E9A18D8
:10E0D000B37A5B07DB0D9A18F37ADB079B0DD21836
:10E0E000337BDB075B0DD218737B1B075B0CD218ED
:10E0F000AA603269EA6072692A61B2696A61F2698A
:10E10000AA61326AEA61726A2A62B26A6A620F9826
:10E110000870F06AA8623F20C4432C353046E430D2
:10E120000F903046E5300E903046E6300D90304688
:10E13000E7300C903046E8300B903046E9300A90DA
:10E140003046EA3009903046EB3008903046EC30EB
:10E1500007903046ED3006903046EE300590304660
:10E16000EF3004903046F03003903746F1373046B8
:10E17000F230F3360F990A194021525C109B1A4075
:10E180000E9B1B195B5C9B071B0F9A180D9B1B19A1
:10E190005B5C9B079B0E9A180C9B1B195B5C9B019D
:10E1A0009A18D2B20B9B1B195B5C9B079B0D9A18AC
:10E1B0000A9B1B195B5C9B071B0D9A18099B1B197B
:10E1C0005B5C9B079B0C9A18089B1B195B5C9B076D
:10E1D0001B0C9A18079B1B195B5C9B079B0B9A18DF
:10E1E000069B1B195B5C9B071B0B9A18059B1B1955
:10E1F0005B5C9B079B0A9A18049B1B195B5C9B0743
:10E200001B0A9A18039B1B195B5C9B079B099A18B6
:10E210003B195B5C9B071B099A1803195B5C9B0706
:10E220009B089A183319595C8907891802C510345C
:10E23000A0D102980078042101430E48C163002553
:10E24000284611B0F0BD04200090084A284629460F
:10E2500001F056FEF4E703200090044A28462946C0
:10E2600001F04EFEECE7C046449401029F3C0100E1
:10E27000E53C010000100040556E646566696E65FE
:10E2800064206D65616E205052462025640D0A00A1
:10E29000496E76616C6964206D65616E20505246EE
:10E2A0002025640D0A0000007047704780B50E49B4
:10E2B0000E480246083A1268920000D46031426863
:10E2C0000A4342600A490A6808239A430A60091F00
:10E2D000012252040A600321890402688A43026011
:10E2E000FBF732FA80BDC0462000008028000040C5
:10E2F00004020040B0B5032000072D490A6882439C
:10E30000012568071018086000242046FFF7CDFF9C
:10E310002046FFF7C9FFEFF31080284002D1EFF34A
:10E32000108172B68021C943224A53680B40536062
:10E3300093680B409360D3680B40D36013690B4024
:10E34000136153690B405361002800D162B6B0BD20
:10E3500070B50C4603210907154A13680B43136077
:10E360000122EFF31081114002D1EFF3108272B657
:10E370008025EA430F4B5E6816405E609E682E4320
:10E380009E60DD681540DD601D6915401D615D6999
:10E3900015405D61002900D162B6002802D001203D
:10E3A000FFF783FF002C02D00120FFF77DFF70BD37
:10E3B00000040040D89501020D4A002907D0012928
:10E3C0000BD10121814010688843106007E00121D2
:10E3D000814010680843106001E001218140101F56
:10E3E00002680A430121C907114301607047C04612
:10E3F00044000040032804D840000649085A00B2EF
:10E400007047002000B27047032802D84000014A3C
:10E410001152704706D301029E4908707047C046EA
:10E4200070B58AB00C460546FF20FC30A8490E683E
:10E43000315C59208000335CB278307808AE0696A3
:10E4400009AE05960C4E04962126760603960B4ED1
:10E450000296012601960E2600965B1CDBB2F7F7AA
:10E46000EDFB0998F2F79AFA28700898F2F796FAF5
:10E4700020700AB070BDC046000020410000044377
:10E48000F0B58BB00446457C82480078824900286C
:10E4900022D000200880814A1080814B01269E7680
:10E4A0001E830A907F4800787F4E36786DB20595BE
:10E4B0007E4D04957E4D03950AAD02957D4D0195E7
:10E4C0000096F7F7F9F80A9D112020567A497B4A01
:10E4D00000F022FC064626E000260E806F4A1680D9
:10E4E0006F4B01209876188309966E4800786E4F1E
:10E4F0003F786DB205956D4D04956D4D039509AD51
:10E5000002956C4D01950097F7F7D6F8099D1120FB
:10E5100021567F20C005009001900296664A674B05
:10E520003046F8F71DFA432001062846F1F76CFF44
:10E53000F2F734FA089062480078002824D051207D
:10E54000800060494A7D42438D185F480068A86496
:10E550002F46403750480078B87450480078F87417
:10E5600055480078387555480078787557480078D0
:10E57000F87550480069F2F711FAB87552484069C9
:10E58000E8644C4800686864FF20FE305049096820
:10E59000085C3922D2008918022812D303D04E48D1
:10E5A000007801280DD14B480660434800883A4A5C
:10E5B000108042480088394A108009200790089648
:10E5C00005E04448089A02603548C08B07900B78F4
:10E5D0000022002B01D0114600E0D1430125002B81
:10E5E00001D0042300E0EB43A67AAD1BEE175B19C4
:10E5F00071416568AE0F277AAD00ED195641677A13
:10E600003F1FF817ED1970414000EE0F80196D00A3
:10E61000EB1848418001990E4118980127239B026D
:10E62000C31A91411D4805881B480088854201D0C6
:10E630000798421B10202056C001194D2D8C032D28
:10E6400007D1E468E5176D0A6419E4150519EC179C
:10E650000FE0E468E5176D0A6519EC17ED15C617AC
:10E660004519744197B2002F00D03446002F00D0D6
:10E670000546581BA141130409D012B2D2015242DF
:10E68000D31780185941089BDA17C01A91410BB073
:10E69000F0BDC046C693010274AD010272AD010225
:10E6A0009C940102B5900102B490010260A30102A2
:10E6B0005CA1010278AD0102C2AD0102C0AD010250
:10E6C0002CA7010264A401026420004070AD010285
:10E6D000449401026CAD0102D0AD0102C10D4002B3
:10E6E000803070470120C0071B4908607047C04652
:10E6F00010B519480068C10710D1810711D441072E
:10E7000012D4010713D4C10614D4810615D44106CE
:10E7100016D48021084016D031A215E001240FA2A2
:10E7200013E0022411A210E0032414A20DE004243B
:10E7300016A20AE0052419A207E006241CA204E0A0
:10E74000072421A201E0254A04090220032101F047
:10E75000D7FB204610BDC0465C0000405265736583
:10E760007420627920504F520D0A00005265736583
:10E770007420627920424F520D0A00005265736581
:10E78000742062792050494E0D0A0000526573656D
:10E7900074206279205744540D0A00005265736555
:10E7A00074206279204C4F434B55500D0A000000F5
:10E7B0005265736574206279205357205265626FE9
:10E7C0006F740D0A00000000526573657420627951
:10E7D000205359535245510D0A0000004A2F0100A1
:10E7E000526573657420627920445644440D0A00D2
:10E7F00001218140044A1F2802D01068884310601C
:10E8000010680843106070471C000040F0B583B0EA
:10E81000029104469949F1F75DFC05469849019437
:10E820002046F1F757FC97494618974971430095E0
:10E830006F189649441864212046F1F74BFC3818AC
:10E84000A108471A92492046F1F75AFC3818914915
:10E850004518914F05D464213046F1F73BFC0C4636
:10E8600014E0A6B264213046F1F734FCB720400032
:10E87000A20701D1002907D1884B73430422D34159
:10E88000874A934200D3401E0C46451900984743DF
:10E8900002980680192001013046F1F71BFC2A4638
:10E8A0001F3A284600DB1046019BFF18B30705D12D
:10E8B000002C03D01F2D05DA0120C5E01F2D0BDA37
:10E8C0000120C1E005461D3D034600DB2B461C2808
:10E8D00008DC02201546B7E000290CD01C21451A9F
:10E8E0000CD50CE019461F39184600DB08461F2BD3
:10E8F0001DDA0320A8E01D21451A00D42846002D6A
:10E9000008D401461F39024600DB0A461F2804DAF4
:10E91000032099E00220154696E015461E3D10465C
:10E9200000DB28461E2A0CDA04200D468CE0054642
:10E930001E3D024600DB2A461E280BDA04200D4647
:10E9400082E001461F39024600DB0A461F280ADA28
:10E95000052079E011461F39104600DB08461F2AC2
:10E960000BDA052070E015461E3D104600DB2846F8
:10E970001E2A0CDA06200D4666E005461E3D0246BC
:10E9800000DB2A461E280BDA06200D465CE0014615
:10E990001F39024600DB0A461F280ADA072053E027
:10E9A00011461F39104600DB08461F2A0BDA0720E4
:10E9B0004AE015461F3D134600DB2B461F2A0CDAA2
:10E9C00008200D4640E005461F3D024600DB2A4672
:10E9D0001F280BDA08200D4636E019461E39184666
:10E9E00000DB08461E2B0ADA09202DE011461E39ED
:10E9F000104600DB08461E2A0BDA092024E01F28F7
:10EA0000054601DB05461F3D1F280CDA0A200D468E
:10EA10001AE01F28054601DB05461F3D1F2806DAC0
:10EA20000A200D4610E01E2D05DB0C2004E01E2DF3
:10EA300006DB0C2005E00B201E2D05DB1E3D03E050
:10EA40000B201E2D00DB1E3D029EB070681CF07076
:10EA5000E12001013846F1F73DFB3071C0B21149A8
:10EA60004143CC193C212046F1F734FB70713B2126
:10EA7000C94341430819B07103B0F0BD8051010092
:10EA80008033E101B207000093FEFFFFB1070000F1
:10EA900070FEFFFFA7FA0A0080AEFEFF295C8FC25E
:10EAA0000BD7A300F0F1FFFFF0B581B00446FFF7EC
:10EAB00021FCA08A00280ED0FFF71EFA2049086129
:10EAC00020482CCC2CC02CCC2CC02CCC2CC0002012
:10EAD000888101B0F0BDE08A194FB881A169BA8977
:10EAE0001948F1F747FB174D204629464CC84CC141
:10EAF0004CC84CC14CC84CC1FFF7FEF938616E6878
:10EB0000FFF790F9301AB8622846FFF7B9FC0646BD
:10EB10000D460E48007BFFF76DFC0121F970617C0A
:10EB20007971396C491C396481B2C90B401800B243
:10EB3000C1174010301A38658D417D6501B0F0BDB8
:10EB400068990102449A010210D30102B6900102B1
:10EB500070B50446FFF7CEFBA08A1B4E7082718A07
:10EB6000002908D0B0820220707100203082FFF7A7
:10EB7000C3F9F06170BDE08A3082A169328A13481E
:10EB8000F1F7F8FA2046FFF77BFC05460C461048E3
:10EB9000007BFFF72FFC81B2C90B401800B2C117F0
:10EBA0004010281A30668C417466FFF7A5F9B061F1
:10EBB000F06C401CF064FEF73FF9F063FAF78AFC52
:10EBC00030640120707170BDE8960102A8D3010283
:10EBD000C4900102F0B581B0EFF3108072B600204E
:10EBE0000146FBF791FE0446002803D062B620469A
:10EBF00001B0F0BD01273A030025074E28463146F3
:10EC0000FBF7DCFDBB021A4A28463146FCF7B4FA92
:10EC100062B6204601B0F0BD00E0020410B5F5F781
:10EC200010FE114CE078002801D0F9F773F9F9F7DC
:10EC3000E7F9F7F755FF0D490120C8720A7B034633
:10EC40009343CB71521C0A73094A928F002A08D051
:10EC50008A7A4B78134304D04A7A501C48720120B8
:10EC60009043607010BDC0461C900102B89801022C
:10EC70006AA9010270B514460D4606461120FAF73E
:10EC8000E1FE2248042101600C4804601E48056032
:10EC90008660002E0DD0FF20000609490A688243D5
:10ECA0000120C007101808600648082101600648C6
:10ECB00001601A200221FFF77FFB70BDA8D401027A
:10ECC00000E400E080E200E000E100E00C490860C0
:10ECD0007047C04610B504460948006860430949BA
:10ECE000F1F70EFA0019084948600848002202604E
:10ECF00002460C3A4B6813600968016010BDC046BB
:10ED0000A4D4010240420F000C9001022C100140DB
:10ED100000480047C100000080B582B013460A4693
:10ED200000900348011D0348F7F7C6FD02B080BDFF
:10ED3000E4D4010294A0010210B50C498A1C90424F
:10ED40000DD2401E0D4A50600D4803680B40032150
:10ED50008C071B19036000209060116010BD0448EF
:10ED60000449E622044B00F06FF8C046FFFFFF00A5
:10ED7000212F01003B2F0100072F010010E000E0D0
:10ED800020ED00E0B0B50120EFF31081014002D189
:10ED9000EFF3108272B6124A1368124C226864684C
:10EDA0008506114800682840850E5D192923DB007F
:10EDB0006B43002C1D4606D1002809D11E20684354
:10EDC00000290AD0B0BD121BD218551C0028F5D05E
:10EDD0001D461E2068430029F4D162B6B0BDC0466E
:10EDE00014E0010214E000E004ED00E080B5002032
:10EDF000FBF734F8404280BDB0B586B01048694694
:10EE00000A4638C838C238C838C200242046FBF742
:10EE10002BF803992046FBF7C1F80198012803D08D
:10EE20000824002804D102E00424002800D104466C
:10EE30000220FAF70FFEE0400249086006B0B0BDBC
:10EE4000CC1F010028E0010290B01C4605AB07C3AF
:10EE5000EFF31080C00702D1EFF3108072B6EFF32A
:10EE600010800B9068460E907046089010AB0F9380
:10EE7000CF4F3E1D01200490C50230462946224650
:10EE800000F0B8FC00213154EFF303800990EFF358
:10EE900008800C90EFF309800D90EFF314800A9036
:10EEA00000F02CFC3868012833D80028C14F00D06E
:10EEB000C14F2A20C1497A69920703D50A783A607E
:10EEC000401E491C0028F6D1B948041D2046F1F720
:10EED0007FF9002807D079698907FAD52178396048
:10EEE000401E641CF5E70220B5497A69920703D5F4
:10EEF0000A783A60401E491C0028F6D12A20AF4902
:10EF00007A69920703D50A783A60401E491C0028A6
:10EF1000F6D1FFF737FF0346AA4A30462946FDF7E8
:10EF2000BDFE04463018291B089F3B1F049A9343DB
:10EF3000A5A2FDF7B3FE9E490968012966D800190C
:10EF400000299C4C00D09C4C00280AD09849091DEF
:10EF50006269920703D50A782260401E491C002886
:10EF6000F6D10A209F496269920703D50A78226088
:10EF7000401E491C0028F6D10598F1F729F9002810
:10EF800009D061698907FAD5059A11782160401E78
:10EF9000521C0592F3E7022089496269920703D562
:10EFA0000A782260401E491C0028F6D10A208EA152
:10EFB0006269920703D50A782260401E491C002826
:10EFC000F6D10698F1F704F9002809D0616989079C
:10EFD000FAD5069A11782160401E521C0692F3E77A
:10EFE000022077496269920703D50A782260401EA1
:10EFF000491C0028F6D10A207EA16269920703D538
:10F000000A782260401E491C0028F6D17CA23046B6
:10F010002946079BFDF742FE6549096801290E9BB9
:10F020001BD80029634900D0634900280AD0604AF0
:10F03000121D4C69A40703D514780C60401E521CA5
:10F040000028F6D102205E4A4C69A40703D5147843
:10F050000C60401E521C0028F6D16AA23046294698
:10F06000FDF71CFE04463018291B694A3B46FDF794
:10F0700015FE4F490968012911D8001900294D4989
:10F0800000D04D4900280AD0494A121D4B699B0700
:10F0900003D513780B60401E521C0028F6D15D4A40
:10F0A00030462946099F3B46FDF7F8FD0446F80027
:10F0B000C00FB900C90F7A00D20F009201910290DF
:10F0C0003019291BFB0F544AFDF7E8FD04193019CC
:10F0D000291B3F233B40514AFDF7E0FD34490968B5
:10F0E000012911D820180029324900D032490028BE
:10F0F0000AD02F4A121D4B699B0703D513780B606A
:10F10000401E521C0028F6D1454A304629460B9B2A
:10F11000FDF7C4FD04463018291B424A0A9BFDF73F
:10F12000BDFD23490968012911D800190029214989
:10F1300000D0214900280AD01D4A121D4B699B07A7
:10F1400003D513780B60401E521C0028F6D1364AB6
:10F15000304629460C9BFDF7A1FD04463018291BBB
:10F16000324A0D9BFDF79AFD114909680129114AA0
:10F170000DD80019002908D00F4A06E05169890707
:10F1800003D531781160401E761C0028F6D128493D
:10F190000E98091AA94200D32946890800F03AFEC0
:10F1A00024480068002800D0804700F045F8C04699
:10F1B000F8E001020090014000A001407B2F010017
:10F1C000093D0100642F01000D0A23232320415330
:10F1D000534552542040203078253038582023237E
:10F1E000230D0A003E30010046554E4354494F4E10
:10F1F0003A2000004C494E45202020203A200000B3
:10F20000256400000D0A53503D253038580D0A0082
:10F210000330010019300100253001000D300100DC
:10F22000C22F0100D12F0100E02F0100EB2F0100C0
:10F2300000F80202F4E00102F7480068012811D842
:10F24000002801D00B4800E0FC480C210A4A01E0EC
:10F25000002907D043699B07FAD513780360491E3C
:10F26000521CF5E71E20FFF7C3FA00BF00BF00BF26
:10F2700000BFFAE700A001406E2F01008AB00646E9
:10F28000E448B06600F03AFAFFF77CFD0346E24836
:10F29000041D01200590C502E04A20462946FDF7DD
:10F2A000FDFC074608942018DB4C0995E91BF36C1C
:10F2B0003F2206921340DAA2FDF7F0FC21680129F3
:10F2C00010D8C0190029DD4900D0DD49002809D037
:10F2D000221D4B699B0703D513780B60401E521CFF
:10F2E0000028F6D1F36BD7A2089C2046099D294639
:10F2F000FDF7D4FC0746291A2018336C069A1340F0
:10F3000007D1D8A2FDF7CAFCC34C2168012907D94F
:10F3100017E0CEA2FDF7C2FCBF4C2168012910D82E
:10F32000C0190029C54900D0C549002809D0221DAF
:10F330004B699B0703D513780B60401E521C0028B5
:10F34000F6D10027CBA5B80030580090089809994D
:10F350002A463B46FDF7A2FC216801290FD8002967
:10F36000B64900D0B649002809D0221D4B699B0739
:10F3700003D513780B60401E521C0028F6D17F1C69
:10F380000D2FE0D1736BBFA2089C2046099D294632
:10F39000FDF784FC074620189F4CE91BB36BBC4A61
:10F3A000FDF77CFC2168012910D8C0190029A34968
:10F3B00000D0A349002809D0221D4B699B0703D523
:10F3C00013780B60401E521C0028F6D1336CB14AF2
:10F3D000089C2046099D2946FDF760FC0746326CD3
:10F3E000D000C00F9100C90F5300DB0F00930191B3
:10F3F0000290E019E91BD30FA74AFDF74FFC3246F4
:10F40000C619A019A91B1546136C069A1340A34AE6
:10F41000FDF744FC80490968012911D880190029A9
:10F42000864900D0864900280AD07B4A121D4B69C4
:10F430009B0703D513780B60401E521C0028F6D1A1
:10F440002E466B6C964A089C2046099D2946FDF77E
:10F4500025FC07462018E91B0796B36C914AFDF777
:10F460001DFC6D4A1168012910D8C0190029734983
:10F4700000D07349002809D0121D4B699B0703D5A2
:10F4800013780B60401E521C0028F6D10798426E7C
:10F49000042360215C2004931A400B4600D00346ED
:10F4A0000693002A00D00846079E33587E4A089CDF
:10F4B0002046099D2946FDF7F1FB0746069833587B
:10F4C000E019E91B794AFDF7E9FBC619A019A91B48
:10F4D000079A536E76A2FDF7E1FB4F4909680229AE
:10F4E00011D280190029554900D0554900280AD069
:10F4F000494A121D4B699B0703D513780B60401EC8
:10F50000521C0028F6D10798C36C06466DA2089CD1
:10F510002046099D2946FDF7C1FB07462018E91B37
:10F52000336D6B4AFDF7BAFBC619A019A91B079FDB
:10F530007B6D68A2FDF7B2FB8619A019A91BBB6DF4
:10F5400067A2FDF7ABFB344909680129059C11D876
:10F5500080190029394900D0394900280AD02E4A9B
:10F56000121D4B699B0703D513780B60401E521C7C
:10F570000028F6D10798476B5D4A974237D203209F
:10F5800087430026059CB00039580246049B1A4365
:10F59000BA5808230343FB580C2505437D590091B5
:10F5A0000192029303953B1808980999514AFDF777
:10F5B00075FB1949096801290FD800291F4900D096
:10F5C0001F49002809D0089A4B699B0703D5137877
:10F5D0000B60401E521C0028F6D11B2E444A06D850
:10F5E0000798406B361DB10040189042CBD3079866
:10F5F000406B111A099A914201D8890800E0610212
:10F6000000F008FC3C480068002800D08047FFF765
:10F6100013FEC04622224B4DF8E00102642F010088
:10F620000D0A0D0A23232320455843455054494FC2
:10F630004E202564202323230D0A00000090014062
:10F6400000A0014050433D25303858002C2045781B
:10F6500063657074696F6E4E756D6265723D256489
:10F660000D0A00002C205468726561644D6F64655A
:10F670000D0A000052252D32643D253038580D0A00
:10F680000000000053503D253038580D0A0000009E
:10F690000330010019300100253001000D30010058
:10F6A000C22F0100D12F0100E02F0100EB2F01003C
:10F6B0004558435F52455455524E3D253038580DFC
:10F6C0000A000000494353523D253038580D0A00C6
:10F6D000F62F01005343523D253038580D0A0000E3
:10F6E0004343523D253038580D0A0D0A00000000F2
:10F6F00000F80202A62F0100F4E00102F0B583B089
:10F70000344D2C68012C06D8601E8441204601F03F
:10F7100073FB0028FAD10120EFF310810140019121
:10F7200002D1EFF3108072B62B48285A2B49695A40
:10F73000814245D02A68002A01D02A4E00E0284E96
:10F740001F23DB020293284C022A27D205E0104631
:10F75000214AA85282B2914232D087B2B9420A46B7
:10F7600000D8621C131A21482B5218040DD0E81936
:10F77000001D9FB201E0002F07D073699B07FAD5E7
:10F78000037833607F1E401CF5E7A242DFD9029860
:10F790001018DDE7304683B299420CD0024680B2A1
:10F7A00081420E4600D8661CA642F3D90298301852
:10F7B00083B29942F2D108496852B01A0B49685293
:10F7C0000B48002129540198002800D162B603B0EB
:10F7D000F0BDC046F8E001020A0800000808000079
:10F7E0000090014000A00140FF0700000C0800004D
:10F7F0000F080000F0B58DB00793174600240C9455
:10F8000009AA13C215E006986849F0F7FDFDF1F763
:10F81000C5F8C117401848406549F0F75BFC0095F2
:10F8200009A806223346F9F7C9FABDE0002C00D535
:10F83000BEE138787F1C25280DD0002800D1B7E123
:10F840000B9A511C0A9B9942F0D8099B9854641C4E
:10F850000C940B91EAE708940025397823390D2997
:10F8600014D801207944097949008F44090F0F0FFA
:10F870000F0F0F0F0B0F060F0F0D05437F1CECE74B
:10F880000820FAE70420F8E70220F6E73878014676
:10F8900030390024092902D9264639460BE00026D2
:10F8A0000A2171430E18303E791C78780246303AAE
:10F8B0000A2A0F46F4D32E2817D14A1C487801464D
:10F8C0003039092905D911464F1C2538532811D93B
:10F8D0006AE000240A2161430C18303C511C507826
:10F8E0000246303A0A2A0A46F4D34F1C25385328D8
:10F8F00000D959E04000C0467844808840008744E1
:10F90000A000530053005300530053005300530012
:10F91000530053005300530053005300530053004F
:10F92000530053005300530053005300530053003F
:10F93000530053005300530053005300530053002F
:10F940005300600053005300530053005300530012
:10F95000530053005300530053005300530053000F
:10F9600053005300530098005300530053005300BA
:10F97000530053005300530053005300AD00B60032
:10F9800053006000530059005300530053005900C6
:10F99000530053005300DE0053005300BD005300DA
:10F9A000D3005300530098000C9C3FE70024744997
:10F9B00040420F00791C38780F4625385328F3D879
:10F9C00098E70799C91D072081430868079149688E
:10F9D000F1F772F800210690F0F740FF00280BD1F4
:10F9E0000B99481C0A9A904206D8099A2D23535421
:10F9F0000899491C0C910B900798083007900698BD
:10FA0000F0F7CCFF0095C2178118514009A8224693
:10FA10003346F9F7D3F90B98411C0A9A914200D961
:10FA2000F1E6099A2E2313540B910C98401C0C906C
:10FA3000E9E6079802C807900096019509A81022E8
:10FA400039E00B98411C0A9A9142ADD8099A2523B6
:10FA500013540B910C98401C0C90A5E70B9A511C69
:10FA6000079C201D0A9B994239D907909CE707986B
:10FA700002C80790009509A82246D3E6079901C954
:10FA8000079109990A9A089E02E0401C002E8BD427
:10FA90000378002B88D00B9D6C1C9442F5D84B55F5
:10FAA000761C0C960B94F0E7079802C80790009616
:10FAB000019509A80A222346F9F71EFA74E7079B65
:10FAC00010CB102C079308D300202146401C0A09B4
:10FAD000FF291146FAD806280AD8082009E0236829
:10FAE000099CA354089A521C0C920B9107905BE757
:10FAF000401C069009230C980B9D099905910A9EBC
:10FB000004940DE0202104463046059E71550646BA
:10FB10002046049C401C15460146089100290AD441
:10FB20005B1E0699994206D26A1CB242EAD908992C
:10FB300008910029F4D50C900B950898002800D561
:10FB400032E70126082501E06D1E3601022DFBD2A9
:10FB500020463146F0F7BEFA0F28F6D80C980590EB
:10FB6000099803900A9806900B9D20463146F0F7BD
:10FB7000B1FA691C069A914204D9089908910029A2
:10FB80000CD511E00C4A125C039B5A55089A521C82
:10FB90000D46059211460891002905D47043241A98
:10FBA0003009102E0646E0D205980C900B95FBE626
:10FBB00020460DB0F0BDC046C022010070B588B02F
:10FBC0000022032803D9D243104608B070BD7F4CF1
:10FBD000C34D2A510F4B104EEE5081231E010123BD
:10FBE000AB5528602C1962600128EDD807930022DC
:10FBF00006920592049203230393029201920091CC
:10FC0000411E8841694600F027FD0246104608B0B3
:10FC100070BDC04604080000FFC0FFC0F0B583B04F
:10FC20000C460023D943012C56DB074602910126DE
:10FC3000EFF31085354002D1EFF3108072B65849CA
:10FC4000584A505C002800D0A3E056545E48115A30
:10FC50005E48105A0196F202161A814240D8324686
:10FC60005218A24240DB00930295A642354600DBC3
:10FC700025464C490818001D39462A46F0F77AFAFD
:10FC8000A642484E04DA7919621B301DF0F772FA69
:10FC90004E48305A001981B24D4A914201D94D491E
:10FCA0004018029D009B4949705230464A4E805D83
:10FCB000002865D1EFF310850198054002D1EFF3DC
:10FCC000108072B6374A4048115A4048105A88424C
:10FCD00032D1424813524FE00C46204603B0F0BDEB
:10FCE00042425218A242BEDA3B4A2E4EB25C002A71
:10FCF0000CD03A4AB25A51188AB2354CA242284C1A
:10FD0000029F01D9334A8918304A02E0244C2F4A15
:10FD1000029F3355B152421A89B2884202D22C480E
:10FD20008018421C93B22F4801212FA200F0E8F85E
:10FD30003C46002DD1D128E0019F9755884201D83B
:10FD40002348401C421A90B2800A01D001988202D6
:10FD50002248144F3A52386801280DD8431E984162
:10FD6000104B5918091D92B21D4B00F08BFE009BE1
:10FD7000002801D00B488355002D029D00D162B6AA
:10FD8000074808490B54002DA7D162B6204603B09E
:10FD9000F0BD21200201044804A108A3FFF754F894
:10FDA0000E080000F8E00102BA30010074726163CD
:10FDB000655F6F75747075740000000054524143A4
:10FDC00045204255535900000A0800000808000069
:10FDD000FF07000000F8FFFF0F0800000C080000FC
:10FDE0002D00010002FF00000D0A547261636520BE
:10FDF0006275666665722069732066756C6C2C206E
:10FE00006469736361726473202575206279746517
:10FE1000730D0A00F0B587B00546002606960596D4
:10FE2000049603960296800701D007B0F0BD0191B9
:10FE300002A8142126A2FCF731FF294909680129EB
:10FE400011D80029274900D0274900280BD002AA41
:10FE500001E0002807D04B699B07FAD513780B60A7
:10FE6000401E521CF5E701990029DED0204C374690
:10FE7000B8002B58D80724D0581EA04204D31B48E2
:10FE800018181C4A90421CD802A814211AA2FCF788
:10FE900005FF13490968012911D80029114900D02B
:10FEA000114900280BD002AA01E0002807D04B69B5
:10FEB0009B07FAD513780B60401E521CF5E7761CA1
:10FEC00001997F1C8F42B0D2322ED1D3ADE7C0460C
:10FED0000D0A4261636B74726163653A200D0A001A
:10FEE000F8E001020090014000A00140FFFFFFFC8C
:10FEF000FFFF0200FEFF0100253038580D0A000008
:10FF000081B0F0B5C4B00E46074649938120000188
:10FF10002F49085C002845D002920120050204A860
:10FF20002946F0F740F9FCB20021C8430C2C3AD81E
:10FF3000721E032A37D82748005DB042084632D3E4
:10FF4000F80535D50021B8050DD404A80190401856
:10FF5000691AA20022A39B582E4AFCF79FFE019823
:10FF6000F0F736F9014678050ED404AF7818691A0F
:10FF7000B20029A3D218121F1368264AFCF78EFE7E
:10FF80003846F0F725F90146029A04AE70180C467F
:10FF9000691A49AB0393FFF72DFC01193046FFF7AF
:10FFA0003DFE00E0002044B0F0BC02BC01B00847B8
:10FFB000FEF7E8FE034604A8019007A22946FCF7D5
:10FFC0006DFE0198F0F704F90146B805BDD5CAE702
:10FFD000F8E00102EC48010025313075207C20005A
:10FFE0005E300100B4300100AE3001008D30010000
:10FFF0005830010079300100A7300100A030010025
:020000040001F9
:100000009B30010051300100643001007430010068
:10001000493001006D390100933001007F3001004B
:10002000863001006A30010000000000F0B581B0A8
:100030000B460120EFF31084044002D1EFF310814E
:1000400072B6990F07D0022001212DA2FFF758FFA9
:10005000002C3DD141E02249224D00276F54224A15
:10006000AB5A224AAE5AF3189EB2F60A01D0204E7D
:100070009B19AB52EFF31086064002D1EFF31083C9
:1000800072B6AA5A1C4BEB5A934202D116482F5211
:100090001AE06854934201D8164B5B1C9B1A99B224
:1000A000890A00D0830210482B52286801280BD8F7
:1000B000411E8841A918091D9AB2104B00F0E2FCBC
:1000C000002801D006482F54002E03D0002C04D065
:1000D00001B0F0BD62B6002CFAD162B601B0F0BD3D
:1000E0000F080000F8E001020C0800000A080000F8
:1000F00000F8FFFFFF070000080800002D000100C6
:1001000055415254204572726F722025780D0A00B5
:1001100010B50446FEF7EEF8A08A002800D010BD06
:10012000FDF7EAFE034908620861486C401C486418
:1001300010BDC0466899010210B50446FEF7DAF812
:10014000A08A002800D010BD0A4CA06C401CA064FE
:10015000FDF7D2FE6062606C002805D0FDF7CCFE92
:1001600060650020606410BDA069206501206064A6
:1001700010BDC046E896010210B50A2000242146B1
:10018000FBF7D4FC09202146FBF7D0FC01242046D4
:1001900000F038F80E200421FBF7C8FC0549204682
:1001A00000F05AFAA2021549154B204600F028FB30
:1001B00010BDC046DC940102B0B50E2000242146DB
:1001C000FBF7B4FC0D202146FBF7B0FC01242046D0
:1001D00000F018F80A2004252946FBF7A7FC09209F
:1001E0002946FBF7A3FC2046F9F77AFAA202034955
:1001F000034B204600F004FBB0BDC04618CE010200
:10020000390A010070B5012801D9012070BD4822CA
:100210004243734B9C58A5691F218D43A561062558
:10022000A5600F2525629C18A27C002A05D1627C5E
:10023000002A02D1227C002A14D06368002B11D43A
:10024000251D0B40012216469E400C4B1E60BFF33D
:100250004F8FBFF36F8F2B68002B03D40B409A4056
:1002600007490A60002803D0012804D1092000E0D2
:100270000820F9F7DFFB0020A06170BD80E100E0FD
:1002800080E200E0F0B585B00D460278E348C3682F
:10029000934219D0446D944216D08368934203D0A0
:1002A000016D914200D07FE09B1A591E8B4104934F
:1002B00048215943032D46D14418E16900294ED005
:1002C0001C34002020606DE09B1A5A1E9341049359
:1002D000032D1AD1039548225A438418A26B012199
:1002E000EFF310850D4002D1EFF3108772B6A769C6
:1002F0001026B743A761A669002E01D118342160EA
:10030000002D00D162B6039D0CE0482159434218EC
:1003100091691832302902D0116810294CD18021FE
:100320001160002248215943401800218163016275
:100330008162243000210160002A33D004A82946BC
:10034000904705B0F0BD421891691832302902D0AB
:100350001168202939D180211160002216E003950F
:10036000E26B0126EFF31085354002D1EFF31081E7
:1003700072B6A1692027B943A161A169002901D101
:1003800018342660002D00D162B6039D48215943E0
:1003900040180021C163C162416330300021016017
:1003A000002ACBD105B0F0BD00920E4A2E329C48F7
:1003B0000D490E4BFEF748FD1068009301909848D8
:1003C0000949084A0A4BFEF73FFD10680093019067
:1003D000044A243292480449054BFEF735FDC046D5
:1003E000FC940102B1020000363101000B31010022
:1003F000EF300100F0B585B0049048210A46424331
:10040000864B9C58E6690F2535409A18167C002EBD
:1004100031D04F2040026169014200D185E0A069DE
:1004200004218843A061022020620120810769180D
:10043000D161D36BEFF31084044002D1EFF3108548
:1004400072B695692026B54395619569002D00D156
:1004500073E010463C30002C00D162B600240460EA
:10046000D4625463303200201060002B63D004A8A3
:10047000984705B0F0BD0C2D5DD8C0467D442D7960
:100480006D00AF4467586B580658A16358585858C8
:1004900006009569202D04D0154618352D68302D9D
:1004A00049D1156B566B3432AE4217D266693607A6
:1004B00014D5646815686E1C166048431818C06A25
:1004C000445504980C4644431A19156B566B343244
:1004D000AE4203D21C5966693607EAD41268AA42B2
:1004E00029D14143585882690524A24382615A1890
:1004F000D36B0121EFF31080084002D1EFF3108499
:1005000072B694692025AC4394619469002C02D1A1
:1005100014461834216014463C34002800D162B6D9
:1005200000212160D16251639CE70C2D00D176E758
:10053000012D00D173E705B0F0BD154618352860D0
:1005400010463C30002C00D187E787E7042020626A
:1005500005B0F0BD0120206205B0F0BD0825256280
:10056000164618369569102D02D03568302D4BD1BE
:100570000396566A15462835976AB74228D1A0696E
:1005800002218843A061936B0121EFF310800840A2
:1005900002D1EFF3108472B6039E34681027BC4377
:1005A00034603468002C00D131601446383400289F
:1005B00000D162B60021216029601162243200203E
:1005C0001060002BB7D052E70220206205B0F0BDCA
:1005D0002A68B242AFD262699207ACD52A68561C2B
:1005E0002E6048431818006A805C206004980A4610
:1005F00042439D18AC6A6E6AB4429CD228359C581E
:1006000062699207EAD496E7316800900191044844
:1006100004A1094A09A3FEF717FCC046FC94010295
:10062000D5300100756172745F6972715F68616EC7
:10063000646C6572000000003D0300005561727437
:1006400020256420737461746520676F657320775B
:10065000726F6E6720256400F0B585B00E460546C2
:10066000022804D3002E02D1012005B0F0BD002DD8
:1006700003D0012D08D1092400E008242046F9F711
:10068000E1F92046FEF7B4F848216943E74A50589B
:1006900083691F240294A3438361062383600F238D
:1006A0000193036257180023BB62BB63FB633B6289
:1006B0007B62FB623B63317F3974727F7A74B27FF5
:1006C000BA7404937B637368B268F468920022433F
:1006D0005B1E032B0ED8C0467B441B795B009F44F6
:1006E00001050307082304E0282302E0182300E0A3
:1006F00038231A43C260C907090F72699201D2B246
:100700008918B2699207920E8918491C8160796133
:100710003169012901D122210161012D5CD83168A3
:100720000E2959D23846123003900324002D01D0EF
:10073000204600E004204C432D490E19B178F9F70A
:1007400011FA3968CA68802510462843C8602848CD
:10075000005D73781B021818C862AA43CA60F9F7D3
:1007600049FA03980078002809D1384611300078FA
:10077000002804D1384610300078002827D0786847
:10078000002815D4032102468A431B495358840785
:10079000E40EFF26A640B343A5401D4355500299E1
:1007A000014001208840A2490860144908600EE019
:1007B0008107C90EFF228A40019C0440083C0320A7
:1007C00084430C48235893438D401D4325500120FA
:1007D000B861049805B0F0BD02480349DA22034B22
:1007E000FEF732FBD5300100483101002531010010
:1007F000542001001CED00E000E400E000E100E016
:10080000F0B58FB00E900125002900D14BE0039385
:1008100004910592002A00D145E00121EFF31082F6
:1008200001910A4002D1EFF3108172B64827029776
:1008300047437E49CE19B5690023302D23D8314670
:100840001831C0467D442D796D00AF442024262602
:100850002626262626262626262626265E26262600
:100860002626262626262626262626261826262636
:100870002626262626262626262626261800022373
:10088000002A0CD00CE0402D01D0802D05D1012391
:10089000002A04D004E020240C60002A00D162B6B3
:1008A0001D46002B02D028460FB0F0BD0025756311
:1008B0000399F1630499F162059931635B4CE35943
:1008C00059691322D202114205D0062199600F21E5
:1008D000196271699960317C00290CD0F561099524
:1008E0000895079506950D950B9502210A9101280B
:1008F00010D017200FE0717C9A6900292CD0952028
:1009000002439A6128460FB0F0BD30240C60002AE3
:10091000C5D0C5E71920049F0C907068002805D445
:100920001F210840019981404148016014209861CD
:10093000B06806A9F9F7CEF90E98029941436018FC
:10094000806861583B4A0092091D3A46059BF9F7B9
:1009500031FA28460FB0F0BD3436110602D5802199
:100960008A439A6131680025059A91422DD20595F6
:100970005D694F214A0215421BD1E90502D4029C50
:10098000F24F0AE0596833685C1C3460029C604393
:10099000EE4F3818C06AC1540E98214641437E1864
:1009A000736B346BA34238D234367B585D69154281
:1009B000E3D002211962019EB10729433546E34C79
:1009C000EFF31082324006D008E02946019EEFF393
:1009D0001082324002D1EFF3108372B6029B434380
:1009E000E01883692024A34383618369002B05D029
:1009F000002A08D0C26B002A0AD154E703461833F4
:100A00001E60002AF6D162B6C26B002A00D14AE706
:100A10000EA8904728460FB0F0BD2946059D019EBF
:100A20003C46EFF310823240D5D0D7E7FC94010268
:100A300080E200E08502010080B5012082020249C7
:100A4000024BFFF7DDFE80BD18CE0102390A01001E
:100A5000B0B582B079208400E54D285D01A9087009
:100A6000652080002818F2F7C1FF2F20C000285809
:100A700029190122024BFFF7C3FE02B0B0BDC046E8
:100A8000510A0100F0B591B010900126002900D163
:100A90009BE003930591002A00D196E00790012185
:100AA000EFF310800291084002D1EFF3108172B68B
:100AB00004924823069307994B43D649C9188D6978
:100AC0000026302D6ED80C461834AD00374602A6ED
:100AD00075593E46AF46C046AD0B0100B50B01004F
:100AE000B90B0100B90B0100B90B0100B90B0100F2
:100AF000B90B0100B90B0100B90B0100B90B0100E2
:100B0000B90B0100B90B0100B90B0100B90B0100D1
:100B1000B90B0100B90B01009D0B0100B90B0100DD
:100B2000B90B0100B90B0100B90B0100B90B0100B1
:100B3000B90B0100B90B0100B90B0100B90B0100A1
:100B4000B90B0100B90B0100B90B0100B90B010091
:100B5000B90B0100B90B01004B0C0100B90B0100EE
:100B6000B90B0100B90B0100B90B0100B90B010071
:100B7000B90B0100B90B0100B90B0100B90B010061
:100B8000B90B0100B90B0100B90B0100B90B010051
:100B9000B90B0100B90B01009D0B010002260028D2
:100BA0000CD00CE0402D01D0802D05D1012600286D
:100BB00004D004E010252560002800D162B6002E84
:100BC000069D944F049C079802D0304611B0F0BDAA
:100BD00000268E62039A8A63059A0A624C620A7C36
:100BE000002A0BD00C960B960A96099608960E963C
:100BF00002220D9201282DD018202CE08A7C283169
:100C0000002A3BD00A68A24216D22B464343FA5828
:100C10005469A40710D50868441C0C60F918096AC7
:100C2000085C10601098294641437A181146283113
:100C3000936A526A9342E8D3454378598169822284
:100C40000A438261304611B0F0BD3025256000288E
:100C5000B4D0B4E71A200F90C86808A9F9F73AF899
:100C6000109845437A597819C06839490091059917
:100C70002346F9F79FF8304611B0F0BDFB589A694A
:100C8000140602D58024A2439A610A6800260498BB
:100C900082422ED25D694F225202154207980AD035
:100CA00002211962029EB10729431FE028315D69C4
:100CB00015423E46F4D137465C69A40702D4069932
:100CC000544E0AE00C68661C0E6006994843514E6B
:100CD0003018006A005D186010984143735871180D
:100CE0008C6A4E6AB442E1D329463E46069D494F7E
:100CF00001E0314607985A6A002AFCD1EFF31082CE
:100D0000029B1A4002D1EFF3108372B64543781963
:100D100083691024A34383618369002B05D0002AD3
:100D200009D0826B002A0BD14FE703461833029C8F
:100D30001C60002AF5D162B6826B002A00D144E71C
:100D400010A89047304611B0F0BDC046FC94010297
:100D500085020100B0B5264900684A68824202D186
:100D60000D1D002016E080228A58824203D10D46D4
:100D7000803501200EE0FC228A58824203D10D46C4
:100D8000FC35022006E02F22D2008B5883422ED160
:100D90008D1803207C2242438C18A068012814D0AF
:100DA000002824D140342046F3F70FFA01462046AC
:100DB000F3F7E1F92046F3F708FA002817D006C840
:100DC00028680C4BFFF75EFEB0BD40342046F3F7B9
:100DD000FCF901462046F3F7CEF92046F3F7F5F982
:100DE000002804D006C82868024BFFF74BFEB0BDB0
:100DF00090BE0102550D01004821414305484218AB
:100E00009269D20601D40020704740584169012000
:100E100008407047FC94010280B511480078C00179
:100E200010490978890101430F48007840010843BF
:100E30000E490978090101430D480078C0000843B4
:100E40000C490978890001430B48007840000843A9
:100E50000A4909780143C8B2F3F768FC80BDC0466F
:100E6000189F0102E69601021D9001029CEA010210
:100E7000D1AD0102199F01025CA301025DA3010231
:100E8000F0B587B001460127022505283A4600D073
:100E90002A4600200929014600D01146C900374AD8
:100EA00054180E210591615EFDF7AEFA1026A15F80
:100EB0003846FDF7A9FA1227E15F2846FDF7A4FAA4
:100EC00006951425615F03200490FDF79DFA0598AF
:100ED000235EA05FE15F625F00AD07C528A2069FA9
:100EE0003846049D2946FFF70BF820462630042695
:100EF0003146FBF749FF2620235E2820205E2A2169
:100F0000615E2C22A25E00900191029224A23846DA
:100F10002946FEF7F5FF27463E3738463146FBF7B0
:100F200051FF3E20235E06983C5EB95F0622BA5E02
:100F300000940191029221A207462E462946FEF70F
:100F4000DFFF56240D4D285FFBF730FF2B5F2C464B
:100F500021A2384631463546FEF7D2FF264658369E
:100F60003046FBF70FFF5820235EF05F00901FA272
:100F700038462946FEF7C4FF07B0F0BDFCA00102C9
:100F8000546F4620616E742064656C61797320250E
:100F9000642025642025642025640D0A00000000DB
:100FA00050446F412064656C61797320256420256D
:100FB000642025642025640D0A00000050446F4120
:100FC000206761696E7320256420256420256420D4
:100FD00025640D0A0000000050446F4120616E74CA
:100FE0002073706163652025640D0A0050446F41D1
:100FF00020616E676C65206F66667365747320256B
:10100000642025640D0A0000F0B587B015467A4BC0
:101010001A680F24A2432F783A431A60774C23466C
:101020002C3B774A1A60049003462246283A1268FD
:101030001207FAD5734E092F029306D9754A32600A
:1010400072600C2F09D175480FE0042F07D9704A40
:101050003260704A7260092F06D3714805E06A4811
:1010600030607060694800E06B486E4A1060EB7A4F
:10107000FF2B039102D10020B0620AE003210B4054
:101080006948C05C40220243B2620220674AFEF710
:1010900037FF029F0021384605952A460B46FBF78D
:1010A000FDFE06460225032161A228460191334632
:1010B000FEF726FF06963046FCF7C4FB0121049894
:1010C000009108402CD13D4033D1604900283AD1ED
:1010D000002D1ED06548A062E06220636063644812
:1010E000606264480860152085046E1C8E608D6007
:1010F000642420460F46F8F77DFD3E603D602046A3
:10110000F8F778FD281D386003215BA24E48FEF7F2
:10111000F7FE0598007BFAF7CFFF069807B0F0BD01
:101120002E4605460698FCF719FF284635463D40F1
:10113000CBD02E4605460698FCF78CFB2846354654
:1011400042490028C4D042480861424848614248A8
:1011500088611520C8614148016840220A43026045
:1011600007210803274B5A6982430098400310184F
:1011700058610522039842432A4803689818334E61
:10118000766B47780F40995C0907490EC919CA0365
:10119000334B33409A18C9015118324A89182B4AE7
:1011A00051632A49896B3822914382785207920E03
:1011B000891804220A4325498A63124B1969027966
:1011C000019E3240C0784007C00E80181F22914314
:1011D0000818186155204003411C216020606420DC
:1011E000F8F708FD204A18483146039BFEF788FEB1
:1011F0001649002D8DD06DE7040400402C6000409E
:1012000000040080000600400F040F04DD2A0100E6
:1012100003040304000400040E2C0100AC290100A7
:101220003F2D010048940102702E0100743101002D
:1012300050485920706172616D732073657473201A
:10124000253038780D0A0000020800009060004048
:1012500012A83E009DD79B5AD579BD493402004063
:101260003F0080FF4040000056310100200882000E
:1012700002D50F00020255007577625F72785F69D0
:101280006E69740D0A00000080B5224800210170CB
:1012900022480078C001204909788901014320488B
:1012A0000078400108431F490978C90001431E48DE
:1012B0000078800008431D490978490001431C4813
:1012C00000780843C0B2F3F731FA80BD80B5114809
:1012D0000121017010480078800110490978C90186
:1012E00001430F480078400108430E490978C900BE
:1012F00001430D480078800008430C4909784900F3
:1013000001430B480078084310210143C8B2F3F7AA
:101310000DFA80BD9CEA0102E6960102189F0102C7
:101320001D900102D1AD0102199F01025CA30102CF
:101330005DA30102F0B581B01820FDF759FA19201C
:10134000FDF756FA002420462146F8F727F82046F4
:101350002146FAF735FE012603257F23304629462C
:101360002A46FAF745FF3046FBF7EAF802273846E7
:10137000FBF774FD30463146FCF7C2FD03A2384648
:101380002946FEF7BDFD204601B0F0BD7577625FCE
:101390006F70656E0D0A0000F0B581B016460091C1
:1013A0000446002001273946FCF7D2FFEFF31085F1
:1013B0003D4002D1EFF3108072B627204001704308
:1013C0000A21EEF787FE0246002C02D00020009989
:1013D00001E002200021FBF7B9F80446FBF780F991
:1013E000002D00D162B6204601B0F0BD70B50446B4
:1013F0000E4D29680F2001400629FAD029680140C6
:10140000072912D10120EFF31086064002D1EFF335
:10141000108072B6FCF770FDFA30A860002C01D085
:10142000FAF7E0FE002E00D162B670BD0004004065
:10143000F0B581B01D460E460446022A09D10127A7
:1014400038463946FCF784FF009600223846294684
:101450000FE0174601200021FCF77AFF012F04D18D
:10146000009600202946024603E000960220002153
:101470000A462346FBF74CF90446FBF731F92046B0
:1014800001B0F0BD70B5002801D0012070BD03256A
:10149000A9020F4802680F4B5350002494600122A8
:1014A00053030D4E3360BFF34F8FBFF36F8F0B4E5F
:1014B000336003685A50847204811020F8F7BAFA36
:1014C000022007A22946FEF71BFD204670BDC0463C
:1014D0008C95010251E5CC1A80E100E080E200E049
:1014E00057445420636C6F73650D0A000FB47CB5CC
:1014F0000C0009AD01D0611E00E0002101910090B7
:10150000074B6A462946089800F012F9002C02D0D1
:10151000009A002111707CBC08BC04B01847000080
:10152000691E01007CB51D4616460C0001D0611EE7
:1015300000E0002101910090054B6A4629463046A3
:1015400000F0F6F8002C02D0009A002111707CBD4A
:10155000691E01002021020C01D010211046020A50
:1015600001D010460839020901D01046091F82082F
:1015700001D01046891E420801D0881E7047081A03
:1015800070470000004870470890010202E008C858
:10159000121F08C1002AFAD170477047002001E0ED
:1015A00001C1121F002AFBD170470000F0B51FB423
:1015B00086B00998089A030D0021024314D05148BF
:1015C000514A1818504305141198012810981AD040
:1015D000281A401C00264D4F4D4900960191049059
:1015E000002812DA444211E01198012449A301288D
:1015F00001D11098C1430698119A84600360C260BB
:1016000041600BB0F0BD4042E4E7044621050020F4
:101610003F4A001C51410391029012E0E00707D0BD
:1016200032463B4601990098EFF71CF80191009073
:1016300032463B4610461946EFF714F806460F4669
:101640006410002CEAD10498039B0028029A09999F
:10165000089806DAEFF706F8019B009AEFF702F810
:1016600005E0EFF767F8019B009AEFF763F804468F
:101670000E460022284BEFF729FC03D80020C04378
:10168000014607E00022254B20463146EEF738FFA1
:10169000EFF7FCFB102409E0002C0ADB0A220023F0
:1016A000EFF726FA079B30321A55641E02460A43AA
:1016B000F2D11122641C079B121B1C19119B012BD8
:1016C00003D0012308430ED10AE0084304D01120BF
:1016D00010900020119077E71098151A6D1E0BE0FE
:1016E0001098824202DD00236D1C03E0824201DA81
:1016F00000236D1E002BEED0069811998260C16008
:1017000030C07EE701FCFFFF104D000000001440D8
:101710000000F03F300000000000F0430000E03F18
:1017200030380A2801D2012070470020704700009D
:10173000FFB597B00646002518E2252877D100248A
:101740002746FD49049400E00443761C32780120CA
:10175000203A90400842F7D130782A280ED0022251
:10176000307801463039092916D804990A2359439B
:10177000303940181443761C0490F1E7189802C8D9
:1017800004911890002904DA0120400304434842E0
:10179000049002200443761C30782E2814D10420B3
:1017A00004437078761C2A2809D11898761C80C8C2
:1017B000189009E00A214F43303FC719761C307852
:1017C000014630390929F5D930786C2810D006DC6B
:1017D0004C281AD068280ED06A2817D104E0742843
:1017E00013D07A2812D110E00120400504430CE008
:1017F0000121090501E0032109050C4371788142AB
:1018000003D1012000052418761C761C3078119035
:1018100066280BD013DC58287DD009DC00287BD04B
:101820004528F6D04628F4D047281AD1A5E118E07B
:10183000632835D0642870D0652812D19DE17028C6
:101840006CD008DC6728F1D069287BD06E280DD0D9
:101850006F2806D1BAE073282ED0752871D0782869
:1018600059D01A9A199990476D1C7EE16002400F79
:10187000022809D003280DD00428189801680DD03B
:101880000D60001D189070E11898EA1701680D604E
:101890004A60F6E7189801680D80F2E70D70F0E7EE
:1018A00018986A4601781172001D18900020507235
:1018B00002A80090012005E0189802C818900020A6
:1018C0000091C04361070DD5002101E00199491C39
:1018D0000191B94212DA8142F8DB009A515C002989
:1018E000F4D10BE0002101E00199491C01918142F2
:1018F000FADB019A0099895C0029F5D101990498D5
:101900001A9B471A21463846199A00F097FA01990E
:10191000401945180BE04FE02CE113E04EE0009831
:1019200000990078491C00911A9A199990470198DA
:10193000401E0190401CF2D1214638461A9B199A4C
:1019400010E137E00A200021009001916002410F70
:10195000022907D0189A01CA1892C217944603297F
:1019600008D00AE01898C01DC108C90005C918911F
:10197000944607E000B2C2179446042902D140B24F
:10198000C1178C4600226146944506DA0A460021BA
:10199000404291418C462D2102E0210504D52B21A6
:1019A0006A461173012103E0E10701D02021F7E726
:1019B000029155E00A200AE0102008E01020009073
:1019C0000021042004430191082703E0082000219E
:1019D000019100906002410F022907D0189A01CAB4
:1019E000189200229446032908D008E01898C01DD8
:1019F000C108C90005C91891944603E080B20429C2
:101A000000D1C0B200210291210729D51199702976
:101A100006D0009A1021019B4A401A4305D00EE0DF
:101A200040216A461173012108E06146014306D056
:101A300030216A4611731199517302210291009A63
:101A40000821019B4A401A430AD16146014301D152
:101A5000610705D530216A46117301217F1E02916D
:101A60001199582904D035A10E910DA90D910DE0C1
:101A700037A1F9E76146019B009AEFF739F80E9B11
:101A80008C469B5C0D9A521E0D9213706146014369
:101A9000F0D10D9805A9081A20300190600703D5F0
:101AA00001200004844300E001270198874201DD02
:101AB000381A00E000200199009041180298091896
:101AC0000498401A0490E00306D421461A9B199A00
:101AD000049800F0B3F94519002706E003A81A9A04
:101AE000C05D199990476D1C7F1C02988742F5DBF9
:101AF000E0030CD521461A9B199A049800F09EF930
:101B0000451904E01A9A3020199990476D1C0099E4
:101B1000481E00900029F5DC08E00D980D9900782A
:101B2000491C0D911A9A199990476D1C0199481EEC
:101B300001900029F1DC63E10928010030313233E2
:101B400034353637383961626364656600000000F9
:101B500030313233343536373839414243444546E3
:101B60000000000000F05AF94519761C3078002872
:101B700000D0E2E528461BB0F0BD600700D4062780
:101B80001898C01DC108C90048680A680831C30F09
:101B9000DB071891190001D09CA108E0210501D5AF
:101BA0009BA104E0E10701D09AA100E09AA14300C3
:101BB00011985B08109165280CD006DC452809D0E7
:101BC00046281DD0472841D141E0662818D0672813
:101BD0003CD13CE00021112F01DB112000E0781CFA
:101BE0000191009008A911A8FFF7E0FC1399059155
:101BF0000021119A15927F1C12980197009150E0D4
